:020000040800F2
:1000000000800020C1F700083D040108013C000801
:100010003F040108410401084304010800000000F6
:10002000000000000000000000000000912C00080B
:100030004504010800000000212D0008652D00087E
:1000400047040108490401084B0401084D04010854
:100050004F04010851040108D1030108D703010826
:10006000DD030108E3030108E90301085304010863
:100070005504010857040108590401085B040108EC
:100080005D0401085F0401086104010863040108BC
:10009000650401086704010869040108EF03010809
:1000A0006B0401086D0401086F0401087104010864
:1000B0007304010875040108770401087904010834
:1000C0007B0401087D0401087F0401088104010804
:1000D00083040108110C01085D1001088504010862
:1000E00013040108BD0401088704010889040108FC
:1000F0008B04010800000000000000000000000068
:1001000000000000000000005FF808F110B5054C89
:10011000237833B9044B13B10448AFF300800123B3
:10012000237010BD18030020000000001CEE010821
:1001300008B5034B1BB103490348AFF3008008BD6A
:10014000000000001C0300201CEE010808B5034855
:100150000BF0B6F8BDE8084010F0B0BFB69D01083E
:1001600010F0ACBF10B50446C06910B101210AF00F
:10017000DDF9206910B101210AF0D8F9204610BD3F
:10018000F8B50025C0E901120570C0E90335C0E9E2
:100190000555C0E90755456206990446164600F123
:1001A0001C0704F0EFF838B9314607480BF088F81F
:1001B0002021064803F0A2FC069A3946204604F0A6
:1001C000ABF82046F8BD00BFD49D0108FF9D010893
:1001D000F8B50025C0E901120570C0E90335C0E992
:1001E0000555C0E90755456206990446164600F1D3
:1001F0001C0704F01BF838B9314607480BF060F8CB
:100200002021064803F07AFC069A3946204603F07E
:10021000F6FF2046F8BD00BFD49D0108FF9D0108F0
:100220002DE9F04100259DF81860C0E90112057024
:10023000C0E90335C0E90555C0E9075545623146B7
:100240000446174600F11C0803F000FF38B9394690
:1002500007480BF035F82021064803F04FFC3246E2
:100260004146204603F0E0FE2046BDE8F08100BF95
:10027000D49D0108FF9D010870B5AAB008F0F8FBF5
:10028000014604460EA808F0F9FE05F0E7F8054619
:100290000EA90BF0B5FE04F111036B632134564B2C
:1002A0002C6304AC554A00930321554B2046FFF7BD
:1002B00067FF2146284605F07DF92046FFF752FFEB
:1002C0004FF416534F4A009302214F4B2046FFF73D
:1002D0007FFF2146284605F06DF92046FFF742FFD3
:1002E00008230126494A00930221494B2046FFF783
:1002F0006FFF2146284605F05DF92046FFF732FFE3
:10030000444B454A00930321444B2046FFF738FFF6
:100310002146284605F04EF92046FFF723FF404BC3
:10032000404A00930321404B2046FFF729FF214616
:10033000284605F03FF92046FFF714FF3B4B3C4AA7
:10034000009303213B4B2046FFF71AFF2146284626
:1003500005F030F92046FFF705FF374B374A009389
:100360000321374B2046FFF70BFF2146284605F0B7
:1003700021F92046FFF7F6FE324B334A0096022160
:100380002046FFF725FF2146284605F013F92046B1
:10039000FFF7E8FE2D4B2E4A314600962046FFF728
:1003A0003FFF2146284605F005F92046FFF7DAFE13
:1003B0000023284A00933146274B2046FFF730FFA1
:1003C0002146284605F0F6F82046FFF7CBFE2846E2
:1003D000224B234A234904F0B1FF234B0493234BC0
:1003E0000593234B0693234B009394E807000623C1
:1003F00005F0C8FA2AB070BD739B01086C9B010818
:10040000589B0108859B0108779B0108A19B010867
:100410008C9B0108D9C90108E99B0108AB9B010825
:10042000159C01081A9C0108F49B0108709C0108A6
:10043000699C0108209C0108DD9C0108D79C0108EB
:100440007E9C0108EA9C01082C9D0108329D010850
:10045000639D0108819D0108689D010861010008F4
:100460008C9D0108B09D010841FD0008C9FC0008F1
:100470004D0100080000080807B5064B8DF807007D
:1004800001220DF10701186809F0BEFE03B05DF806
:1004900004FB00BF34030020A0F14103052B02D868
:1004A000373840B27047A0F16103052B01D85738A7
:1004B000F7E73038C0B20928F3D94FF0FF30704762
:1004C0002DE9F04F89B004F0E3FF037833B14648DB
:1004D0000AF0F6FE3E21454803F010FB4FF49670FB
:1004E0000AF01EF80446C8200AF01AF807466420ED
:1004F0000AF016F80646C8200AF012F83C4D4FF4F0
:100500009671804603A82860079409F076FE00F0F3
:10051000A9F9012109F0BCFB00F0C6F9012107F09F
:1005200075FC34480AF0CCFE334810F05FFBDFF86E
:10053000DC90DFF8DCB0C8223946286809F098FE64
:10054000002819DD4FF0FF32002407F1FF3A1AF8B6
:10055000011F01B3632C2AD80A291CD00D291AD0F7
:100560002029F4D00929F2D00846FFF795FF00288A
:1005700006DA22480AF0A4FE0A2001F0E7FCDAE7D6
:10058000531C1FBF40EA021030554FF0FF320134B8
:1005900008BF0246DBE7013203D019480AF090FE9B
:1005A000EAE7012C01D11748F8E7002CE4D01648FF
:1005B0000AF086FE214630460AF0E8FE48460AF078
:1005C0007FFE00F071F9C823E2B231460093434642
:1005D00007F006FF044658460AF072FE40462146E0
:1005E0000AF0D4FE4846D9E7389E0108599E010812
:1005F00034030020A69E010879040008FA9E010831
:10060000219F01084D9F0108609F010862AC01080D
:100610006C9F010870470000F8B54FF000470026B6
:10062000174CD4E90223BB4208BFB24225D005F0E3
:10063000AFFCD4E902231349013243F100030978E6
:1006400006F0DBF9B94208BFB04204460D4614D0AB
:1006500008F00EFA036E60301B689847A04271EBF9
:1006600005030ADB294620460AF0AAFD0146064892
:100670000AF026FE054B1878F8BD054BFBE700BFD6
:1006800008000020A905002015A001089F460020B1
:100690009C46002010B50020002106F08FFE044685
:1006A00088B14179042905D080290FD00B480AF080
:1006B00007FE01E000F07CFE204607F0C7F90821A4
:1006C000204609F033FF064B187810BD054B027920
:1006D0000168186804F04CFAEEE700BF53A0010867
:1006E0009C460020AC05002038B508F0C1F905464D
:1006F00008F046FB034C6082284608F035FB208258
:1007000038BD00BF0800002008B508480AF0D8FD31
:1007100008F0AEF9036E60301B689847044BC3E9DC
:100720000201FFF7E1FF034B187808BD43A0010861
:10073000080000209C46002038B5114C2368DB07D8
:1007400008D404F0A5FE802201460E4803F074FF91
:10075000012323600C4B0B4A1A60FFF7C5FF08F01A
:1007600087F905461C2009F0BFFE044605F1740117
:1007700007F0EAFE054B1C60054B187838BD00BF3A
:100780003803002048050020AC0500205803002055
:100790009C46002008B508F06BF9BDE8084008F059
:1007A000A1B90000104BD0B51878D0B90F4CD4E9DE
:1007B0000023B3F1004F08BF002A13D008F058F906
:1007C000036E60301B689847D4E90032C61A4FF0B8
:1007D000000361EB0207064AB242BB41B4BF0120ED
:1007E0000020D0BD0120FCE7A80500204800002023
:1007F0004351010008B50B4B1B685B680BB101202E
:1008000008BD094B1B78002BF9D1FFF7CBFF00285F
:10081000F5D1064B186803685B689847003018BF2D
:100820000120EDE7AC0500204C0300205803002018
:100830001FB56123CDE9013101A9039205F0C2FB87
:1008400005B05DF804FB07B58DF8041001A98DF81B
:1008500005208DF8063005F07BFC03B05DF804FB45
:1008600008F006B938B50C4C2368DB0712D408F041
:10087000FFF8054608F0FCF805F1480100F15802C0
:10088000064809F03FF90123054A06490348236059
:1008900015F077F8014838BD440300205C050020BE
:1008A000000000201506000810B5074C2368DB0780
:1008B00008D4FFF7D7FF00F11C01044807F064FAE1
:1008C00001232360014810BD480300208805002053
:1008D0002DE9F04F8BB008F0CBF8044607F0ACFDE3
:1008E000204607F0BFFDFFF7C7FCFA2001F02EFB02
:1008F00004F0CEFD054604F0A3F9284606F008FEF4
:10090000654B664C1A6812F0010F07D108224E2180
:10091000C4E901120A22E26001221A6060492846F5
:1009200004F03CFC5F492060284604F037FC0828AE
:1009300003D0092801D0072869D10026A0605A49B0
:10094000284604F034FC07460146584817F038FBA7
:10095000002861D10523E3605549284604F027FCAF
:1009600007460146534817F02BFB00286ED145235C
:1009700063604FF487734FF00108238284F812807C
:10098000FFF792FF8146454F03AC0FCF0FC43B6882
:100990000DF10C0C09F10C072360BCE80F000FC728
:1009A000236845493B60284604F001FC04460146A3
:1009B000424817F005FB00285BD1C9F80400404904
:1009C000284604F0EBFB431E022B01465ED93D484E
:1009D0000AF076FC01263C49284604F0E8FB3B4B34
:1009E00003A91860002302AA02930AF04FFA0299A1
:1009F000002900F08B8036480AF062FC35480AF086
:100A00005FFC40F2FD11344803F078F881E0334890
:100A10000AF056FC012692E73946314817F0D0FA21
:100A200008B90A2397E739462E4817F0C9FA08B9DA
:100A30000F2390E739462C4817F0C2FA08B914235F
:100A400089E72A480AF03CFC012685E73946284810
:100A500017F0B6FA08B94F238AE73946254817F048
:100A6000AFFA08B94E2383E723480AF029FC012690
:100A70007FE72146214817F0A3FA10B9C9F804808E
:100A80009DE71F480AF01CFC464698E71D4B18706E
:100A90001D480AF015FC9EE73C03002030000020B2
:100AA000859B0108A19B0108E99B01089EA0010804
:100AB0001A9C0108DCA001086C9B0108739B0108CB
:100AC0002C9D010832A10108699C010850030020F7
:100AD00068A1010883A1010896A1010879A0010875
:100AE000D9C90108A2A0010821CA0108A6A00108CD
:100AF000E1A00108159C0108E5A00108669B01081A
:100B00000EA101085403002051A10108002E7FF41A
:100B100075AF284600F042FD04F0BAFC684904F0C5
:100B200023FB08B1FFF7CCFC66480AF0C9FB07F0CD
:100B30009FFF654D06462B68644C13F0010F04D1EE
:100B400005F026FA012320602B6006F16001206881
:100B500005F0E8F820685E4905F0E6F85D4B256889
:100B60001A685D4903A805F0C7F803A9284605F0EF
:100B70001DF95A4D5A4A28705A492068FFF758FE05
:100B8000594A8DF8060059492068FFF751FE8DF843
:100B90000700206806F068F9554A814655492068E3
:100BA000FFF746FE544A834654492068FFF740FE4B
:100BB000534B8246534A5449206806F07DFE534AFF
:100BC000064653492068FFF733FE524A8DF8050068
:100BD00051492068FFF72CFE2A7880464F4920684B
:100BE00006F086FA07464E4D20689DF806302A78B2
:100BF00080F828309DF806109DF80730FFF723FE97
:100C00004B462A789DF807102068FFF71CFE454ADE
:100C10005B46494620681278FFF715FEDFF8109111
:100C200033462A7859462068FFF70DFE33462A7866
:100C30009DF805102068FFF706FE9DF8053099F82D
:100C4000002031462068FFF7FEFD43462A783146F2
:100C50002068FFF7F8FD344A534641462068127871
:100C6000FFF7F1FD3B462A7841462068FFF7EBFD90
:100C70009DF8053099F8002039462068FFF7E3FD1C
:100C8000164A5346394620681278FFF7DCFD5B466A
:100C90002A7851462068FFF7D6FD206805F016FC3B
:100CA00022480AF00DFB01224FF4FA71206805F08A
:100CB000A7FB002000F0C4FE0BB0BDE8F08F00BF22
:100CC000DDA10108E8A1010840030020580500202B
:100CD000950700085003002005A20108A90500207F
:100CE00039070008BCB80108B90D00080AA20108BC
:100CF000350D000815A201080907000820A2010807
:100D0000850F0008F507000827A2010895060008CE
:100D100034A20108190600083DA2010891B8010893
:100D20009C460020A04600209F46002047A20108C4
:100D30004D47002010B51B4C20680368DB699847BD
:100D400007F096FE036E60301B689847164BC3E9A8
:100D500000010AF035FA014614480AF0B1FAFFF72B
:100D600081FD012108F094FFFFF79EFD012107F0AE
:100D70004DF8206800F038FAFFF796FD002107F0E3
:100D800045F8FFF76FFD002108F082FF2068036837
:100D90005B68984710B90122054B1A70054B18780B
:100DA00010BD00BF580300200800002061A2010808
:100DB000A80500209C46002010B5FFF795FC1148BF
:100DC0000AF07EFA104CFFF74DFD012108F060FF9C
:100DD000FFF76AFD012107F019F8206800F004FA16
:100DE000FFF762FD002107F011F8FFF73BFD00213E
:100DF00008F04EFF20680368DB699847034B1878BA
:100E000010BD00BF75A20108580300209C460020B9
:100E10002DE9F04FB2F5827FC9B007468946924668
:100E2000049303D99421554802F068FE40F205135B
:100E3000534528BF53464FF0004405930023002636
:100E40004FF00108CDE902343B6838465B689847AB
:100E5000002800F08E803B68059A1B6906A9384679
:100E600098470528044607D845480AF029FA3B6800
:100E700038469B699847E7E70DF119009DF818502F
:100E80000AF032FBCDE90001E1B28C1F042DE4B27F
:100E90002ED80539C9B24B1DDBB2B8F1000F42D0D4
:100EA000529A9A4515702DD3062D26D8DDE90023D8
:100EB000484602910AF046FB80460299AAEB0803D5
:100EC0008B421DD3033D012D94BF0125002509EB65
:100ED0000800284498BF09F8084022460DF11E0179
:100EE00016F06EF92544EDB2A8445FFA88F80BE0DD
:100EF000072D2146CFD12346CFE74FF00008DDE78D
:100F00000025F1E74FF000083B6838469B69984799
:100F1000049B46449E422CD2DDE900344FF0000889
:100F2000CDE9023490E7049A8B19934221D8529B61
:100F30001B78AB421DD1DDE90223DDE900BC63452E
:100F400008BF5A4515D1049B9B1B9942DCD8033D31
:100F5000012D98BF4FF0010809EB0600404498BFEF
:100F600009F8064022460DF11E0116F029F9A044A9
:100F7000BBE7304649B0BDE8F08F00BF96A101083D
:100F8000FC9F01082DE9F0414F4E88B004460D4604
:100F9000DE22314604A809F00CFA00234B4F8DF8ED
:100FA0000E303B68D3F80480B8F1000F0FD04848EA
:100FB0000AF086F90DF10F032A463146386803F02E
:100FC0008BFB9DF80F3026606371207119E0414E54
:100FD0003778CFB140480AF073F9404A4049136866
:100FE0000968C91A8D4228BF0D464FF0050161718D
:100FF0003C4928BF86F8008019442B4421602571A4
:10100000136008B0BDE8F081FFF7CCFB00283ED0AC
:1010100035480AF055F907F02BFD036E60301B6868
:101020009847324DC5E90001012104A809F0ECF907
:10103000394604A809F0E8F9022104A809F0E4F906
:101040002B4B197809B101211F702A4E04A809F011
:10105000DBF9B6F9121004A809F006FA318A04A8DF
:1010600009F01AFAD5E9002304A809F009FA224B7D
:1010700004A8197809F0C8F904A809F0D0F90546C0
:1010800004A809F0CEF90123256063719DE71B4890
:101090000AF016F9134F0DF10E03194800934FF49F
:1010A00082722B4639460068FFF7B2FE0C4B854230
:1010B00018609DF80E302760637186D2074B25714A
:1010C0001D60012333709CE764030020AC05002001
:1010D000779F01084C0300209D9F010860030020BA
:1010E0005C03002042040020C19F0108480000204A
:1010F000A80500200800002054030020DE9F0108FE
:1011000058030020F7B507F0B3FC0F25044640F65E
:10111000C13707F029FE1D4EB8420CDC01463046AF
:101120000AF0CEF84FF47A700EF0ACFD204607F0CE
:101130001BFE013DF0D1236820469B689847FFF7CE
:1011400091FB0146204607F0BBF9204607F074F9F1
:10115000204607F09FFC002401234FF496720C49AF
:10116000CDE900340B48234600F07CFB0A480AF026
:10117000A7F80A480AF0A4F800F04EFD40F23D211D
:10118000074802F0BBFC204603B0F0BDAEA2010848
:10119000E8A20108D1080008F1A2010804A301088F
:1011A00096A1010810B504462C2109F0BFF920468C
:1011B00010BD0000FF22014B1A707047A9050020E6
:1011C00003463038C0B209280DD9A3F14102052ADF
:1011D00002D8373BD8B27047A3F16102052A01D883
:1011E000573BF7E7FF2070472DE9F04F684CD5B02B
:1011F0004FF49672814609A905A809F0DAF8236828
:101200005A681B689A4205D162480AF059F855B0ED
:10121000BDE8F08FFFF748FB012106F0F7FD2368DA
:101220005D4F5A68D3F80080DFF880B10292029BCC
:10123000434500F0A7803B7858F8044B012B03D1BD
:10124000032105A809F0E0F83B78022B72D10621B2
:1012500005A809F0D9F8DBE9002305A809F010F981
:1012600021794E480AF02CF8217920680AF08EF88E
:101270004B480AF025F8FFF717FB054605A8266836
:1012800094F804A009F0D6F8039005A809F0CEF868
:10129000C0B2039B524631460090284607F0A0F8A2
:1012A0000646014605463F480AF00AF805A809F037
:1012B000C1F831460AF06AF839480AF001F83B787B
:1012C000023B012B0BD8226805A80392257909F06F
:1012D000B1F8052D8246039A30D80025EDB2294693
:1012E00005A809F0ABF83B78012B11D12379032B2A
:1012F00043D90222216805A8114409F067F823792F
:1013000005A8052B8ABF23680021597909F07CF8CC
:10131000D9F8003005A89C6809F083F809A90246AD
:101320004846A04710B9204809F0CAFF05A809F0AF
:101330007AF87CE7032B8ED1072189E7022ECCD9DE
:101340001046294606F002FD421ED2B2F92AC4D840
:101350009AF901200546002A05DA0246FF21504687
:1013600015F056FFBAE7C21C9642B6D302460AF100
:101370000301504615F032FFB0E7002105A809F03F
:101380008BF8BCE7FFF790FA002106F03FFD3EE73F
:10139000B005002035A30108540300205CA3010818
:1013A00062AC01086FA301087EA3010808000020B9
:1013B0002DE9F04FD7B0044604F06AF8524903F023
:1013C000D3FE28B9514809F07BFF57B0BDE8F08F34
:1013D000FFF746FA036E60301B6898474FF4967229
:1013E000CDE902010BA907A808F0E3FF26792768D9
:1013F0003146474809F064FF3146384609F0C6FFD8
:10140000444809F05DFFFFF72DFA012108F040FC88
:10141000FFF74AFA012106F0F9FC0025DFF80491F4
:10142000DFF804A1B54207D26C1C7D5DE4B2022D49
:101430000DD8394809F044FFFFF736FA002106F0CD
:10144000E5FCFFF70FFA002108F022FCBDE7321B94
:10145000D2B2954204D92946304809F031FFEBE772
:10146000042107A808F0D0FFDDE9022307A809F04E
:1014700007F8FFF719FA834607A808F0DBFF059085
:1014800007A808F0D3FF07EB0408C0B2059B2A4663
:1014900000904146584606F0A3FF83460146204887
:1014A00009F00EFF594607A808F0C8FF032D09D020
:1014B000A11C0222394407A808F088FF052D06D890
:1014C000002106E0002107A808F0E6FFF8E798F8F9
:1014D000051007A808F098FFD9F8008007A8D8F8E9
:1014E0000030D3F808B008F09CFF0BA90246404634
:1014F000D84710B9504609F0E3FE2C4407A8E5B2DE
:1015000008F091FF8EE700BF639D0108DFA401088A
:1015100035A5010862AC010845A501087AA50108B6
:10152000C0A5010858030020CEA50108F8B504465F
:101530000E46D0E9002180688B1A9B100133091AEE
:10154000B3EBA10F4FEA83070CD83A4462606FF007
:101550004043216862683068521A03EBA20341F8E5
:101560002300F8BD384609F047FF054618B9692140
:10157000094802F0C3FAD4E900128A4203D0521A91
:10158000284615F02BFE206809F020FF25603D4419
:10159000C4E90155DBE700BF02A601082DE9F04FC1
:1015A0000446C5B00C2008F09FFF00254D4FC0E950
:1015B0000055856038604C49204603F0F8FD4FF037
:1015C0000108834681462C46DFF840A119F8016BDB
:1015D000B8F1000F0BD12C2E00D066B9A9EB0B018E
:1015E000424809F06DFE2821504602F087FA2C2E61
:1015F0002FD0002E54D03046FFF7E2FDFF280346DF
:10160000A9EB0B0209D100903146394809F058FE88
:101610004221504602F072FA009BFF2C08D1354857
:10162000009309F04DFE4621504602F067FA009BF8
:10163000B8F1000F04D01D01EDB24FF00008C5E76E
:101640001D43EDB2631C04AA15554FF00108DCB22E
:10165000BCE71CB32849204608F064FF034640B9A4
:101660000090264809F02CFE3021504602F046FA40
:10167000009B04A918462246019315F0A1FD3A6883
:101680000820009208F030FF019B009A036004716B
:10169000039003A91046FFF749FF1EB1002495E708
:1016A000002CD7D13B68164859681B68154EC91ADB
:1016B000891009F005FE3B68134FD3E90048444503
:1016C0000CD054F8045B384609F0FAFD28682979F3
:1016D00009F05CFE304609F0F3FDF0E745B0BDE8E7
:1016E000F08F00BFB0050020D79C0108A9A3010816
:1016F00043A401087BA4010826EB01082EA40108DD
:10170000A3A4010862AC0108D7A40108E5A301085D
:10171000064A13681968064B19B94FF0FF321A6070
:1017200070471268D268D2685268F8E7B80500209E
:101730006806002010B5044620B940F2F26108485E
:1017400002F0DCF96269074B9A4207D1A06A064BA6
:10175000984203D0B0FA80F0400910BD0020FCE7A9
:101760003AA601088806002070060020F8B51B4B39
:101770001B4E1C68054630680F46043001F037FAEE
:10178000334640B901203168164EC96A3268884034
:1017900022EA000232606A1C07D137B11968124888
:1017A0000431BDE8F84001F0FFB91A6864195460CB
:1017B00007D30E4A10681968BDE8F840043101F0FB
:1017C000FFB90B4A10681968043101F0F9F9094BA7
:1017D0001A68A24288BF1C60F8BD00BFB006002096
:1017E000B40500203806002088060020BC05002033
:1017F000B80500206806002080B5DFF86480144F2B
:10180000144C154E236863B9144B1B68012BF8D98F
:101810004FF08053C8F80030BFF34F8FBFF36F8F86
:10182000EEE701F047FAFB68DD68281D01F0DFF9FB
:101830003368013B33602368013B236001F05AFAAF
:10184000286B01F0FBFB284601F0F8FBDAE700BF4C
:101850009C0600202806002024060020C005002049
:1018600004ED00E02DE9F84F4FEA820A8046504629
:101870000D4699460B9E01F055FB0746002800F0E7
:10188000AA805C2001F04EFB0446002800F0A080F6
:10189000076325B94FF45871564802F02FF95246A4
:1018A000A521206B15F0B4FC236BAAF1040A9A441D
:1018B0002AF0070A6B1E04F134020F3513F8011FDA
:1018C00002F8011B09B19D42F8D10A9D4FF0000BAF
:1018D000042D28BF0425271DE562C4E9135B3846A3
:1018E00084F843B001F05DF9C5F1050504F1180075
:1018F00001F057F9C4F854B02461A561646284F81A
:1019000058B04A464146504601F0B0F9206006B151
:10191000346001F0CFF9384B384E1A68DFF818817F
:1019200001321A603268002A58D134601B68012BDA
:1019300025D1334801F02AF9324801F027F932481D
:1019400001F024F9DFF8F490304801F01FF9304D30
:10195000304801F01BF9484601F018F9284601F01B
:1019600015F92D4801F012F92C4801F00FF92C4817
:1019700001F00CF92B4BC3F800902B4B1D60012597
:101980002A4A2B491368086801331360E26A6364CA
:1019900005FA02F3034314200B60194B394600FB90
:1019A000023001F001F901F0A5F9D8F8003063B177
:1019B0003368DA6AE36A9A4207D24FF080521D4BCD
:1019C0001A60BFF34F8FBFF36F8F2846BDE8F88FC3
:1019D000384601F033FB4FF0FF35F6E7D8F800301A
:1019E000002BCCD13368DA6AE36A9A4298BF34603C
:1019F000C5E700BF3AA6010824060020B405002070
:101A0000C0050020D4050020E8050020FC050020CA
:101A10005006002010060020700600209C060020C2
:101A200088060020B8050020BC05002034060020F0
:101A30003806002004ED00E0840600203C0600206B
:101A400070B50446284D01F035F904B92C68261DFF
:101A5000304601F0CCF860B91421E06A234B4143D1
:101A60005B5833B90122224982400B6823EA020302
:101A70000B60A36A1BB104F1180001F0B8F81D4A0D
:101A80001368013313602B68A34220D131461A48F2
:101A900001F08AF8194A13680133136001F02AF93A
:101AA000174B1B6893B12B68A3420FD1154B1B68D2
:101AB00023B140F2B641144802F020F84FF08052B2
:101AC000124B1A60BFF34F8FBFF36F8F70BD104A78
:101AD000206B1368013B136001F0B0FA204601F05F
:101AE000ADFAFFF715FED9E7B4050020C0050020C8
:101AF00038060020340600209C060020280600201E
:101B000084060020300600203AA6010804ED00E01B
:101B100024060020F8B5054620B940F24C5117487C
:101B200001F0ECFF164B1B68AB4220D001F0C2F86D
:101B3000144B6C691F68144B1E6801F0DBF8BC4243
:101B400017D0B44215D0114B9C4208D1AB6A83B96F
:101B500095F85830012B0CBF02200320F8BD0C4B28
:101B60009C4208D0002C0CBF04200120F6E7002086
:101B7000F4E70220F2E70420F0E700BF3AA60108EC
:101B8000B4050020B8050020BC0500208806002010
:101B90009C06002070B5044620B940F21C7119481B
:101BA00001F0ACFF184D2B68A34229D044B301F0DB
:101BB00081F82046FFF7BEFDF0B1261D304601F04A
:101BC00016F801231149E26A086893400343142080
:101BD0000B600F4B314600FB023000F0E5FF2B6835
:101BE000E26ADB6A9A4207D34FF08052094B1A60CF
:101BF000BFF34F8FBFF36F8FBDE8704001F07AB82D
:101C000070BD00BF3AA60108B405002038060020C8
:101C1000C005002004ED00E013B50024174B00942C
:101C200001935022234616491648FFF71BFE012850
:101C300018D100F023FE012814D14FF0500383F394
:101C40001188BFF36F8FBFF34F8F4FF0FF320E4BF2
:101C50001A600E4B18600E4B1C6002B0BDE81040BD
:101C600001F0A8B8013007D140F60401094802B0DC
:101C7000BDE8104001F042BF02B010BD6406002074
:101C80007EA60108F91700086806002084060020D7
:101C9000B00600203AA60108024A13680133136017
:101CA000704700BF30060020014B1868704700BF26
:101CB000B006002008B501F0D5F8014B186808BD42
:101CC000B00600202DE9F84F3A4B1B68002B6AD173
:101CD000394B1C6801341C609CB9384D2B681B685B
:101CE00023B140F66221364801F008FF354B2A68DF
:101CF000196829601A60344A136801331360FFF7CA
:101D000007FD324D4FF0000B2B68314FA34211D924
:101D10003A68304BD16A14224A439A58022A28BFA3
:101D20004FF0010B2C4A1268002A0CBF58460120C4
:101D3000BDE8F88FDFF884A0DFF8A490DAF800207F
:101D400012681AB94FF0FF322A60E1E7DAF8002092
:101D5000D268D66871688C4201D22960D8E706F152
:101D60000408404600F043FFB16A19B106F11800BB
:101D700000F03DFF01224FF0140CF06AD9F800305A
:101D800002FA00F11943134BC9F800100CFB0030A4
:101D9000414600F009FF3868F16AC26A914228BFE3
:101DA0004FF0010BCAE70D4A4FF0000B13680133E7
:101DB0001360B7E730060020B0060020B805002009
:101DC0003AA60108BC0500206C0600206806002029
:101DD000B4050020C0050020B40600202C06002019
:101DE000380600202DE9F8432E4C236823B940F62D
:101DF00068012D4801F082FE00F05CFF2368013B82
:101E0000236024682CB1002400F074FF2046BDE854
:101E1000F883264B1B68002BF5D0254D254EDFF8A7
:101E2000A8801FE0EB680127DC6804F1040904F1D5
:101E3000180000F0DCFE484600F0D9FE1420E26AEB
:101E4000316807FA02F30B4300FB02804946336016
:101E500000F0AAFE184BE26A1B68DB6A9A4201D3C3
:101E6000164B1F602B68002BDCD10CB1FFF750FC28
:101E7000134D2C6844B10127104EFFF723FF00B12A
:101E80003760013CF9D12C600C4B1B68002BBAD099
:101E90004FF080520B4B1A60BFF34F8FBFF36F8F21
:101EA0000124B1E7300600203AA6010824060020EC
:101EB0007006002038060020B4050020B40600207B
:101EC0002C06002004ED00E0C005002038B50C46CB
:101ED000054620B940F2CA41184801F00FFE24B966
:101EE00040F2CB41154801F009FE154B1B6823B1A8
:101EF00040F2CC41114801F001FEFFF7CDFE114B3D
:101F00002A68186814192CBF0121002182422C6014
:101F10000CD961B9FFF766FF38B94FF080520A4B10
:101F20001A60BFF34F8FBFF36F8F38BD09B9A0425E
:101F3000F0D20021201AFFF719FCEBE73AA60108BE
:101F400030060020B006002004ED00E010B5044685
:101F500040B94FF080520D4B1A60BFF34F8FBFF363
:101F60006F8F10BD0A4B1B6823B14FF4A461094861
:101F700001F0C4FDFFF790FE00212046FFF7F6FBBD
:101F8000FFF730FF0028E4D0EBE700BF04ED00E0EE
:101F9000300600203AA60108224B70B51A68224B81
:101FA00012B101221A6070BD204E1A6033681B6B9B
:101FB0001A68B2F1A53F0BD15A68B2F1A53F07D11B
:101FC0009A68B2F1A53F03D1DB68B3F1A53F04D015
:101FD00030683168343101F05DFD154B1C68B4FA8E
:101FE00084F41423E4B2C4F11F046343114DEB588D
:101FF00023B940F68831104801F080FD142202FB1D
:1020000004F3E9184868083340682B44984202FBFF
:10201000045408BF4368486008BF4B606368DB68CE
:102020003360C0E730060020B4060020B40500206D
:1020300038060020C00500203AA6010870B5044605
:102040002A4E00F037FE04B93468251D284600F0FA
:10205000CEFD60B91421E06A254B41435B5833B98A
:102060000122244982400B6823EA02030B60A36A21
:102070001BB104F1180000F0BAFD29461E4800F01B
:1020800093FD94F858301D4D012B04BF002384F8B4
:10209000583000F02FFE2A682AB100F00BFEFFF73F
:1020A00037FB00F027FE3368A34211D12B6883B1C0
:1020B000134B1B6823B14FF4D961124801F01EFD88
:1020C0004FF08052104B1A60BFF34F8FBFF36F8FEA
:1020D00070BD094A11680D4A1268914201D13360FE
:1020E000F6E7BDE87040FFF757BF00BFB40500201A
:1020F000C005002038060020880600208406002045
:10210000300600203AA6010804ED00E02406002075
:1021100038B50D46044620B940F69F31074801F016
:10212000EDFC074B20461968183100F049FD2846A0
:10213000BDE838400121FFF719BB00BF3AA60108EE
:10214000B405002070B50E461446054620B940F689
:10215000CA310A4801F0D2FC094B284619681831E7
:1021600000F022FD002C214608BF3046BDE870403B
:1021700018BF4FF0FF30FFF7F9BA00BF3AA60108C9
:10218000B405002038B5C368DC6824B940F6FA31DC
:10219000154801F0B3FC04F11805284600F027FDAE
:1021A000124B1B68E3B9251D284600F020FD0123D2
:1021B0000F49E26A08689340034314200B602946E4
:1021C0000C4B00FB023000F0EFFC0B4BE26A1B688B
:1021D000DB6A9A4285BF0120084B0020186038BD99
:1021E00029460748EFE700BF3AA60108300600205D
:1021F00038060020C0050020B4050020B4060020E9
:1022000070060020034B1B680360034B1B68436090
:10221000704700BF6C060020B006002070B50C4669
:10222000054620B940F66541144801F067FC24B921
:1022300040F66641114801F061FC00F03BFD104B97
:10224000196823685A1C10D00E482E6800686A6806
:10225000864201D08A420FD9881A83420AD95B1A72
:10226000134423602846FFF7CDFF002400F042FD11
:10227000204670BD002323600124F7E73AA6010839
:10228000B00600206C0600200122014B1A60704746
:10229000B406002070B50C461646054608B91B4A20
:1022A000156805F134026260EA6A052B22612A6B27
:1022B0002560E2616A6CA260EA6C62614FF0000224
:1022C000A26119D011490968A94209D12273D6B176
:1022D0000023296BCA5CA52A13D09B08238470BDF8
:1022E000032B2373F3D1FFF7D7FCAB6A0BB10223A7
:1022F0002373FFF777FDEAE72846FFF70BFC20730F
:10230000E5E70133E6E72684E9E700BFB4050020EE
:1023100008B9064B1868026B0020135CA52B02D08D
:10232000C0F38F0070470130F7E700BFB40500200D
:10233000014B1868704700BFB4050020054B1B68AF
:1023400033B1054B1B68002B0CBF022000207047E7
:102350000120704784060020300600202DE9F0415E
:102360000446002836D0234AC36A11681746C96A52
:102370008B4237D2142682691F4D002AA8BF3A68C3
:1023800006FB0353A2BFD26AC2F105028261426911
:102390009A4221D100F10408404600F028FC174B76
:1023A00048B9E06A4643AA592AB901211A6881400E
:1023B00022EA01021A603A681968D26AE2620124CC
:1023C00004FA02F0084318601420414600FB025052
:1023D00000F0EAFB204603E03B68DB6AC3620120B1
:1023E000BDE8F0811368C06CDC6AA0422CBF0020FD
:1023F0000120F5E7B4050020C005002038060020C4
:10240000F8B5044608B90020F8BD1F4B1B6883428D
:1024100004D040F67A711D4801F070FB236D23B99A
:1024200040F67B71194801F069FB236DE16AE26CAB
:10243000013B91422365E6D0002BE4D1251D2846BF
:1024400000F0D5FB124E134A50B91421E76A7943C4
:1024500073582BB901201368B84023EA00031360B6
:10246000E36CC3F10501A161E3620124116804FA80
:1024700003F0084310601420294600FB036000F0BD
:1024800093FB2046C0E700BFB40500203AA6010830
:10249000C005002038060020F8B50D460446002887
:1024A00045D0036D23B940F6C971214801F026FBE0
:1024B000E36C9D4238BF1D46E36AAB4237D0236DC3
:1024C000012B34D11B4B1B68A34204D140F6E471AD
:1024D000174801F013FB1426A269E36A002AE5629B
:1024E000A4BFC5F10505A561134D626906FB035341
:1024F0009A421CD1271D384600F079FBE26A0F4C46
:1025000040B95643AB592BB901212368914023EAC6
:102510000103236001231420216893400B432360AF
:10252000394600FB0250BDE8F84000F03DBBF8BD65
:102530003AA60108B4050020C00500203806002096
:10254000044B1A681AB119680A6D01320A651868D5
:10255000704700BFB40500202DE9F0411E4C1E4617
:1025600080460F46154600F0A5FB236893F85830C7
:10257000022B14D0012123685A6D22EA08025A6501
:10258000236883F8581056B13046FFF7EFF84FF044
:102590008052124B1A60BFF34F8FBFF36F8F00F062
:1025A000A9FB00F087FB15B123685B6D2B602368E6
:1025B000002293F85830022B09BF0125002523681B
:1025C000596D04BFB9435965236883F8582000F05A
:1025D00091FB2846BDE8F081B405002004ED00E041
:1025E000F8B50E4617461D46044620B941F219219A
:1025F0002B4801F083FA00F05DFB0DB1636D2B6099
:10260000022394F8585084F85830EDB2042F16D8AD
:10261000DFE807F00A0307051100636D1E436665D6
:1026200002E0636D01336365012D11D0012400F0D8
:1026300061FB2046F8BD022DF1D10024F7E7636D60
:102640000133F1D041F24A21154801F057FAEBE786
:10265000261D304600F0CBFA1420124AE36A1168B6
:102660009D400D431560104A314600FB032000F0E9
:102670009BFAA36A23B141F25921094801F03EFABD
:102680000A4BE26A1B68DB6A9A42CFD94FF080524C
:10269000074B1A60BFF34F8FBFF36F8FC6E700BFC2
:1026A0003AA6010838060020C0050020B405002025
:1026B00004ED00E02DE9F843DDF820800E46914658
:1026C0001D46044620B941F28C21354801F016FA26
:1026D00000F0C8FBEFF311874FF0500383F311882C
:1026E000BFF36F8FBFF34F8F0DB1636D2B6002236C
:1026F00094F8585084F85830EDB2B9F1040F16D858
:10270000DFE809F00A0307051100636D1E436665E3
:1027100002E0636D01336365012D11D0012087F361
:102720001188BDE8F883022DF1D10020F7E7636D31
:102730000133F1D041F2CF21194801F0DFF9EBE785
:10274000A36A23B141F2DA21154801F0D7F9154BFC
:102750001B6803BB251D284600F049FA01231249D6
:10276000E26A08689340034314200B6029460F4B2C
:1027700000FB023000F018FA0D4BE26A1B68DB6ABE
:102780009A42CBD90123B8F1000F01D0C8F800302C
:10279000084A1360C2E704F118010748EAE700BFDE
:1027A0003AA601083006002038060020C0050020A7
:1027B000B4050020B40600207006002038B5054698
:1027C00008B9084B1D68002400F074FA95F85830D9
:1027D000022B04BF85F85840012400F08BFA2046F4
:1027E00038BD00BFB4050020F8B50F4C00F062FA08
:1027F0002568ADB90D4F0E4E384600F0C7F930468A
:1028000000F0C4F90B4B2A461F600B4B0C210A2029
:102810001E6000F015FD206010B1084901F0D4F8E9
:10282000BDE8F84000F066BAEC060020C0060020C3
:10283000D4060020B8060020BC06002083A60108AC
:10284000914208B5416000610AD8D21A83699A4260
:102850000DD2084B011D186800F0B2F9002008BD28
:102860009A4201D2994202D2011D034BF3E70120A3
:10287000F5E700BFBC060020B806002007B5FFF74B
:10288000B3FF0C4B1B6843B90B484FF4897101F03F
:1028900035F9002003B05DF804FB084BC822019312
:1028A00001230749009307480023FEF7DBFF0028B8
:1028B000EAD0EFE7EC06002088A60108F006002029
:1028C000CDA60108E12900082DE9F04180462C2021
:1028D0000D4617461E4600F025FB044688B125B973
:1028E0004FF4B671084801F009F9FFF77DFF069B28
:1028F000C4F80080C4E9065726626362201D00F018
:1029000050F92046BDE8F08188A601082DE9FF4175
:102910000D4690461F46064620B94FF4C3710F4836
:1029200001F0ECF80E4C206878B1052DCDE9015886
:1029300003960DDCFFF702FD002302280CBF0A9A64
:102940001A4601A9206800F09FFC04B0BDE8F081A0
:1029500000233A4601A900F04DFDF6E788A60108DC
:10296000EC0600202DE9F74300271A4DDFF86C80B4
:102970002B681A6832B9184A11681360296003B0CD
:10298000BDE8F083DB68DC681E6804F10409484692
:1029900000F02DF9636A20469847E369012BE7D1DF
:1029A000A36933449E4206D2636024614946286885
:1029B00000F006F9DCE7002300973246194620466E
:1029C000FFF7A4FF0028D3D140F27231404601F056
:1029D00095F8CDE7B8060020BC06002088A60108BF
:1029E0002DE9F04F4FF00108624D87B0DFF898B144
:1029F000DBF80020136843B30024D368D3F80090B9
:102A0000FFF74AF9FFF750F95B4B82461A681F46F9
:102A100090425A4E1CD31860002C4BD0584B1B6868
:102A20001A68B2FA82F25209A9EB0A01306801F081
:102A300007F8FFF7D7F990B94FF08052514B1A6061
:102A4000BFF34F8FBFF36F8F09E001249946D7E79B
:102A5000FFF788FF484BC3F800A0FFF7C3F9002237
:102A600003A9306800F06AFD0028BFD0039B002B4B
:102A7000F5DB059C636913B1201D00F0B8F8FFF782
:102A800013F93B688146984201D2FFF76BFF039B25
:102A9000C7F80090092BE2D808FA03F313F4047A7C
:102AA00057D113F0C70F33D19B06D8D5204600F07D
:102AB000C5FAD4E7814529D8FFF794F9DBF800304F
:102AC000DB68D3F80CB00BF1040000F090F8DBF8F1
:102AD0001C30012B15D1DBF818104B4652464944E7
:102AE0005846FFF7ADFE60B1009423464A462146A2
:102AF0005846FFF70BFF20B94FF4F471284600F059
:102B0000FDFFDBF8243058469847A8E722468BE7BC
:102B1000A169049B4A4619442046FFF791FE00280C
:102B20009DD0636A20469847E369012B97D1A2693B
:102B30000499CDF800A00A44534651462046FFF7B9
:102B4000E5FE00288BD140F20131284600F0D6FF87
:102B500085E7049BA36123B94FF44671284600F032
:102B6000CDFFA1694B464A4649442046FFF768FE1F
:102B700075E700BF88A60108E8060020EC060020E3
:102B8000BC06002004ED00E0B80600204FF0FF3244
:102B900000F108034360C0E90223036100230360DE
:102BA000704700230361704743689A684B608A60EE
:102BB0009A68516099600368086101330360704747
:102BC0000A6830B5531C0AD103695A684A6091609B
:102BD0008B605960036808610133036030BD00F108
:102BE00008035C6825689542EFD82346F9E7036936
:102BF000D0E901128A6051605968814208BF5A6069
:102C0000002202611A68013A1A60186870470000D1
:102C100006480068006880F3088862B661B6BFF3B2
:102C20004F8FBFF36F8F00DF00BF000008ED00E0A3
:102C3000002307B501930B4B1B68013303D0CA2156
:102C4000094800F05BFF4FF0500383F31188BFF396
:102C50006F8FBFF34F8F019B002BFCD003B05DF84B
:102C600004FB00BF50000020D5A601084FF0807380
:102C700040F8043C054B21F0010140F8081C40F8E5
:102C80000C3C40F8202C4038704700BF312C000825
:102C9000074B19680868B0E8F00F80F30988BFF3A4
:102CA0006F8F4FF0000080F311884EF00D0E7047CB
:102CB000B40500204FF0500383F31188BFF36F8FEA
:102CC000BFF34F8F084A13680133012B136009D1FA
:102CD000064B1B6813F0FF0F04D040F27511044837
:102CE00000F00CBF704700BF5000002004ED00E072
:102CF000D5A6010810B5074C236823B94FF4BE715F
:102D0000054800F0FBFE2368013B23600BB983F309
:102D1000118810BD50000020D5A601080000000059
:102D2000EFF30980BFF36F8F0D4B1A6820E9F00FA6
:102D300010602DE908404FF0500080F31188FFF734
:102D40002BF94FF0000080F31188BDE808401968A6
:102D50000868B0E8F00F80F30988BFF36F8F704701
:102D6000B405002008B54FF0500383F31188BFF37A
:102D70006F8FBFF34F8FFEF7A5FF18B14FF0805252
:102D8000024B1A60002383F3118808BD04ED00E0B4
:102D90000022054B05491A600A6041F26701044AA6
:102DA000116007221A60704710E000E018E000E0B0
:102DB00014E000E013B5254B254C1A78D2B20192ED
:102DC000FF221A701B78234ADBB28DF803309DF87E
:102DD000033003F0500313700723002223609DF893
:102DE0000310581E090628D412B1032B236004D007
:102DF0004FF49B71184800F081FE2368134A1B02B0
:102E000003F4E06323600024019BDBB21370134BD7
:102E10001A6842F470021A601A6842F070421A602E
:102E2000FFF7B6FF0E4B1C60FFF7F2FEFFF7B4F89A
:102E3000FFF7FEFE204602B010BD9DF803300122D0
:102E40005B00DBB28DF803300346C8E700E400E026
:102E5000F8060020F4060020D5A6010820ED00E0C9
:102E60005000002008B5EFF305830F2B0AD90D4A57
:102E70009B5C0D4A12789A4204D940F2A5210B4876
:102E800000F03CFE0A4B0B4A1B68126803F4E06337
:102E9000934206D9BDE8084040F2B521034800F04E
:102EA0002DBE08BDF0E300E0F4060020D5A6010821
:102EB0000CED00E0F806002010B50F4B1A688242B6
:102EC00018D35C681919884201BF4168184609196E
:102ED0005960446801198A4207D1084909688A4241
:102EE0001FBF51681268091941609842026018BFFB
:102EF000186010BD1346E1E70C430020FC060020DB
:102F000038B5064B064D1C68246804B938BD630704
:102F1000FAD07921284600F0F1FDF5E70C430020B6
:102F20002DA701082DE9F8430746FEF7B5FE3B49FA
:102F30003B4D0B68D3B93B4B3B4A58074FF0000061
:102F40001CBF073323F0070313605060374A22F099
:102F50000702C2E90000D01AC3E90020344B0A601E
:102F60001860344B18604FF000432B602B681F42F1
:102F700052D1002F41D007F1080462071CBF24F092
:102F800007040834002C47D02A4B1A689846A242FE
:102F900042D3254B1E687268A24202D230680028D4
:102FA00037D10968B14237D01F683168121B102A27
:102FB00007F10807196010D906EB040919F0070F8B
:102FC00003D0D7211C4800F099FD736848461B1BAD
:102FD000C9F804307460FFF76FFF15497268D8F8BC
:102FE000003008689B1A8342C8F8003038BF0B6075
:102FF0002B681343736000233360FEF7F3FE7B07F7
:1030000004D040F217110C4800F078FD3846BDE8B6
:10301000F88333460646BEE70027EEE7FC060020AD
:1030200000430020000700200C430020F84200204D
:1030300008430020044300202DA7010838B50446AA
:1030400070B3184D50F8041C2A68114204D140F2A4
:103050002B11154800F052FD54F8083C23B14FF4F1
:103060009671114800F04AFD54F8043C2A68134256
:1030700016D054F8081C99B923EA020344F8043C1A
:10308000FEF70AFE094A54F8043C1168A4F108004E
:103090000B441360FFF710FFBDE83840FEF7A2BEF7
:1030A00038BD00BF004300202DA7010804430020C5
:1030B00010B50446FFF7FEFDA46BFFF71BFEB4FA44
:1030C00084F0400910BD70B51546026C0446866B4D
:1030D00042B905689DB98068FFF792F9A56001368D
:1030E000A66370BD6DB9406814F06AF86368226C1D
:1030F0001344A2686360934201D323686360002095
:10310000EDE7C06814F05CF8236CE2685B4221686C
:103110001A448A42E2603EBFA2689B18E360022D17
:10312000EDD10EB1013EEAE73046D8E703461A6C0E
:1031300010B4084662B1D9689C681144A142D960B4
:1031400028BF196810BC28BFD960D96814F038B8F6
:1031500010BC704770B50446FFF7ACFD94F84550BD
:1031600004F124066DB2002D14DCFF2384F84530F1
:10317000FFF7C0FDFFF79EFD94F8445004F11006E0
:103180006DB2002D12DCFF2384F84430BDE870409E
:10319000FFF7B0BD636A002BE7D03046FEF7F2FFC1
:1031A00008B1FFF771F8013D6DB2DCE72369002B30
:1031B000E9D03046FEF7E6FF08B1FFF765F8013DBC
:1031C0006DB2DEE738B50D46044620B940F2031172
:1031D000194800F093FCFFF76DFDD4E90F314B4324
:1031E0002268D0185B1A1344A060E3600020FF231C
:1031F000A063626084F8443084F8453095B923694F
:1032000063B104F11000FEF7BDFF38B14FF08052FA
:103210000A4B1A60BFF34F8FBFF36F8FFFF76AFD42
:10322000012038BD04F11000FFF7B0FC04F12400C8
:10323000FFF7ACFCF2E700BF83A7010804ED00E054
:10324000F8B50D461746064620B94FF4BB710D4838
:1032500000F054FC05FB06F05030FFF763FE044617
:1032600058B165B100F150032360C4E90F65012135
:103270002046FFF7A7FF84F84C702046F8BD0346B0
:10328000F2E700BF83A701082DE9FF4788460192B6
:103290001E46044620B940F2F1214B4800F02EFCB6
:1032A000B8F1000F06D1236C23B140F2F221464859
:1032B00000F024FC022E07D1E36B012B04D040F276
:1032C000F321414800F01AFCFFF738F830B9019BB0
:1032D00023B140F2F6213C4800F010FC0027B9462B
:1032E000DFF8E8A0FFF7E6FCA26BE36B9A4201D39C
:1032F000022E19D1324641462046FFF7E4FE636AAA
:103300001BB104F12400FEF73DFF38B14FF08052AD
:103310002E4B1A60BFF34F8FBFF36F8FFFF7EAFC9E
:10332000012004B0BDE8F087019D1DB9FFF7E2FC64
:103330000020F6E717B902A8FEF764FFFFF7DAFCF2
:10334000FEF7AAFCFFF7B6FC94F84430FF2B08BF49
:1033500084F8449094F84530FF2B08BF84F84590DA
:10336000FFF7C8FC01A902A8FEF758FF28BBFFF72A
:10337000A1FCA26BE36B9A420ED1FFF7BBFC019953
:1033800004F11000FEF7C4FE2046FFF7E3FEFEF74F
:1033900029FD48B10127A5E7FFF7ACFC2046FFF760
:1033A000D9FEFEF71FFDF5E74FF08053CAF8003055
:1033B000BFF34F8FBFF36F8FECE72046FFF7CAFED6
:1033C000FEF710FDB4E700BF83A7010804ED00E09D
:1033D00010B5024600210120FFF732FF044638B144
:1033E000002383600360C3601A461946FFF74CFF51
:1033F000204610BD2DE9F843894690461F460446F5
:1034000020B940F2C331274800F078FBB9F1000F32
:1034100006D1236C23B14FF47171224800F06EFB8A
:10342000022F07D1E36B012B04D040F2C5311D48B8
:1034300000F064FBFFF716FDEFF311864FF0500329
:1034400083F31188BFF36F8FBFF34F8FA26BE36BD2
:103450009A4201D3022F22D194F845503A466DB2D8
:1034600049462046FFF72FFE6B1C13D1636A0BB948
:1034700001200BE004F12400FEF784FE0028F7D0C1
:10348000B8F1000FF4D00120C8F8000086F31188CD
:10349000BDE8F88301356DB284F84550E8E70020B7
:1034A000F4E700BF83A7010870B50D46044620B9B4
:1034B0004FF48C61204800F021FB236C23B140F2D3
:1034C00064411D4800F01AFB236833B9A36823B197
:1034D00040F26941184800F011FBFFF7C3FCEFF31D
:1034E00011864FF0500383F31188BFF36F8FBFF342
:1034F0004F8FA26BE36B93421CD994F84530013295
:103500005BB2A2635A1C10D1636A0BB9012009E0B7
:1035100004F12400FEF736FE0028F7D0002DF5D088
:103520000120286086F3118870BD01335BB284F8F6
:103530004530EBE70020F5E783A701082DE9F043CC
:1035400085B00F460192044620B94FF4A06142486D
:1035500000F0D4FA37B9236C23B140F204513E484D
:1035600000F0CCFAFEF7EAFE30B9019B23B140F23D
:103570000951394800F0C2FA0026B046DFF8DC9065
:10358000FFF798FBA56BD5B139462046013DFFF703
:10359000CDFDA563236963B104F11000FEF7F2FDD0
:1035A00038B14FF080522D4B1A60BFF34F8FBFF3ED
:1035B0006F8FFFF79FFB012005B0BDE8F083019DF1
:1035C0001DB9FFF797FB0020F6E716B902A8FEF732
:1035D00019FEFFF78FFBFEF75FFBFFF76BFB94F81D
:1035E0004430FF2B08BF84F8448094F84530FF2B0B
:1035F00008BF84F84580FFF77DFB01A902A8FEF70C
:103600000DFEF0B92046FFF753FDA0B1019904F17A
:103610002400FEF77DFD2046FFF79CFDFEF7E2FB50
:1036200038B94FF08053C9F80030BFF34F8FBFF364
:103630006F8F0126A4E72046FFF78CFDFEF7D2FB33
:10364000F7E72046FFF786FDFEF7CCFB2046FFF7A5
:103650002FFD0028EDD0B6E783A7010804ED00E0B8
:103660002DE9FF410446019120B940F291515248A1
:1036700000F044FA236C23B140F295514E4800F01B
:103680003DFAFEF75BFE30B9019B23B140F29A513F
:10369000494800F033FA00252F462E46DFF81C81FA
:1036A000FFF708FBA36BE3B1013BA363236813B9E6
:1036B000FEF746FFA060236963B104F11000FEF736
:1036C00061FD38B14FF080523C4B1A60BFF34F8F11
:1036D000BFF36F8FFFF70EFB0125284604B0BDE84E
:1036E000F081019B4BB925B140F2E151324800F025
:1036F00005FAFFF7FFFA0025EFE717B902A8FEF772
:1037000081FDFFF7F7FAFEF7C7FAFFF7D3FA94F84F
:103710004430FF2B08BF84F8446094F84530FF2BF9
:1037200008BF84F84560FFF7E5FA01A902A8FEF793
:1037300075FD40BB2046FFF7BBFCF0B123683BB9E9
:10374000FFF7B8FAA068FEF709FE0546FFF7D2FAC0
:10375000019904F12400FEF7DBFC2046FFF7FAFC98
:10376000FEF740FB38B94FF08053C8F80030BFF384
:103770004F8FBFF36F8F012792E72046FFF7EAFCD8
:10378000FEF730FBF7E72046FFF7E4FCFEF72AFBE5
:103790002046FFF78DFC0028EDD0002D9DD0FFF7CF
:1037A00089FA616A19B1236B1968C1F10501A06832
:1037B000FEF772FE9DE700BF83A7010804ED00E05D
:1037C0002DE9F04385B00F460192044620B94FF42D
:1037D000CD61424800F092F937B9236C23B140F231
:1037E0006C613E4800F08AF9FEF7A8FD30B9019BF4
:1037F00023B140F27161394800F080F90026B046EB
:10380000DFF8DC90FFF756FAA36BD3B139462046B8
:10381000E568FFF78BFC636AE56063B104F124009F
:10382000FEF7B0FC38B14FF080522D4B1A60BFF359
:103830004F8FBFF36F8FFFF75DFA012005B0BDE832
:10384000F083019D1DB9FFF755FA0020F6E716B980
:1038500002A8FEF7D7FCFFF74DFAFEF71DFAFFF7B7
:1038600029FA94F84430FF2B08BF84F8448094F878
:103870004530FF2B08BF84F84580FFF73BFA01A9CC
:1038800002A8FEF7CBFCF0B92046FFF711FCA0B16F
:10389000019904F12400FEF73BFC2046FFF75AFC97
:1038A000FEF7A0FA38B94FF08053C9F80030BFF3E3
:1038B0004F8FBFF36F8F0126A4E72046FFF74AFC26
:1038C000FEF790FAF7E72046FFF744FCFEF78AFA86
:1038D0002046FFF7EDFB0028EDD0B6E783A70108EF
:1038E00004ED00E02DE9F84389469046054620B9ED
:1038F00040F2FB61204800F001F9B9F1000F06D158
:103900002B6C23B140F2FC611B4800F0F7F8FFF785
:10391000A9FAEFF311874FF0500383F31188BFF337
:103920006F8FBFF34F8FAC6B1CB395F84460494663
:1039300076B22846FFF7FAFB013C731CAC6313D147
:103940002B690BB901200BE005F11000FEF71AFC02
:103950000028F7D0B8F1000FF4D00120C8F800001B
:1039600087F31188BDE8F883013676B285F84460A4
:10397000E8E72046F4E700BF83A7010810B5044636
:1039800020B940F28A71054800F0B8F8FFF792F9C3
:10399000A46BFFF7AFF9204610BD00BF83A7010855
:1039A00038B5054620B940F2A471064800F0A6F8E3
:1039B000FFF780F9A86BEC6B241AFFF79BF9204600
:1039C00038BD00BF83A70108002330B5064A52F86E
:1039D000335002EBC3041DB942F83310606030BDB0
:1039E0000133052BF3D1FAE7144F0020002310B563
:1039F000084951F83320DC00824206D10021064AF2
:103A000042F833102244516010BD0133052BF0D130
:103A1000FAE700BF184F0020144F002010B50446ED
:103A200020B94FF4F861054800F068F82046FFF728
:103A3000DDFFBDE81040FFF701BB00BF83A7010811
:103A400070B504460D461646FFF734F994F8443035
:103A5000FF2B04BF002384F8443094F84530FF2B3B
:103A600004BF002384F84530FFF744F9A36B2BB95A
:103A70003246294604F12400FEF764FB2046BDE8E7
:103A80007040FFF767BB0000014B1860704700BF34
:103A9000A043002073B5134C064623780D46124A06
:103AA0001BB913780BB172B6FEE701230021137026
:103AB0000E48642213F0ACFB2B4600960C4A64219E
:103AC0000A4814F029FA0B4B1B6803B198470125EB
:103AD000064E304607F038FC72B6074B2570013BA6
:103AE000FDD1F6E780430020144300201643002058
:103AF000DAA70108A0430020FFFF0F00F7B5164C1E
:103B0000064623780D46154A1BB913780BB172B6D9
:103B1000FEE70123002113701148642213F078FBA3
:103B20002B4600960F4A64210D4814F0F5F90E4B10
:103B30001B6803B198470125094E0C4F304607F02A
:103B400003FC384607F000FC72B64FF0FF332570D7
:103B5000013BFDD1F2E700BF814300201543002067
:103B60001643002002A80108A043002011A8010864
:103B70000368DFF888C080B5CCF80030164F436882
:103B8000164E3B608368164D3360C36815492B6041
:103B90000369154A0B604369144C13608369C0695B
:103BA0002360134B1860DCF8000038683068286820
:103BB0000968104812680021226864221B6813F00B
:103BC00027FB23680C4A64210A4814F0A5F9094828
:103BD00007F0BAFBFEE700BF9043002098430020A7
:103BE0009C430020944300207C4300208443002019
:103BF0008843002016430020C7A701088C430020FB
:103C0000074B1B6803B198471EF0040F0CBFEFF37E
:103C10000880EFF309808169004A1047713B000872
:103C2000A043002010B1012106F080BC704708B10C
:103C300007F0E2BB70478068704740687047436890
:103C4000012B08D1D0E90432934204D01878003017
:103C500018BF01207047002070474B6870B5042BD7
:103C600004460E464FF0000304D0C0E900338360E1
:103C7000204670BDD1E90425AD1AC0E90033836048
:103C80002846FFF7D4FFC4E900000544A560D6E943
:103C9000041305460A46934204D012F8016B05F856
:103CA000016BF8E75B1A18446060E1E7426803467D
:103CB000022A06D1D3E904031B1A032B01D907F00A
:103CC00011BC002070474368032B06D1D0E90432B1
:103CD0009A4208BF0023184670470023FBE7000004
:103CE000037870B581680446B3B1284A284807F0C4
:103CF000E7FA6368022B12D12046FFF7D7FF01468F
:103D0000244807F0DDFAE1680B78002B3CD022480C
:103D1000BDE8704007F0D4BA204A2148E7E7032BFA
:103D200005D12046FFF7CFFF01461E48E9E7042BE7
:103D30000ED100251C4ED4E90431C91A8D4205D29A
:103D4000595D304607F0BCFA0135F4E71748D8E76B
:103D5000012B08D12046FFF772FF1549154B0028AB
:103D600008BF1946E1E700250F4ED4E904239B1A4A
:103D70009D4205D2515D304607F0A2FA0135F4E7C5
:103D80000D4807F09DFABEE70C48C1E77C9C01088E
:103D9000B5A80108C9A80108F0A8010863AC01088A
:103DA000BFA8010885AA0108D3A80108D8A801085E
:103DB000AAA80108AFA80108DEA8010862AC0108A2
:103DC000B1F5705F2DE9F84304460F4602D9164855
:103DD00006F06EFB056883685B1B994218D9D0F822
:103DE00004900846FFF723FF06460346A9EB0508A3
:103DF000A94504D015F8012B03F8012BF8E720683A
:103E0000FFF710FF06EB080326603E446360A660E0
:103E100025683DB92846C4E90155FFF703FF284648
:103E2000BDE8F8830120FBE72DA801082DE9F0414A
:103E30000368561A904682680446D21A96420D4686
:103E400014D93046FFF7F3FE07460346A84504D0D1
:103E500015F8012B03F8012BF8E720683E44FFF723
:103E6000E1FEC4E901662760BDE8F0814768481EAD
:103E7000FF1ABE4211D81A469D19A91A002904DD5D
:103E800010F8011F02F8011BF7E7002EA8BF9B19CD
:103E900062689A42E8D06360E6E73D441F44FA1A3C
:103EA000002A04DD10F8012F03F8012BF7E76368FF
:103EB00028461A46804504D010F8011B02F8011B61
:103EC000F8E7A8EB05084344E5E708B509C81B1A5D
:103ED000C3F57050884202D2104606F0E9FA9942C2
:103EE00038BF1946C81805D2B0F5705F28BF4FF427
:103EF000705008BD4FF47050FBE700002DE9F84307
:103F00000C46591C204615461E46FFF759FF8046B1
:103F100078B14FF00003AA1929462046FFF786FF23
:103F2000D4E901639E4207D00023337063680133F4
:103F300063604046BDE8F883104A01212046FFF740
:103F4000C4FF27688146FFF772FE0022F31BC254AC
:103F500005463A46411EB24202F1010304D01078F0
:103F60001A4601F8010FF6E7DB1BEE183846FFF79B
:103F700059FEC4E900564D44A560DAE768A8010877
:103F80001346426810B5032A06D1BDE810400A4620
:103F900000F11001FFF7B2BF8168024807F090F905
:103FA000002010BDF7A801082DE9F041D0E9002359
:103FB0009E1AB14204460D462ED9891B0AD082684A
:103FC000D21A914208D80022194403F8012B8B42DF
:103FD000FBD16360BDE8F081124AFFF776FF8046AF
:103FE000FFF725FE002307460644054406F8013B7B
:103FF000B542FBD1D4E900303A46834204D013F8ED
:10400000011B02F8011BF8E72068FFF70BFEC4E96B
:1040100000754744A760DDE7DCD215449D4218BF18
:104020004560D7E7DBA9010870B50C4601212046A1
:104030001646FFF7C5FE054628B101212046FFF7C9
:10404000B3FF23681E70284670BD0000426808B5A3
:10405000012A06D1BDE808400A4600F11001FFF729
:10406000E3BF8168024807F02BF9002008BD00BFBC
:104070006AA9010810B50C1A134605D0014622465C
:10408000184613F0ABF80346181910BD2DE9F0419E
:104090008368A2EB01081746026804469B1A9845FC
:1040A0000D4614D94046FFF7C2FD06460346AF420F
:1040B00004D015F8012B03F8012BF8E72068FFF76F
:1040C000B1FD26604644C4E90166BDE8F08146685A
:1040D000B61AB04508D839462846FFF7CBFF6368C3
:1040E0008342F2D06060F0E70E4431462846FFF785
:1040F000C1FF636832461946974204D012F8010B9B
:1041000001F8010BF8E7BE1B1E446660DDE7000006
:1041100070B5D0E9043100F110060446C91A3046E2
:10412000FFF74EFE054640B1D4E90712914206D191
:10413000A168064807F0C4F80025284670BD4FF076
:1041400000033046FFF7A2FFF7E700BF82A801088F
:104150002DE9F0418368A2EB010816460268044687
:104160009B1A98450F4614D94046FFF760FD054657
:104170000346BE4204D017F8012B03F8012BF8E7E1
:104180002068FFF74FFD25604544C4E90155BDE8AF
:10419000F0814568AD1AA84508D831463846FFF782
:1041A00069FF63688342F2D06060F0E70D442946FE
:1041B0003846FFF75FFF63682A461946964204D0E7
:1041C00012F8010B01F8010BF8E7751B1D4465603F
:1041D000DDE737B50D4601A8114607F0A1F9042126
:1041E0002846FFF7EDFD044630B14FF0000302AA68
:1041F00001A92846FFF7ACFF204603B030BDFFF70A
:10420000E8BF0000426808B5022A06D1BDE80840B0
:104210000A4600F11001FFF7DCBF8168024807F091
:104220004FF8002008BD00BFA2A90108FFF7EABFB0
:10423000F7B50E4604461046154613F0D3FE00238C
:104240007268C4E90033013AA360032A12D8DFE898
:1042500002F0022A393F2C49284613F0B1FE20B162
:104260002A49284613F0ACFE38B9012221463046CF
:10427000FFF7DAFE204603B0F0BD2549284613F0CB
:104280009FFE20B12349284613F09AFE08B9002268
:10429000ECE7002201A92846019213F0B5FF021CA9
:1042A00018BF0122E2E7002201A92846019313F07A
:1042B000ABFF019B0246AB42DCD021463046FFF704
:1042C00088FFD7E72A462146304600F025F8D1E797
:1042D00010F00106CED1470839462046FFF770FDA1
:1042E0000028C7D039462046FFF75EFEB742C1D04E
:1042F000022105EB460007F0DEF80028BADB236850
:1043000098550136F2E700BFAAA801083DA80108A8
:10431000AFA8010842A80108F0B5436885B0032B97
:104320000D46164615D0014601A8FFF781FFDDE9CD
:1043300001128A420BD04FF000032846FFF7A6FE79
:1043400001240198FFF76EFC204605B0F0BD002463
:10435000F7E7104613F046FE471C39462846FFF79C
:104360002FFD044618B9064806F0AAFFECE74FF007
:104370000003F21931462846FFF758FDE4E700BF75
:1043800048A801080A4600F11001FFF7C5BFF8B5BB
:104390000D461946284616461F46FFF711FD0446EE
:1043A00030B14FF00003F21931462846FFF7D0FE36
:1043B0002046F8BD1346426810B5042A06D1BDE870
:1043C00010400A4600F11001FFF7E1BF8168024882
:1043D00006F076FF002010BD31A901082DE9F0415B
:1043E0000C4690461D46064640B139B1084918466C
:1043F00006F098F8074618B930602060BDE8F081F3
:104400002A46414612F0DCFE37602560F6E700BF21
:1044100026EB010870B5054610460E46144613F00B
:10442000E1FD2246034631462846BDE87040FFF7CD
:10443000D5BF000010B50C4631B1044900F0D0FCE6
:10444000231A5842584110BD0846FCE775AB0108D5
:1044500010B500B121B9064806F032FF002010BDAA
:104460001AB9044AFFF7D6FFF8E70120F7E700BFC3
:10447000F5A9010802AA01082DE9F3410D461646E7
:104480001F46FFF7E5FFB8B10E49222006F04AF8B3
:104490000446A0B13046FFF7CEFB80463046FFF71A
:1044A00012FC13F09FFD3B46CDE90080064A222115
:1044B000204613F031FD286002B0BDE8F08128608D
:1044C000FAE700BF26EB01083CAA01082DE9F843F2
:1044D0000E46984616F8013B02F1FF39037046601C
:1044E000C0F80890044615463D214A46304612F071
:1044F0004BFE074668BB4B46182B28BF1823C4F851
:104500003001A36204F10C05A26A3146284612F07C
:1045100057FE0022A66AA3191A7337B1D4F83021C6
:10452000791C04F12C0012F04BFE0022D4F830313B
:10453000234483F82C202EB12946404600F050FC3D
:10454000C4F83401D4E901120A48BDE8F84306F082
:104550002DBF831B023DED1A182B1A46A8BF182247
:10456000B5F5807F28BF4FF48075A262C4F8305142
:10457000C8E700BF44AA010830B504460D46084B01
:104580009DB00093074A084B642103A813F0C4FCB4
:1045900003AA29462046FFF73DFF1DB030BD00BFEE
:1045A00036AA01082EAA010811AA01082DE9F04334
:1045B0001646642203F10C048FB007468846204655
:1045C0001849ADF8042013F0FBFC70B9336B23B12C
:1045D000154A322101A813F09FFC01AA4146384632
:1045E000FFF718FF0FB0BDE8F08320460F4913F026
:1045F000E7FC0446A0B9736B002BEED00125DFF871
:104600003490736B01A81B5DC5F1320128444A4602
:10461000013413F081FC102C05F10205F1D1DCE727
:10462000034ADBE750AA010855AA010859AA010864
:1046300061AA0108D3A80108016000210273C0E942
:1046400001117047F8B5054617460E4639B332B327
:104650001D49182005F05AFF044670B3C0E90067F1
:1046600000261A4B00F108074361C0E902660661A3
:104670008021384605F05AFED4E90012384605F08C
:1046800093FE1149082005F041FF48B16B68C0E96D
:10469000004603B96860AB6803B15860A860F8BD14
:1046A0000B4806F00DFE0121206805F03FFF1821A0
:1046B0002046BDE8F84005F039BF064806F000FE88
:1046C00001213046F5E700BF26EB01088081828397
:1046D000F8AA010814AB010870B54468054604B394
:1046E000266806F1080005F029FED6E903239A4260
:1046F000C4B216D16B681BB96A210B48FFF7FEF9EB
:104700006868082143686B6005F010FF6B6803B9A7
:10471000AB600121306805F009FF1821304605F033
:1047200005FF204670BD00BF9DAA010810B50446D4
:10473000006810B1012105F0F9FE204610BD7FB5DB
:104740000546FFF778FA13F04DFC0446861C284610
:10475000FFF773FA013803281DD8DFE800F00206DE
:10476000080F0734601C04B070BD0D34FAE728460A
:10477000FFF7A9FA13F036FC3418F3E701A829462D
:10478000FFF76BFADDE9014301A81B1B06EB4304AD
:10479000FFF7CCFFE6E70B34E4E700002DE9F04734
:1047A00086B08146884614461D46FFF751FE68B123
:1047B0002046FFF7C4FF4049074605F0B3FE064612
:1047C000C9F8000028B93D4806F07AFD06B0BDE8FA
:1047D000F0872046FFF731FA0138032864D8DFE874
:1047E00000F00214253D2046FFF725FA81462046B9
:1047F000FFF725FA324B334A002814BF18461046FB
:10480000CDE900902B46304A0AE02046FFF713FA24
:1048100081462046FFF74AFA2B46CDE900902B4A05
:104820003946304613F078FB05463AE0612D2046C4
:104830000DD1FFF700FA05462046FFF744FA2B4654
:10484000234A00903946304613F066FBECE7FFF749
:10485000F2F981462046FFF736FAD1E72046FFF706
:10486000EAF92B4600901B4A3946304613F054FBB8
:10487000DFF868902146054603A8FFF7EEF9DDE969
:10488000034AA2450AD0AF4214F8013B06D9791B6E
:1048900070194A4613F040FB0235F2E703A8FFF710
:1048A00045FFC8F8005091E72046FFF7C4F92B46B2
:1048B0000090094AC6E700BF26EB010814AB0108C7
:1048C000AAA80108AFA8010870AA010878AA0108DF
:1048D00081AA010888AA01088EAA0108D3A80108A4
:1048E0002DE9F0410E4607469046D0B04FF49C7239
:1048F000002102A81D46569C12F08AFC31463B4618
:10490000424602A8FFF7E2FD3678642E5AD01CD842
:104910003F2E44D008D82E2E4BD09DF80810694861
:1049200006F0CEFC684A48E0612E00F09380622ECB
:10493000F3D1664806F0C4FC654806F0C1FC4FF4AC
:1049400093716448FFF7DAF830E0722E45D00CD846
:10495000672EE2D105A9604806F0B2FC33464F9AB3
:1049600021462846FFF71AFF20E0732E50D0772EFD
:10497000D3D15A4806F0A4FC0399002900F09F8087
:10498000574813F01DFB0446002840F09880554816
:1049900006F096FC2146384600F0CAFECCE75248A5
:1049A00006F08EFC21462846FFF7E6FD50B0BDE834
:1049B000F0814E4806F084FC4D4A21462846FFF718
:1049C00029FDF3E703994B4806F07AFC02AB3A461F
:1049D00021462846FFF7EAFDE8E705A9464806F024
:1049E0006FFC0399454813F0EBFA20B9384600F004
:1049F00011F9434AE1E74F993846FFF71BFD08B12B
:104A0000404ADAE74F9808B1FFF782FB7223A6E726
:104A100005A93D480DAA06F053FC4F993846FFF70B
:104A200009FD0028ECD14F9810B10DA9FFF7AAFCA1
:104A300073234F9A21462846FFF7B0FE216833487A
:104A400006F03EFC2868216806F0A0FC304806F01D
:104A500037FCABE70DAF2F483A4605A906F030FC0E
:104A60004F9828B3FFF7E9F8032801D02A4AA4E7B2
:104A70004F98FFF728F913F0B5FA08F101088044C0
:104A80002649404605F04EFD064688B14F98FFF78F
:104A90001AF9234A034641460097304613F03CFA80
:104AA00031464F98FFF76EFC0121304605F03EFD80
:104AB00061234F9A21462846FFF7DEFCBEE701211D
:104AC00069E700BF42AC010864AC0108D4AB01083F
:104AD00075AC0108A1AC01083FAB0108F7AB0108B8
:104AE0001FAC010825AC010819AB010823AB010874
:104AF0002DAB010830AB010850AB01087C9C0108CC
:104B000063AB010866AB010880AB010899AB0108F3
:104B100062AC0108AAAB0108C3AB010826EB01088F
:104B2000CFAB01082DE9F0410C4680460D481546F3
:104B30001E46069F06F0C4FB04B14DB90A4806F0B4
:104B4000BFFB39463046BDE8F041084AFFF762BC7A
:104B5000069733462A4621464046BDE8F041FFF716
:104B6000BFBE00BFE2AC0108F7AC01080AAD010806
:104B70007FB504460D4600680C49164600F0F4FA6D
:104B800078B100F085FC03AB00933246294602ABB6
:104B9000FFF7C8FFDDE902122046FFF753FD04B01E
:104BA00070BD034806F08CFBF9E700BF75AB010848
:104BB000D9AA010810B10C2105F0B8BC704710B19A
:104BC000012105F0B3BC704710B5044638B1FBF7BE
:104BD000C9FA2046BDE81040282105F0A7BC10BD49
:104BE00070B50446406AFFF7E5FFD4E90656AE42C9
:104BF00004D02846FBF7B6FA2835F8E7A56935B1A1
:104C00002846FBF7AFFA2821284605F08FFC2046FE
:104C100070BD0000F8B5054600242826074FD5E9E9
:104C200006031B1ADB107B439C4205D206FB0400E3
:104C3000FFF76EFA0134F2E7F8BD00BFCDCCCCCC63
:104C4000F8B50446224806F03BFB224806F038FB44
:104C5000D4E90631994218D0C91A1F4EC9107143C0
:104C60001E4806F02DFB00252827D4E906031B1A51
:104C7000DB1073439D4205D207FB0500FFF730F8B8
:104C80000135F2E7164806F01BFBD4E90931154E51
:104C9000C91A89107143144806F012FB00250C272D
:104CA000D4E909031B1A9B1073439D4205D207FBED
:104CB000050000F079FF0135F2E70C4806F000FB33
:104CC0000B4806F0FDFABDE8F8400A4806F0F8BACD
:104CD000F1AD010895BF0108CDCCCCCCFBAD0108EE
:104CE0000DAE0108ABAAAAAA46AE010862AC010843
:104CF00056AE01080FA301082DE9F043002487B048
:104D000006466846CDE90044029405F039F9684644
:104D100005F0CEF94FF028082F4F304DD6E9062385
:104D20009B1ADB107B439C424ED208FB04F302EB40
:104D30000309D35C002B43D14846FEF77CFF0146B4
:104D4000684605F0A7F94846FEF777FF042837D8EC
:104D5000DFE800F03803101A24004846FEF76FFF22
:104D60000146684605F04CF950BBC2212846FEF7C3
:104D7000C5FE25E04846FEF799FF0146684605F066
:104D800025F9E8B9C621F1E74846FEF79CFF014640
:104D9000684605F07FF998B9CA21E7E7494603A8B4
:104DA000FEF75BFFDDE903126846521A05F04AF987
:104DB00018B9CF212846FEF7A1FE0398FFF7FFFEA2
:104DC0000134ABE7D321D1E7684605F099F90298A1
:104DD00007B0BDE8F08300BFCDCCCCCC31AD01082D
:104DE0002DE9F04305460E4600244FF028081A4FDF
:104DF0008DB0D5E906239B1ADB107B439C4224D25D
:104E000008FB042931461822684613F005F9484684
:104E1000FEF711FF182201460DEB020013F0FCF81B
:104E2000684606F0ABFB684606F0B8FB06A806F03D
:104E3000A5FB06A806F0B2FB182268460DEB02019E
:104E400013F0D8F818B10134D3E74FF00009484601
:104E50000DB0BDE8F08300BFCDCCCCCC2DE9F04F38
:104E600006460F4600244FF00C09DFF86C808DB029
:104E7000D6E909535B1B9B1008FB03F39C4224D229
:104E800018223946684613F0C7F8182209FB04FBBC
:104E90000DEB020055F80B1013F0BEF8684606F053
:104EA0006DFB684606F07AFB06A806F067FB06A8CD
:104EB00006F074FB182268460DEB020105EB0B0AA5
:104EC00013F098F818B10134D2E74FF0000A5046B9
:104ED0000DB0BDE8F08F00BFABAAAAAA10B514466A
:104EE000FFF77EFF20B12146BDE81040FFF74ABA28
:104EF00010BD0000F8B50C46064640F20112002134
:104F0000224812F085F94FF4807221461F4812F0B2
:104F100057F91E491E4806F0D3F91E491B4813F0E5
:104F2000A5F81C490546002013F0A0F829460746BD
:104F30003046FFF755FFC8B929463046FFF78EFFC8
:104F4000044600B30168144806F0BAF9A36838466D
:104F5000984701242046F8BD104806F0B1F91048E2
:104F600006F0AEF93046FFF76BFEF3E73A46294606
:104F70003046FFF7B3FF04460028EDD13946094813
:104F800006F09EF9E6E729460748F9E7284500209C
:104F90006FAE01088CAA010875AE01088AAE01083F
:104FA00062AC01089EAE0108B7AE010810B54FF41F
:104FB000807204460649043005F05AF9002805DDE0
:104FC0002046BDE810400249FFF794BF10BD00BF66
:104FD0002844002038B514461D46FFF701FF28B1CC
:104FE0002A462146BDE83840FEF7CABF38BD10B595
:104FF0001446FFF7F5FE20B12146BDE81040FFF74B
:1050000001B910BD10B51446FFF7EAFE10B12146F4
:10501000FFF71CF8002010BD38B514461D46FFF7F9
:10502000DFFE28B12A462146BDE83840FFF7C2B965
:1050300038BD00002DE9F04700248CB0074603A8D6
:10504000CDE90344059404F09BFF214603A8009496
:1050500005F0B2F80146002834D0214603A805F037
:1050600034F840F2E7330446009300263546DFF873
:10507000F4A0009BB34271D9214603A805F057F86C
:10508000814600286AD1182321460DEB030203A8AC
:1050900004F0DEFF0444214603A805F056F88046DC
:1050A000B0B1214602AA03A8CDF8089004F06EFF23
:1050B000029A044406A93846FFF799FF00B101356A
:1050C0000136D6E76A4603A805F006F80446CCE7A1
:1050D000214603A805F083F870B102AA214603A86F
:1050E0008DF8088004F07CFF9DF80820044406A990
:1050F0003846FFF787FFE1E7214603A805F040F8AF
:10510000804668B102AB01AA214603A804F0B1FFB2
:10511000DDE90123044406A93846FFF75BFFCDE72C
:10512000214603A805F01EF880B102AB01AA214672
:1051300003A8CDE9018804F074FF9DF80830044409
:10514000019A06A93846FFF767FFB7E7039B504669
:10515000195D01F0E00106F0B3F8B1E728460CB0A4
:10516000BDE8F08780AD010808B5FFF739FE18B13A
:10517000BDE80840FEF763BD08BD10B5044608460B
:105180001146FFF72DFE014620B9C4E90000A060DA
:10519000204610BD2046FEF760FDF9E708B5FFF791
:1051A0001FFE18B1BDE80840FEF780BD08BD08B578
:1051B000FFF716FE18B1BDE80840FEF784BD08BD34
:1051C000037810B5044643B1044806F079F800218D
:1051D000204600F0ADFA0023237010BD6BAD01082E
:1051E000002370B5D1E90025AD1A0446C0E90033AB
:1051F00083600E46284601D006F0FEF8C4E90000A0
:105200000544A560D6E9001305460A46934204D03A
:1052100012F8016B05F8016BF8E75B1A184460603F
:10522000204670BD38B504460D460B78103000F8A6
:10523000103C4B68103140F80C3C51F8083C40F8E9
:10524000083C51F8043C40F8043CFFF7C9FF05F165
:105250001C0104F11C00FFF7C3FF204638BD00000D
:105260002DE9F84FD0E90075EC1BA310304C064631
:105270005C43B4F5705F8946934602D12D4805F032
:1052800017F9002C14BF23460123E418A1EB070AE9
:1052900019D2B4F5705F16D8C4B10C20604306F083
:1052A000ABF880469BE8070008EB0A0383E8070099
:1052B0000023DA1991450BD007CA08EB030C8CE8E0
:1052C00007000C33F5E74FF47054E6E7A046E9E732
:1052D0000C2219494FF000098C464FEA9A034B43C0
:1052E00023F0404302FB037E03FB0223434409EB0C
:1052F0000E02954207D007CA03EB090A8AE80700A5
:1053000009F10C09F3E74FF00C09A5EB0E05AD0808
:105310000CFB05F525F0404509FB053509FB048428
:105320003846FFF747FCC6E90085B460BDE8F88F52
:10533000ABAAAAAA68A80108ABAAAA2A2DE9FF4726
:10534000044608460D4617461E4612F04BFE172827
:1053500003D982212C48FEF7D1FBD4E9099A2B4AC4
:10536000AAEB0908CDE901574FEAA80555430135D5
:10537000B5F5705F039602D9254805F099F8E36A00
:10538000A3EB09039B1053439D4229D90C266E437E
:105390007DB1304606F030F80746002309EB0302E2
:1053A000924508D007CA07EB030C8CE807000C33C2
:1053B000F4E72F46F1E7606AFFF7FCFB07EB080311
:1053C000A362124B67623744B6105E43B542E76290
:1053D00006D9104805F074FF8C210B48FEF78EFBB0
:1053E000D4E90A32934201AA07D007CA83E807002A
:1053F0000C33A36204B0BDE8F087194604F1240021
:10540000FFF72EFFF6E700BF31AD0108ABAAAAAA4D
:105410002DA8010816AD0108002310B5044603703D
:10542000C0E90633C0E90833C0E90A33C0E90C33E8
:10543000064B80214361043004F0DFFE2046044B1C
:10544000044A0549FFF77AFF204610BDA843002013
:1054500095540008DAAE0108E6AE010810B5084C14
:105460002368DB0709D40748FFF7D6FF0123064A64
:1054700006490448236010F084FA024810BD00BFBA
:10548000A44300202C46002000000020E14B00082F
:10549000FFF7E4BF08B5FFF7E1FFBDE80840FFF7FD
:1054A000CFBB0022C0E90022826010B50C68046006
:1054B0000A6042684C6844604A6082688C68846014
:1054C0008A6010BDF8B50F46154600F11004A4F12E
:1054D00010039F4205F128061AD014F8103C21460B
:1054E00006F8283C54F80C3C05F110006B6054F8A9
:1054F000083CAB6054F8043CEB60FFF7D2FF04F1CA
:105500000C0105F11C00FFF7CCFF28343546DEE71F
:105510002846F8BD2DE9F84FD0E90067BC1BE31021
:10552000224C05465C43B4F5705F8846924602D132
:105530001F4804F0BDFF002C14BF23460123E418CC
:10554000A1EB060B22D2B4F5705F1FD80CB3282054
:10555000604305F051FF8146514609EB0B00FFF710
:1055600061FE41464A463046FFF7ACFF394600F13E
:1055700028024046FFF7A6FFB0468246B8450AD04B
:105580004046FAF7EFFD08F12808F7E74FF47054AA
:10559000DDE7A146E0E73046FFF716FB282303FBD3
:1055A0000494C5E9009AAC60BDE8F88FCDCCCCCCB2
:1055B00068A801082DE9F04FD0E906560446884650
:1055C0003B4F8BB0AE421BD029466846FFF72AFE00
:1055D0006846FEF730FB81464046FEF72CFB01464D
:1055E000484606F001F830B14046FEF724FB01467C
:1055F000384605F065FE6846FAF7B4FD2835E1E760
:10560000D4E906AB2B4AABEB0A094FEAE90555434F
:105610000135B5F5705F02D9274804F049FF236AC8
:10562000A3EB0A03DB1053439D422CD928266E437B
:1056300095B1304605F0E0FE0746594650463A46D9
:10564000FFF740FFD4E906ABD34507D05046FAF741
:1056500089FD0AF1280AF7E72F46EEE7A069FFF770
:10566000B3FA07EB0903E361124BA7613744F61065
:105670005E43B542276206D9104805F021FE772126
:105680000F48FEF73BFAD4E90703984208D0414699
:10569000FFF7C8FDE3692833E3610BB0BDE8F08F85
:1056A0000146424604F11800FFF734FFF5E700BF5A
:1056B000A0AD0108CDCCCCCC2DA80108D2AD0108FD
:1056C00031AD01080023042213B50193094B0DEB02
:1056D00002015868084B00F580605B6898470446F3
:1056E00028B1064805F0ECFD204602B010BD044884
:1056F000F8E700BF744600206846002044B1010866
:1057000058B1010808B5084805F0DAFDFFF7A6FE14
:10571000FFF780FA054805F0D3FDFFF79FFEBDE8CF
:105720000840FFF78DBA00BF75B101088DB10108BF
:1057300073B504464FF400700E4605F05DFE054655
:1057400030B91E4805F0BCFD20211D48FEF7D6F9F2
:105750004FF400720021284611F05AFD29462046D8
:105760004FF40072FFF7C8FA164C01460190FEB1E3
:10577000154805F0A5FD646804F58064134E042205
:105780007368104920469847042273680DEB0201A4
:10579000A01898477368019A294604F108009847B1
:1057A0000B4805F08DFD284605F010FE02B070BDD7
:1057B000084805F085FD6468E0E700BFE3AF010835
:1057C000EEAF01087446002036B00108684600209C
:1057D00070B0010855B001082DE9F74FFFF73EFE04
:1057E0002F4F06462F4805F06BFDB846DFF8D090E6
:1057F000DFF8D0A0FCF758FA2B4D38602B68AB4689
:105800002A4C002B37D003F56A436033984232D2DA
:1058100023782BB9264805F053FD264805F050FDA6
:10582000012330462370FFF7C1FB41F28833524613
:105830004FF0FF310020FCF78FFE0190FCF734FAA7
:10584000019BC8F8000023B9237813B13046FFF755
:10585000ADFBDAF80030DA0744BFD8F800202A6040
:105860009B07C7D50023CBF80030D9F80830002BB0
:10587000BED09847BCE723786BB100213046FFF7D4
:1058800057FF0D4805F01CFD0C4805F019FDD9F82F
:10589000083003B19847002323702B60C5E700BF91
:1058A00088460020B4B00108844600207C460020D1
:1058B000C9B00108ECB001080FB1010821B101081D
:1058C000684600208046002010B5FFF7C7FD04465B
:1058D0000021FFF72DFF2046FFF7B2F9BDE8104089
:1058E00003480023012202210068FCF779BE00BFB3
:1058F0006446002010B5FFF7B1FD04460021FFF714
:1059000017FF2046BDE81040FFF79AB92DE9F7438D
:10591000184E0746884675680AB105F5806500246B
:10592000DFF85C90042269460094D9F800302846DC
:105930009847326800998A4204D00F4805F0C0FCAD
:10594000204614E00422D9F800300DEB0201A8181B
:1059500098470199094805F0B3FC019A4245EFD8F0
:10596000D9F80030394605F108009847019803B08E
:10597000BDE8F083744600207FB001089AB00108AA
:105980006846002082B0F0B589B003AC84E8070017
:105990000F93049B23B940F21B116E48FEF7AEF83B
:1059A000039B23B94FF48E716A48FEF7A7F894E879
:1059B0000700694F694E0FAB87E8070093E80300C3
:1059C00086E80300FFF74AFD0446654B654A6649D1
:1059D000FFF7B4FC654B664A66492046FFF7AEFC0C
:1059E000654B664A66492046FFF7A8FC4FF40070F5
:1059F00005F002FD0546002873D04FF40072002127
:105A000011F006FC70683B68042207A900F580606D
:105A10009847002859D03268079B9A4255D1594877
:105A200005F04EFC01224FF400712846FFF76EFF8F
:105A30000646554805F044FCFFF744FE002E40D0D2
:105A400001232370324629462046FFF7F3FA284601
:105A500005F0BCFC2578FDB94FF4007005F0CCFCD6
:105A600006464FF40072294611F0D2FB2A464FF445
:105A700000713046FFF74AFF074600283FD105F086
:105A8000A5FC304605F0A2FC404805F019FCFFF7E4
:105A9000E5FC0021FFF74CFE3D4BFA220193012368
:105AA0003C4900933C480023FBF7DCFE20B94FF44F
:105AB0009D712848FEF722F809B0BDE8F04002B019
:105AC0007047364805F0FCFB267000224FF4007149
:105AD0002846FFF71BFF06460028B3D1284605F0ED
:105AE00075FC2F4805F0ECFB2046FFF793F80023E8
:105AF0002370FFF7E7FD2B4805F0E2FBAAE74FF420
:105B0000007005F079FC054618B981211148FDF7B0
:105B1000F5FF4FF400720021284611F079FB4FF495
:105B2000007229462046FFF7E7F808B92846A6E79D
:105B30008742FBD10023E95CF25C9142F6D101334C
:105B40009F42F8D1284605F041FC304605F03EFC66
:105B5000A2E700BFEEAF01086846002074460020AF
:105B6000F5580008EAAE0108F6AE0108055700082E
:105B7000FBAE010816AF0108C95800081EAF0108A6
:105B800036AF01083BAF01085FAF0108C1AF0108A4
:105B900064460020D8AF0108D957000874AF010847
:105BA0009DAF01088DB1010810B504460168074892
:105BB00005F086FB616831B10B7823B10448BDE87C
:105BC000104005F07DBB0348F9E700BFA5B101080F
:105BD000F0A8010862AC010810B50446C06908B11C
:105BE00005F0F4FB206908B105F0F0FB606808B12E
:105BF00005F0ECFB204610BD10B504460068FDF72B
:105C00000DFF204610BD00001FB5536802931378A6
:105C100001934B6800930B6842680178024805F0D5
:105C20004FFB05B05DF804FBAAB10108C92101488A
:105C3000FDF764BFC8B10108FE2307B58DF8043035
:105C4000054B01A91868002300681A46FDF7D2FB2E
:105C500003B05DF804FB00BF98460020D0B51F4696
:105C60007423C0E9003100230446836008201646EF
:105C700004F03AFCC0E90067A0602046D0BD0000F7
:105C80002DE9D043DDE9066799467223C0E900316A
:105C900000239642836077EB09030446904603DABB
:105CA0002B210748FDF72AFF102004F01DFCC0E956
:105CB0000089C0E90267A0602046BDE8D08300BF2C
:105CC0000AB20108036837B5632B04460D4601D0BC
:105CD000FFF7ACFF002301AAA1682846019305F055
:105CE000D5F8019B1BB138210248FDF707FF03B02F
:105CF00030BD00BF0AB2010870B563230025C0E9BA
:105D00000031044685601A20164604F0EDFB1A2285
:105D1000294611F07DFA3146A0602046FFF7D2FFF8
:105D2000204670BD81647047C16470472DE9F84317
:105D3000D0E90173884600254FF00C09DB1B0A4EA1
:105D40009B105E43ECB2B4420BD209FB0472414695
:105D5000506812F035F901350028F3D12046BDE82E
:105D6000F8834FF0FF30FAE7ABAAAAAA2DE9F8436F
:105D7000D0E90473884600254FF00C09DB1B0A4E5E
:105D80009B105E43ECB2B4420BD209FB0472414655
:105D9000506812F015F901350028F3D12046BDE80E
:105DA000F8834FF0FF30FAE7ABAAAAAA2DE9F04733
:105DB0000E4649680446FFF7B9FFC0B2FF2803D07A
:105DC0007C212C48FDF79AFED4E901232A4F9B1A27
:105DD0009B107B437E2B03D97F212648FDF78EFE47
:105DE000D4E901120C25E068531A9B10121A7B4368
:105DF00092107A430133934205FB03F80ED84144D5
:105E0000A160D4E9013496E80700E31A04E9070029
:105E100019489B1058430138BDE8F087404605F00B
:105E2000EBFA054618B969211448FDF767FED4E975
:105E300001C300274FF00C0AA3EB0C030E4A9B1082
:105E400002FB03F9A9EB0703002B0ADD0AFB07F3AA
:105E500005EB030E634493E8070001378EE8070063
:105E6000F0E7604605F0B2FA65604544C4E90255C2
:105E7000C7E700BF0AB20108ABAAAAAA02A6010896
:105E80001FB56E23CDE90131002301A90393FFF76C
:105E90008DFF05B05DF804FB0023FF2270B54FF0C5
:105EA0000041C0E90033C0E90233C0E90433C0E96E
:105EB0000633C0E9083380F82820044600206FF03C
:105EC0007F42C4E90C01C4E90E014FF0FF31C4E97F
:105ED0001233C4E91012002305221E4DC4E9142315
:105EE0002A6812F0010212D101211B4E08463260CD
:105EF000FDF7A6F9306018B911211848FDF7FEFD2D
:105F00000123174A174914482B600FF03AFD164B2E
:105F10001A680AB9104A1A6014492046FFF7B0FF00
:105F2000134B144918702046FFF7AAFF124B134970
:105F300018702046FFF7A4FF114B12491870204635
:105F4000FFF79EFFFE22104B1870104B20461A7070
:105F500070BD00BF9446002008470020F1B2010840
:105F600000000020F95B0008984600202BB30108D0
:105F7000A046002033B301089E4600203BB3010831
:105F80009C46002040B301089F4600209D4600200B
:105F900010B5084C2368DB0709D40748FFF77CFFDE
:105FA0000123064A0649044823600FF0EAFC024830
:105FB00010BD00BF90460020B04600200000002029
:105FC000D95B00082DE9F0470E4649680446FFF703
:105FD000CDFEC0B2FF2803D087212C48FDF78EFDEF
:105FE000D4E904232A4F9B1A9B107B437E2B03D9B1
:105FF0008A212648FDF782FDD4E904120C25A06908
:10600000531A9B10121A7B4392107A430133934226
:1060100005FB03F80ED841446161D4E9043496E8E5
:106020000700E31A04E9070019489B105843013898
:10603000BDE8F087404605F0DFF9054618B969214B
:106040001448FDF75BFDD4E904C300274FF00C0AA8
:10605000A3EB0C030E4A9B1002FB03F9A9EB070309
:10606000002B0ADD0AFB07F305EB030E634493E8FC
:10607000070001378EE80700F0E7604605F0A6F953
:1060800025614544C4E90555C7E700BF0AB20108C8
:10609000ABAAAAAA02A6010838B5D0E901239B1A27
:1060A000074A9B105343CDB29D42044603D3A62119
:1060B0000448FDF723FD0C20636800FB053038BD64
:1060C000ABAAAAAA0AB2010838B5CCB21149054652
:1060D0000B6813F0010307D10F4A702013720123DC
:1060E00010600E480B605060FF2C10D0D5E90423DF
:1060F0009B1A0B4A9B1053439C4203D3B22109487D
:10610000FDF7FCFC0C23286903FB040038BD0248A2
:10611000FCE700BF8C460020A44600204CB20108DA
:10612000ABAAAAAA0AB2010810B5D0E90730C9B2D1
:10613000D2B2834209D01C788C4204D15C7894425C
:1061400001D1987810BD0333F3E74FF0FF30F9E742
:106150002DE9F041D0E904239B1A524A9B10534386
:106160000D4609780446994203D393214E48FDF722
:10617000C5FCD4E901239B1A4A4A9B105343697812
:10618000994203D394214848FDF7B8FCD4E904238D
:106190009B1A444A9B105343A978994205D3FE2980
:1061A00003D095214048FDF7A9FC6A78297820465C
:1061B000FFF7BAFFC3B2FF2B064629D02978204645
:1061C000FFF782FF697807462046FFF765FF3146F3
:1061D00080462046FFF778FF414602463846FFF7E3
:1061E00013FD29782046FFF76FFF697806462046A1
:1061F000FFF752FFA97807462046FFF765FF3946AB
:1062000002463046FFF700FD9C212748FDF776FC4B
:10621000D4E90723234F9B1A7B437E2B03D99F216D
:106220002148FDF76BFCD4E90721606A8B1A7B4398
:10623000091A4F430133BB4203EB43080AD84244D7
:1062400022622A88236A23F8032CAA7803F8012CF7
:10625000BDE8F081404605F0CFF8064618B969213F
:106260001248FDF74BFCD4E907010B1A0D495943BD
:106270000023CA1A002A0DDD03EB43028718B7F882
:1062800000E006EB020C26F802E0BA7801338CF845
:106290000220EEE705F09AF8E6614644C4E9086694
:1062A000CFE700BFABAAAAAA0AB2010802A601085A
:1062B00013B5FF24074B8DF804401B680A46186885
:1062C00001A9FDF73BF9012814BF20469DF8040001
:1062D00002B010BD9846002038B5816800681D46A0
:1062E000144605F03EF90346201845EBE37138BD2E
:1062F0002DE9F0410E681046722E1F4624D0742EF0
:1063000008D0632E12D000244FF0004520462946C5
:10631000BDE8F0818B68D3E90023B3F1004F08BFDB
:10632000002A16D0841847EB0305EFE7886804F0CD
:106330006DFE002871F1000304460D46E6DADD210A
:106340000548FDF7DBFBE1E78868BDE8F041FFF7B2
:10635000C3BF14461D46D9E70AB201082DE9F04132
:106360000F4606460024FFB2FFF7AEFED6E90758F7
:10637000454511D02B78BB420CD169783046FFF7E8
:106380008BFE0368692B05D183681B6803B19847AE
:106390000134E4B20335EBE72046BDE8F0812DE996
:1063A000F34180460F460025FFF78EFED8F81C40CB
:1063B000D8F8206003340336FFB2A6421BD0234630
:1063C00033F8032D9B78ADF804208DF8063014F8CF
:1063D000033C9F420DD19DF805104046FFF75CFE3F
:1063E0000368692B05D183685B6803B19847013561
:1063F000EDB20334E1E7284602B0BDE8F0810000C9
:10640000836C73B504460D46164623B94FF48C7160
:106410000B48FDF773FBCDE9006423462A46094982
:106420000948FBF71FFA012807D04FF48F71044881
:1064300002B0BDE87040FDF761BB02B070BD00BFA7
:106440000AB20108E6B20108D569000838B590F82B
:1064500047300446032B0D4604D940F2311106485B
:10646000FDF74CFB94F847305A1C84F847201C4435
:1064700084F8425038BD00BF0AB2010810B590F848
:106480004730044623B94FF49B710648FDF736FBAD
:1064900094F84730013BDBB284F847301C4494F851
:1064A000420010BD0AB20108CBB2FE2B10B5044663
:1064B0000AD0FFF709FE03686D2B05D1017A20464B
:1064C000BDE81040FFF700BE10BD00002DE9F84305
:1064D00004460026114FD4E904239B1A9B107B43EA
:1064E0005FFA86F8434516D941462046FFF7DCFFA0
:1064F000D4E90759A9450CD02B78434507D16978D1
:106500002046FFF7C9FDA9782046FFF7CDFF0335E8
:10651000F0E70136DFE7BDE8F88300BFABAAAAAA1F
:1065200070B56FF04106044600F14205361A94F842
:10653000472073199A4205DD15F8011B2046FFF725
:10654000C3FDF4E770BD00232DE9F04FC0E904332B
:10655000884619464FF000430446C0E90213C0E9DB
:106560000013FF2085B0CDE90013DDE90E6720742C
:106570005FFA82F9D8E907500390039BD4E900AB96
:106580009D4220D02B784B451BD169784046FFF7C0
:1065900083FD32463B4601464046FFF7A9FEDDE952
:1065A0000023994208BF90420BD09B4508BF9245FB
:1065B00003D0504571EB0B0303DA6B78C4E900019B
:1065C00023740335D9E7BBF1004F08BFBAF1000FC0
:1065D00005D0BAEB06066BEB0707C4E90267204655
:1065E00005B0BDE8F08F0000F8B50D460B4B89688B
:1065F00006464B434FF47A71B3FBF1F1FFF758FEB7
:106600000446C7B2B06C03681B689847FF2FC6E901
:106610000E010CBF287C2046F8BD00BF40420F0091
:1066200070B5C36C86B004460D4623B906B0BDE80C
:106630007040FFF7D9BF806C194903681B69984700
:10664000A06C03689B689847D5E9002303A804F071
:106650004FFDA06C9DF80C20036800929DF80F1070
:106660009DF80E205E689DF80D30B047A06C036861
:10667000DB689847E36C9847A06C03689B68984771
:10668000A06C03681B689847C4E90E0100212046EE
:10669000FFF70EFEC0B2FE2808BF287C06B070BD12
:1066A000395C00082DE9F8499046D1E90023B3F19F
:1066B000004F08BF002A05460C463BD0D4E9020132
:1066C000012871F1000302DA207CBDE8F889B8F1F5
:1066D000000F12D021462846FFF786FFC0B2FF28E0
:1066E00016D140F20F211948FDF708FA184B194A44
:1066F0004FF40471154810F035FCD5E9142390428D
:1067000071EB0303E6DB21462846FFF789FFE5E747
:10671000237C8342D9D1D5E90EBCD4E90067B345C7
:106720007CEB0703D1DAB6EB0B0267EB0C03C4E991
:106730000223C3E7B8F1000F03D0BDE8F849FFF723
:1067400053BFBDE8F849FFF76BBF00BF0AB20108AD
:10675000AFA801086DB301082DE9F04188B00446E7
:106760000D46FFF7B1FC03680646702B04D04FF4CA
:106770009E713048FDF7C2F9A06C03681B6898470A
:106780002A46C4E90C01CDE90001214602A8FFF721
:10679000DAFE29462046FFF7E1FD9DF8183007464E
:1067A000FF2B05D120B940F247112248FDF7A6F989
:1067B000D4E90C0104F004FD01461F4804F080FDFB
:1067C00039461E4804F07CFD9DF81810FF2912D1AF
:1067D00000224FF00043CDE90423327A02A920467B
:1067E000FFF760FF064629462046FFF7D8FD3046F2
:1067F00008B0BDE8F0812046FFF74EFCD0E90078F4
:10680000DDE9020104F0DCFC4246034639460C484F
:1068100004F056FDD4E90C3202980399C01A61EBDA
:106820000201CDE9040104F0E1FC0146054804F051
:1068300047FDD2E70AB201085AB2010879B201084D
:1068400094B20108B8B2010870B504460D46FFF7CE
:106850003BFC03686D2B11D0702B09D0612B0DD13F
:10686000836894F8411094F84000BDE870401847E0
:1068700029462046BDE87040FFF76EBF40F22B115D
:106880000248FDF73BF94FF0FF3070BD0AB2010836
:106890002DE9F04790F828300446FF2B04D14FF43F
:1068A000D0714848FDF72AF994F828102046FFF7E0
:1068B0000BFC94F82830DFF8188184F8463094F8FF
:1068C00046102046FFF700FC036805466D2B204666
:1068D00094F846100BD1FFF7B9FD297A204684F8C9
:1068E0004610FFF7F1FB2046FFF71AFEE7E7FFF738
:1068F000ABFFC3B2FF2B06460BD140F2B5113148B6
:10690000FDF7FCF840F2B5112F4B304A2D4810F03E
:1069100029FB024694F846102046FFF705FCC5B255
:10692000FF2D09D140F2BB112648FDF7E7F8264BB1
:10693000264A40F2BB11E9E794F84610FE2D2046A6
:1069400021D1FFF79BFD074601462046FFF7BCFB20
:10695000324639462046FFF7E7FBC5B2FF2D0DD181
:1069600031462046FFF798FB40F2C7111548FDF766
:10697000C5F8154B154A40F2C711C7E72046FFF787
:10698000CFFD3946DAE7FFF79FFB31460746204641
:10699000FFF782FB294681462046FFF795FB82469A
:1069A000404604F08DFC524649463846FFF72CF924
:1069B00094F8463084F8416084F8403084F84650BA
:1069C0007DE700BF0AB20108AFA8010848B301087B
:1069D000D6B2010808B5FFF7DBFAFFF759FFD0B5CB
:1069E0001F461646FFF758FB03688468742B01D0D6
:1069F000FFF71CF9C4E90067D0BDD0B504461646C0
:106A00001F46FFF749FB32463B4601462046BDE89C
:106A1000D040FFF76DBC0000836C10B5044623B96D
:106A200040F279210248FDF769F8A06C10BD00BF63
:106A30000AB20108FF23054A1370054A1370054A7C
:106A40001370054A1370054A13707047A046002062
:106A50009E4600209C4600209F4600209D46002028
:106A6000014B1878704700BF9C46002010B50446C3
:106A70000068FCF7D3FF204610BD00002DE9F0436D
:106A800085B005F0FDFE4FF6FF712E4A2E4C13889F
:106A90008B421CBF01331380FFF77AFAFFF7BCFF6C
:106AA00003681B689847637806460F46FBB9274B77
:106AB000DB88E3B1264AD2E90001B1F1004F08BFFB
:106AC00000280FD0B04271EB070210DA214AB6EB72
:106AD000000802FB03F267EB0109D317904579EB3D
:106AE000030304DB1C4804F0EBFB01236370002369
:106AF000ADF80C3063782BB101238DF80C30144BBA
:106B0000C3E900672378154CBBB1012514488DF803
:106B10000D5004F0D5FB25700023124A124913488A
:106B200000931278039B0978006805F0E7FF30B105
:106B30000F4B187805B0BDE8F0832370ECE70D4BE0
:106B4000F7E700BF4E470020304700203C470020B9
:106B50006800002080510100DAB4010839470020A4
:106B600003B5010833470020324700202C4700209E
:106B70009C4600209E4600201D4B10B5DB882BB99B
:106B80001C4804F09DFB1C4B187810BD1B4BD3E92F
:106B90000023B3F1004F08BF002A01D01848F0E7E6
:106BA000184C23780133DBB2032B237001D916482C
:106BB000E7E7012B0BD90A21002004F0D2FC134B8C
:106BC00058434FF47A73B0FBF3F0FBF7BFF9217829
:106BD0000F4804F075FB00230E4A13700E4A137021
:106BE0000E4A13600E4A1370012353700D4BCBE70E
:106BF0003C47002018B501089C460020600000209A
:106C000034B50108604700204EB5010840420F002E
:106C100065B5010833470020324700202C4700208B
:106C2000304700209F46002008B500231A46FCF795
:106C3000E1FB431E5842584108BD000007B50B78E0
:106C4000012B11D05AB22AB1022B11D00A4804F0FC
:106C500037FB06E00192094B01A91B681868FFF792
:106C6000E3FF03B05DF804FB4FF0FF330193F2E75D
:106C7000024B04311B68F1E7CBB501081C4700202B
:106C80001FB57023CDE90131002301A98DF80C3027
:106C9000FFF798F905B05DF804FB00002DE9F04F0F
:106CA000474B85B01A780446002A40F085800127BA
:106CB00044491F70FFF7E4F8434B444918702046DD
:106CC000FFF7DEF8DFF854A141498AF800002046BA
:106CD000FFF7D6F8DFF848910A22002389F8000070
:106CE0003C4901A8FEF7BAFF01A92046FFF75EF86C
:106CF000394E3A4930702046FFF7C2F8384B3949CF
:106D000018702046FFF7BCF8374B384918702046FA
:106D1000FFF7B6F8364B374A187037492046F9F76F
:106D200087FDDFF800B1354A8BF800003449204672
:106D3000F9F77EFD334905462046FFF7A1FF702392
:106D40000193314B804601A9204602938DF80C70C7
:106D5000FFF738F907462D4A2B4612789BF80010AA
:106D60002046F9F770FD43469AF800202946204650
:106D7000F9F769FD3B4699F8002029462046F9F7C6
:106D800062FD2B46327841462046F9F75CFD2B46E2
:106D9000327839462046F9F756FD1D4A2B461278BF
:106DA00029462046F9F74FFD1A4B1B4A1B781278EB
:106DB00029462046F9F747FD05B0BDE8F08F00BF32
:106DC0006147002021B70108344700202BB7010894
:106DD00036B7010842B70108154700204FB7010830
:106DE0004C4700205BB701085047002068B70108F6
:106DF000514700207D6A000876B70108E57B00084E
:106E000080B7010894B70108A7B701089C46002085
:106E10009F4600209D460020A046002038470020C5
:106E2000144700203647002008B505F007FD18B1CB
:106E3000BDE8084005F024BD08BD000030B504469B
:106E400085B00D46FFF72AFF6D22064B01A91B787E
:106E50002046CDE901258DF80C30FFF7B3F805B0D9
:106E600030BD00BF364700202DE9F84F434B0446A4
:106E70001A68434D12F0010F79D1FF222A700122C6
:106E80001A602046FFF70AFF3E4A3F492046F9F7BD
:106E9000CFFC3E4A28703E492046F9F7C9FC3D4FD9
:106EA0003D4A38703D492046F9F7C2FC3C4E3D4909
:106EB00030702046FFF7C2FF3B4982462046FFF76D
:106EC000DFFE3A4983462046FFF7DAFE8146384A1C
:106ED0003B78297820461278F9F7B5FC354ADFF877
:106EE000E8803378297820461278F9F7ACFC3378BB
:106EF00098F8002039782046F9F7A5FC2B7898F807
:106F0000002031782046F9F79EFC2B4A5B46397801
:106F100020461278F9F797FC28493B780A782046F2
:106F20005946F9F790FC264A4B46397820461278A4
:106F3000F9F789FC21493B780A7820464946F9F758
:106F400082FC1C4A5346317820461278F9F77BFCC4
:106F5000337898F8002051462046F9F774FC194A16
:106F60002B78127831782046F9F76DFC02E02B7807
:106F7000FF2B86D02878BDE8F88F00BF104700208F
:106F8000634700204D760008B7B80108B5710008C6
:106F9000C1B8010835470020796B0008CBB801085B
:106FA00037470020D5B80108E1B80108EFB801085B
:106FB000344700209F460020384700201547002016
:106FC0009E4600209C460020A046002038B504467E
:106FD0000D46FFF763FE034A29462046F9F728FCD1
:106FE00038BD00BF1D740008344B2DE9F04F1A89DD
:106FF0000023044689B0CDE9002303910023002239
:107000002F4905A8FEF73CFE05A92046FEF7CEFE57
:107010002C4982462046FFF733FE2B498346204603
:10702000FFF7D4FF294A804629492046F9F700FC9A
:10703000284A054628492046F9F7FAFB0646274F15
:10704000DFF8A8903B7899F8002029462046F9F708
:10705000FAFB234A5B46294620461278F9F7F3FBF0
:10706000204A4346294620461278F9F7ECFB33467E
:10707000524659462046F9F7E6FB3346524641460A
:107080002046F9F7E0FB184A3B7841462046127843
:10709000F9F7D9FB3B7899F8002031462046F9F7FB
:1070A000D2FB6D230593039B05A9204606938DF81B
:1070B0001C50FEF787FF09B0BDE8F08F3C47002069
:1070C000FEB801080BB901081BB901086D7700086B
:1070D0002CB90108616A00083BB901089D460020EF
:1070E00050470020514700204D4700209C4600207B
:1070F0002DE9FF4790468A461E4A1F490446F9F784
:1071000097FB1E4905462046FFF7BAFD1C498146FC
:107110002046FFF75BFF06461A4A4B4629462046A3
:107120001278F9F790FB184A184F33462946204643
:107130001278F9F788FB3B78424649462046F9F732
:1071400082FB3B78424631462046F9F77CFB104AE9
:107150003B78127831462046F9F775FB6D2301A97B
:107160002046CDE9013A8DF80C50FEF72BFF04B014
:10717000BDE8F087917700088CB8010896B801083F
:10718000A6B8010850470020514700209D46002026
:107190004D47002070B50D460446FEF7F9FE044940
:1071A00022462B46BDE870400978FFF718BC00BFA7
:1071B00015470020F7B55D4C26689EB9042003F002
:1071C00093F932460546066004210120FCF738F8A1
:1071D000286018B911215648FCF790FC55482560E5
:1071E00005F064FB544D554F29685548013129601D
:1071F00004F066F805F044FB3B781BB901233B70B3
:1072000005F06AFB0023019323684E4A01A9186820
:10721000FCF794F9012807D04B4804F051F840F2EC
:107220008D114A48FCF76AFC019E731C51D14848F5
:1072300004F046F82B68042B0FD9FEF729F90378E0
:107240005BB1444804F03CF84FF47A70FAF77EFEE4
:107250004FF4CC713D48FCF751FC00233B702B6888
:107260001E22013BDBB21E2B28BF1E2302FA03F3B2
:10727000394A934226D8B3F5616F1E464FF0000796
:1072800022D2B3F5167F77F1000320DA3C2E77F196
:107290000003ACBF1E210A21002004F062F934185B
:1072A00047EBE0752946204603F0A0FF01462B4836
:1072B00004F006F820462946FFF76CFF284B1878A3
:1072C00003B0F0BD0027244E4FF41671E4E73C21D3
:1072D000E2E74EB13146234803F0F2FF0198002166
:1072E000FFF758FF204BEAE720482E6003F0E8FF45
:1072F00005F07AFAFEF74CFEFFF78EFB03681B6879
:1073000098471B4BC3E9000123686BB1304605F079
:10731000CDFA256835B12868FCF780FB04212846A2
:1073200003F004F900232360124BC8E71C47002038
:10733000F1B201083D6C00085C470020584700206E
:10734000C2B30108A0860100D5B30108EFB301085C
:107350003BB4010852B4010800A302009FB4010825
:107360009E460020B5B4010838470020CAB4010881
:1073700058000020A0460020054B1870054B1A70DD
:107380000022054B1960054B1A705A70704700BFF8
:1073900033470020324700202C4700203047002090
:1073A000027901684079FFF7E7BF08B505F09EFB59
:1073B000C0B2DE2828BFDE2008BD00004FF47A737B
:1073C00037B5002403FB00F20749B2FBF3F20D6866
:1073D00001A928680194FCF7B1F8012814BF2046E0
:1073E000019803B030BD00BF184700204FF47A73F6
:1073F00037B5002403FB00F20749B2FBF3F20D6836
:1074000001A928680194FCF7DBF9012814BF204684
:10741000019803B030BD00BF184700202DE9F04FA0
:107420008FB0FEF7B5FD4FF00009064690F846B064
:10743000FFF7FAFCDFF8C4A0DFF8C480B06C02AD3F
:10744000036808AC1B6898475A46CDE900013146ED
:1074500008A8FFF778F80FCC0FC52368DDE9020113
:10746000B1F1004F08BF00282B70DDE9044516D1AB
:107470001C4803F025FF002501271B4C4FF47A73AD
:10748000A4FB030103FB0511FFF7B0FF10B30122BA
:10749000164B5A72164B18780FB0BDE8F08F03F0F8
:1074A0008FFE29460746204603F0A0FE39460246D5
:1074B000504603F005FFA04579EB050308DA0021EB
:1074C000094803F093FE01460A4803F0F9FED2E7AB
:1074D0000027D3E71FB1084803F0F2FEAEE79DF89E
:1074E0001800D9E753B60108805101002047002059
:1074F0004D4700208DB60108A6B601086BB60108FD
:1075000085510100022818BF002005F06BBC000067
:10751000F8B53B4B05461E78002E6FD101271F7032
:1075200004F07AFE37492846FDF738FEC31F052BC5
:10753000354C42D820710E23344928466371FDF73B
:1075400036FE3349074610F03BFD00283AD1E06093
:1075500030492846FDF708FE2F4960702846FDF7A0
:107560001DFEB0F57A7F3AD8E0802C492846FDF719
:1075700015FE42F21073984236D8208128492846D9
:10758000FDF7F2FD2749A0702846FDF707FEB0F58C
:107590007A7F2ED2608124492846FDF7E5FDE07010
:1075A00036B1224803F08CFE71212148FCF7A6FA7F
:1075B000E068BDE8F840FFF7A5BF1E4803F080FE75
:1075C0003E46B8E71C49384610F0FAFC10B90223D1
:1075D000E360BDE7194803F073FE0126B8E71848D9
:1075E00003F06EFE0126C0E7164803F069FE01268F
:1075F000C4E7154803F064FE0126CCE7F8BD00BFE0
:1076000062470020BBB701083C470020D4B70108FF
:1076100077B80108F7B70108FBB7010822B80108DD
:1076200075AB01084AB8010874B8010879B80108B7
:10763000EFB30108BEB70108A3D40108DBB7010806
:1076400004B801082BB8010855B8010870B5234BE0
:10765000C0B21B78984206D1FDF71AFFFDF7B0FDC6
:107660001F4B187870BD1F4DFDF712FFFFF750FF3D
:1076700095F9050006F086FE05F0D8FA287906F09F
:107680004FFE05F0C7FA687805F0A6FB164B1A689E
:107690001C4612F0010212D10421144E0846326039
:1076A000FBF7CEFD306018B911211148FCF726FA1E
:1076B0000123104A10490D4823600EF062F90F4B68
:1076C0001A680AB9094A1A600D4805F091FBEB786F
:1076D0000BB10C4BC5E70C4BC3E700BF374700208D
:1076E000A04600203C4700200C47002054470020C3
:1076F000F1B20108000000206D6A00081847002060
:10770000697B0008344700209F460020034B93F814
:107710003230022B0CBF022000207047C000002036
:1077200008B5FFF7F3FF30B905F088F818B9BDE8E0
:10773000084005F059B8FFF7E9FF022806D105F027
:107740007DF818B1BDE8084005F09AB808BD000002
:1077500008B5FFF7DBFF02280CBF024B024B18787D
:1077600008BD00BF5147002050470020054B1B8932
:1077700013B9054B18787047044B5B7A002BF8D18E
:10778000FFF7E6BF3C4700209C4600202047002032
:10779000FFF7DEBF01232DE9F743394C002000211C
:1077A0006372FFF723FE10B1364B18781AE0236896
:1077B000984718B9344B1B78002B3CD005F01EFBC2
:1077C000012871F10003804689460EDB2F4803F043
:1077D00077FDFEF7DDFB42464B46217AFFF7FFF8C7
:1077E000FFF7B6FF03B0BDE8F0832368984705466E
:1077F00088B1274803F064FD002364680093ADF866
:107800000430FFF7D2FD01466846A0476846FFF7FF
:10781000C7FD204BC9E71C4B1B7863B11E4803F022
:107820004FFD1E4B1B88022B28D82A462946284686
:10783000FFF7A2FDEDE71A4D6B89EBB1EB78DBB1F9
:10784000FEF7A6FBFFF7E8F803681B689847154AA0
:10785000D2E90032C61A61EB02076B89124A5A4319
:10786000D317B242BB4107DA104803F029FD40F2BA
:1078700049310F48FCF742F9002363720D4B94E73E
:10788000204700204D47002052470020F9B501084D
:107890000AB601084C4700201CB601084E470020DC
:1078A0003C470020580000208051010033B60108F9
:1078B000EFB301089C4600202DE9F04F0446444DEB
:1078C00087B0C5E90023019100230A22414903A89A
:1078D000FEF7C4F903A92046FEF768FA3E4A82463D
:1078E00028723E492046F8F7A3FF3D490546204649
:1078F000FFF7A4FA3B498DF803002046FFF7C0F9D3
:10790000394983462046FFF761FB384980462046C7
:10791000FFF76AFB0746364A364EDFF8EC902B46F7
:10792000014612782046F8F78EFF337899F8002048
:1079300039462046F8F787FF337899F80020294622
:107940002046F8F780FF2A4A3378294620461278E5
:10795000F8F779FF284A9DF8033029462046127827
:10796000F8F771FF254A2B469DF803102046127840
:10797000F8F769FF224A5B46294620461278F8F755
:1079800062FF2B46524659462046F8F75CFF1D4AD7
:107990004346294620461278F8F755FF2B465246B3
:1079A00041462046F8F74FFF337899F800204146CA
:1079B0002046F8F748FF6D230393019B03A9204657
:1079C00004938DF81470FEF7FDFA07B0BDE8F08F50
:1079D000204700204AB90108957700085AB90108E4
:1079E00068B901082BB7010836B7010874B9010856
:1079F0009C4600209D4600204C470020A0460020C9
:107A000050470020514700204D470020F8B51D4643
:107A100000234171BDF8181004460360C180174669
:107A200002B115B923712046F8BD0749284602F076
:107A300079FD064610B920712660F4E72A463946DA
:107A40000FF0BEFB2571F7E726EB010810B50446E1
:107A5000006808B102F068FD204610BD70B5364ED2
:107A600086B03268044622B940F2CB113348FCF7A5
:107A700045F8002C5DD00022314B1A80D4E91C233C
:107A800013431FD02F4B1D68FAF70EF901462E48FD
:107A9000A847D4E91C0103F093FB226F01462B4851
:107AA00003F00EFCD4E91C2303A803F021FBD4E966
:107AB0001C23274903A8C1E900232649C1E9002363
:107AC00008F0A4FDFEF764FAFEF7A6FF03681B6842
:107AD0009847214B214AC3E90001237AC3F3C0032D
:107AE0001370637F2BB3237F1BB31D49082002F063
:107AF0000DFD054630B163890093237FA26E617F3F
:107B0000FFF784FF0395A5B1002330681A4603A947
:107B10000068FBF7B9FB01280BD0124803F0D0FB3B
:107B2000039C34B12046FFF791FF0821204602F064
:107B3000FDFC06B070BD00BF18470020EFB3010880
:107B40004E470020C0000020BCB60108C9B601089D
:107B500060000020680000205800002052470020EC
:107B600026EB0108F6B6010810B50446FFF776FFCC
:107B700024B12046BDE8104006F068BF10BD0000EB
:107B800038B542F2107004F097FE0446124803F034
:107B900097FBECB12578022D16D160680021FFF724
:107BA000F9FAD4F89800FFF759FF237A2BB10B4864
:107BB00003F086FB00220A4B1A70204605F0F2FC07
:107BC000032D06D1284638BD032DEAD10020E5E774
:107BD0000125FFF7A5FDF5E780B501089EB5010871
:107BE00039470020002310B5144C84F8363004F0D7
:107BF00025FE08B104F044FEFFF7C2FF032815D8A4
:107C0000DFE800F005020A080D4803F059FB0D4BB0
:107C1000187810BD0C4BFBE7FFF778FD022809BF71
:107C200001230A4B84F83630094BF1E7094840F24A
:107C3000BA21FBF763FF4FF0FF30EAE7C0000020F6
:107C4000B1B50108A04600209F460020384700201B
:107C500014470020EFB30108FF2300210D4A1370E1
:107C60000D4A13700D4A13700D4A13700D4A1370AC
:107C70000D4A13700D4A13700D4A13700D4A13709C
:107C80000D4A13700D4A13700D4AC2E900111372A8
:107C9000704700BF36470020354700203747002097
:107CA0004D4700204C4700205147002050470020FE
:107CB0003447002038470020144700201547002093
:107CC0002047002010B504460068FBF7A7FE2046B9
:107CD00010BD00002DE9F8430746884615460024EC
:107CE000DFF830900A4E44450FD045B13CB1B4FBAB
:107CF000F5F305FB134313B9484603F0E1FA395D88
:107D0000304603F0DDFA0134EDE7BDE8F88300BF4B
:107D1000D3A801083CD4010807B5074B8DF807002C
:107D2000186800230DF107011A460068FBF762FB93
:107D300003B05DF804FB00BF68470020C0F3C70331
:107D400042071CBF0133DBB218467047052910B546
:107D500001D8002012E04378013B032BF9D8DFE87B
:107D600003F00E0E02020024043003F0D4FB44B1F1
:107D7000FFF7E4FF80B2FA28EBD8C0B210BD0124AF
:107D8000F2E74000F6E700000023194A70B5C0E9A9
:107D9000002381604E234FF416510446C0E90313BB
:107DA0000A2308200121C4E905034FF48773114D0C
:107DB000A3832A68A1770A4012D10F4E4FF4807036
:107DC0003260FBF73DFA306018B911210B48FBF720
:107DD00095FE01230A4A0B4907482B600DF0D1FD9F
:107DE000094B1A680AB9044A1A60204670BD00BFE0
:107DF00000010002644700206C470020F1B2010836
:107E000000000020C57C000868470020024680680A
:107E1000036819B11B6802F10C0118475B68184729
:107E20002DE9F3471C469DF8285006468DF80710AB
:107E30008DF806200DF1070101224FF6FF7002F0C8
:107E400077FB01220DF1060102F072FB2A46214662
:107E500002F06EFB81464FEA202A9DF80620C7B249
:107E60009DF807101B4803F02BFA29461A4803F027
:107E700027FA294601222046FFF72CFF174803F076
:107E80001FFA52464B463946154803F019FAB068B6
:107E90009DF8071003685FFA8AF89B689847B068F6
:107EA0009DF80610036825449B689847B068A54272
:107EB00003689B6803D014F8011B9847F6E739461E
:107EC0009847B068414603689B68984702B0BDE890
:107ED000F08700BFC4B90108EFB9010862AC01081E
:107EE0000ABA01080B4670B505460A11D1B2092A33
:107EF00003F00F038068D4BF30313731092B94BFB2
:107F000003F1300403F1370403689B689847A868BD
:107F10002146BDE8704003689B6818472DE9F14F82
:107F200005461F4698461E469DF828B08A461144CD
:107F30009146C9B203EB0B02964204D016F8013BFE
:107F40001944C9B2F8E749424A46CCB21B485146E7
:107F500003F0B6F959461A4803F0B2F9012259461E
:107F60003846FFF7B7FE174803F0AAF9214616482E
:107F700003F0A6F9A8683A2103689B689847514620
:107F80002846FFF7AFFF49462846FFF7ABFFB0454D
:107F900002D018F8011BF7E721462846FFF7A2FF99
:107FA000A8680D2103689B6898470A21A8680368A0
:107FB0009B6801B0BDE8F04F184700BFC4B9010885
:107FC000EFB9010862AC010825BA010830B4456870
:107FD0009DF808401DB1012D05D030BC70470294BA
:107FE00030BCFFF71DBF029430BCFFF797BF000005
:107FF0002DE9F04F85B090466A4600AF7B6003885C
:10800000464C0733DB08A2EBC3039D4606468A466F
:108010006D46A3462368002207F10F011868FBF79D
:108020008DFA0128F6D0B0683D49036800241B6929
:108030009847F9F739FE4FF47A7300F57A79DBF84F
:1080400000001A4607F10F0100683B60FBF776FA63
:1080500001280AD1621C92B2F97B012A295521D04C
:1080600031883B6891421FD814466CB1297851453C
:108070000AD02C4803F024F9F9F716FEA9EB000307
:10808000B3F57A7F12D90024B068002103681B6918
:1080900098476CB9244803F013F920461437BD46BD
:1080A000BDE8F08F4FF47A731446C8E70022FBE76F
:1080B00021461E4803F004F9002221462846FFF716
:1080C00009FE1B4803F0FCF8032C04D8194803F000
:1080D000F7F80024E1E72B1913F8012C13F8026CD0
:1080E000023C06EB02262946A2B24FF6FF7002F0D0
:1080F0001FFAB6B28642014604D032460E4803F05B
:10810000DFF8E6E77B68E4B29C4228BF1C462946BC
:10811000224640460FF054F8BFE700BF68470020F2
:10812000197D000834BA010862BA010879BA010859
:1081300062AC010897BA0108D0BA01082DE9F04FE6
:1081400085B016466A469846438800AF0733DB0879
:10815000A2EBC3039D46714C824689466D46A346F9
:108160002368002207F10F011868FBF7E7F90128DF
:10817000F6D0DAF808006A4903681B6998470023BB
:10818000DBF8000041F2883207F10F0100687B60E4
:10819000FBF7D4F901287B6826D1FA7B5C1CA4B2DA
:1081A00002F07F02012CFA73EA5408D92B1913F854
:1081B000022C0D2A03D113F8013C0A2B03D0BAF884
:1081C0000230A3420ED8DAF80800002103681B69C8
:1081D00098475CB9534803F073F820461437BD46FE
:1081E000BDE8F08F2346CBE71C46ECE7082C10D8FF
:1081F0004D4803F065F821464C4803F061F82846E5
:1082000001222146FFF766FD494803F059F8002492
:10821000E3E72B783A2B08D12B1913F8022C0D2AFF
:1082200003D113F8013C0A2B01D04248E1E728466C
:10823000AC460021E21ED2B2CBB29A420DD91CF854
:10824000013FA3F1300EBEF1160F04D83A3B062BC6
:1082500001F10101F0D83848CBE7D30705D53748FD
:1082600003F02EF821463648C7E75210D3B26C1EF1
:1082700005EB420C60452AD090F801E0AEF13001E8
:10828000C9B2092907D9AEF1410105298EBF0021E4
:10829000AEF13701C9B290F802A00901AAF1300E7F
:1082A0005FFA8EFEBEF1090FC9B20AD9AAF1410EDA
:1082B000BEF1050F8EBF4FF0000EAAF1370E5FFA28
:1082C0008EFE41EA0E0104F8011F0230D2E70020C1
:1082D0000146013AC4B2944200F1010003DA2C5D78
:1082E0002144C9B2F6E74942AA5CC9B2914203D01F
:1082F000144802F0E5FF8AE72A784A4502D00A4688
:108300001148F6E7013BDCB2444528BF4446294604
:10831000224630460EF054FF5FE700BF684700205A
:10832000197D000862BA010813BB010879BA010877
:1083300062AC01084CBB010868BB0108B2BB010874
:10834000E1BB010800BC010843BC01082DE9F04174
:108350001F460E4B04461B680D46164623B940F2D5
:10836000E3110B48FBF7CAFB63683BB13B4632465F
:1083700029462046BDE8F041FFF7E0BE3B463246C5
:1083800029462046BDE8F041FFF732BE684700208D
:108390007FB901082DE9F34704460D4690469946FA
:1083A00080689DF828A003680121DB690B9E9DF879
:1083B0003070984742464B4629462046CDF800A0EB
:1083C000FFF704FEA06800210368DB6998473B467D
:1083D00032462946204602B0BDE8F047FFF7B6BF57
:1083E000F0B585B09DF828701D46CDE90137931E84
:1083F000DBB200930C4616468B1C4A780978FFF7CF
:10840000C9FF60B9022F0AD9012E08D923780320A9
:108410002B70637863F07F036B700B23AB7005B038
:10842000F0BD0000034A0260002202710274C0E93C
:108430000222704780BC010870B50646084802F069
:108440003FFF002406F108053379A34206DD55F805
:10845000040B013403689B689847F5E770BD00BFC3
:1084600094BC010870B50646002400F10805337974
:10847000A34206DD55F8040B01340368DB68984716
:10848000F5E770BD38B5057900F1080435B1013D57
:1084900054F8250003685B699847F7E738BD70B565
:1084A0000646002400F108053379A34206DD55F89D
:1084B000040B013403681B699847F5E770BD0000A1
:1084C00038B503790446012B0D4603D939210748F5
:1084D000FBF714FB6968064802F0F2FE23795A1C88
:1084E0000233227144F8235038BD00BFACBC0108F0
:1084F000E7BC010870B504460D4603680121DB683E
:1085000098472368294620461B69984723682046D8
:10851000BDE87040DB6800211847806970474069FA
:10852000704738B5036804461B69984705462368B9
:1085300020469B699847284638BD8368C0E90333C5
:10854000002383617047000038B50025094B0446BD
:10855000C0E900310B68C0E90355C0E905551B6847
:1085600008469847A5606061C4E90355A5612046A7
:1085700038BD00BF50BD0108D0E90332934291BF1E
:10858000D01A40698018C01A7047000038B50546F7
:108590000C46FFF7F1FF884203D213210648FBF790
:1085A000ADFAE9686A69AB68214413449942E9600D
:1085B00024BF891AE96038BDFEBC010808B5014630
:1085C000FFF7DAFF4B69181A08BD00002DE9F14FDB
:1085D00002EB03099A464369044699450F469046C3
:1085E00003D93C211F48FBF789FA63696068A668D4
:1085F00025691E440368A6EB050B1B6901219847FA
:10860000D94560680ED803683A465D684346E1681C
:108610005144A8470021606803681B6901B0BDE8A8
:10862000F04F18470368DA45D3F8049012D2E16896
:10863000ABEB0A0B5B463A465144C847606805EB12
:108640000A01026801EB080355689B1B07EB0B024C
:10865000A168DEE7A1684346294451443A46891B94
:10866000C847D7E7FEBC010807B5042200230DEB7D
:108670000201FFF7ABFF019803B05DF804FBF8B50A
:10868000064617460D4679B184695CB1FFF7ECFFE9
:1086900087423C4628BF04460423224629463046EA
:1086A000FFF794FF2046F8BD0C46FBE783690BB14A
:1086B000FFF7DABF1846704738B5836904466BB1D7
:1086C000FFF7D2FF054604212046FFF75FFF29464A
:1086D0002046FFF75BFFA369013BA36138BD0000A3
:1086E00038B5436905468B420C4603D25F210748E3
:1086F000FBF704FA29696A69AB682144134499427B
:10870000296124BF891A296138BD00BFFEBC010858
:108710002DE9F04715461E4A0446136889462B4446
:108720001360FFF74BFFA84203D22B211948FBF738
:10873000E5F963696068A66827691E44036801213A
:108740001B699847A6EB07086068454503680FD882
:108750009E684A462B462169B0476068002103683D
:108760001B69984729462046BDE8F047FFF7B8BF88
:10877000D3F808A04A4643462169D04760687B1970
:1087800002689B1B9768A16809EB0802B847E4E7F9
:1087900070470020FEBC010807B5042201910DEBD3
:1087A0000201FFF7B5FF03B05DF804FB70B5144696
:1087B00005460E46FFF702FF231D98420DD32146C2
:1087C0002846FFF7E9FF224631462846FFF7A0FF7B
:1087D000AB690133AB61204670BD0024FBE70000AC
:1087E00038B50A4C05460121204607F0F1FC00236C
:1087F00020461A46012107F029FC85F00102204697
:10880000BDE83840012107F0EFBC00BF0000024086
:1088100008B50120FFF7E4FFBDE80840032008F099
:108820005DBC0846FFF7DCBF10B50446024B036091
:1088300002F0E2FE204610BD78BD010810B50446E6
:10884000054B503040F8503C044B40F8083CFFF7D3
:10885000EBFF204610BD00BF4CC1010898C30108C2
:1088600010B50446FFF7E0FF2046082101F05EFE48
:10887000204610BD10B50446FFF7E0FF20467821E2
:1088800001F054FE204610BD024B01211868036818
:108890001B68184780470020021C18BF01220321D3
:1088A000014807F0A1BC00BF0004024010B50C460F
:1088B000F9F744FD022808D14FF47A704443B4FB21
:1088C000F0F0BDE81040F9F741BB2046BDE810408C
:1088D00007F0D8B90321014807F08FBC000402401B
:1088E00010B5094C094802F0EBFC20460B2107F0BB
:1088F0006FFC002320461A460B2107F0A7FBBDE8BA
:10890000104007F0A5B900BF00000240E6C0010812
:1089100008B5022007F000F907F062F900F05EFCEC
:1089200007F088F900F048FE07F0E8FE0C48FBF776
:10893000ABF84FF4E13008F045FA0A4B1A680AB96F
:10894000094A1A60094B1A680AB9074A1A600848A6
:1089500002F0B6FCBDE80840064802F0B1BC00BF1A
:108960001188000860480020790C01086448002044
:10897000E8BD010800BE0108F7B50446FFF752FD47
:10898000234600252146214A04F1480043F83C2BA8
:10899000E5635D601E4B1F4E41F8443F01F032F825
:1089A0001D4B84F85C50A3651C4BC4E91A55236623
:1089B0001B4B84F8705063661A4B1B48636702F0C8
:1089C0007FFC3368194F01933B68194D00932B6866
:1089D000184A1B2104F121000FF09EFA296804F1C6
:1089E000110002F0A6FD396804F1150002F0A1FDA6
:1089F000316804F1190002F09CFD296804F11D00A2
:108A000002F097FD204603B0F0BD00BF4CC1010845
:108A100038C201086400F81FCCC20108FCC201087A
:108A2000E8C2010870C201081AC101085400F81F09
:108A30005000F81F2FC1010810B5094CFFF768FF5F
:108A40002368DB0709D40748FFF796FF0123064A8E
:108A50000649044823600CF094FF024810BD00BF93
:108A60007847002084470020000000203D8800084F
:108A700038B5064D064C2B6813F0010F04D1FFF7F3
:108A8000DBFF012320602B60206838BD7C4700207D
:108A9000FC4700204FF4FA71FFF72CBD08B50B21FD
:108AA000054807F0AFFB28B1BDE808400B2102489C
:108AB00007F0BCBB08BD00BF0000024008B519B1FB
:108AC000BDE80840FFF70CBF044802F0F9FBBDE821
:108AD000084002220B21024807F0F6BA02C1010841
:108AE00000000240F8B50446384804F1440502F09D
:108AF000E7FB2846002100F087FD0021284600F012
:108B000099FD334D2046FFF7BDFC03F06DFE204676
:108B10000021FFF7D3FF0BF091FD0CF08DF801223F
:108B20000C21284607F0D0FA07F000FF04F14800B6
:108B300000F056FF23682046DB6804F1640600213C
:108B40009847244F0021304600F078FE07F0CAFB1A
:108B5000214802F0B5FB08F01BF807F06BF8384627
:108B600001220D2107F0B0FA012238460E2107F04C
:108B7000ABFA0021084607F097FE04F1580000F018
:108B8000EDFD0121304600F059FE4FF4E13008F0D0
:108B900019F9124802F094FB28460C2107F018FB43
:108BA000002328461A460C2107F050FA0120002124
:108BB00007F0E0FE0CF052F80BF066FC07F0B4FE94
:108BC0002046BDE8F840FFF76ABC00BFB4C001080A
:108BD0000004024000000240D8C00108B2BF0108F2
:108BE00038B50546FFF75AFF044628B1002128464C
:108BF000FFF764FF07F02CF806F032FF05460CB1D2
:108C0000FFF76EFE284638BD70B50C46064615497E
:108C100020460DF09DFF20B9002120460DF07AFF7F
:108C200070B1114920460DF0D7FD0DF09BFF0146B4
:108C30000E4802F045FB4FF4BB710D48FAF75EFF9A
:108C40003046FFF72BFF054648B93046FFF7C8FF0F
:108C5000014620460DF07CFF08B1FFF741FE284693
:108C600070BD00BF3333534000007A4416BE010884
:108C700045BE010870B52D4AD6B013680546DB071E
:108C800005D42B4900F164030B60012313602949CB
:108C90002846FFF7B9FF0646274802F011FB0021DE
:108CA00005F1440000F0C6FC244C254BE360254B45
:108CB0002361254BA360254B6360254B2360254B27
:108CC0006361254BA361254BE36104F110030FCBD6
:108CD0008DE80F0094E80F000CF0DEF9002305A8E2
:108CE000EB632B640CF060F99DF8143005F13C0443
:108CF000012B14D1DDF8153005A8EB63DDF8193030
:108D00002B640CF021F9164802F0DAFA082120460B
:108D100002F03CFBBDF91611124802F0D1FA3146BF
:108D20002846FFF7CBFE56B070BD00BF7447002049
:108D3000804700200000404081BD0108C84F00204E
:108D400085FC00080DFC000889880008D58800080B
:108D500099880008C1B20008B52C0008F52C00085D
:108D6000A2BD0108C8BD010808B5FFF739FF0349D6
:108D70000DF032FD0DF01CFF80B208BD00007A44FA
:108D800070B507490546FFF73FFF06460CF0A2F80D
:108D9000044631462846FFF791FE204670BD00BFCD
:108DA000000040407FB5F82300F1580506462846EC
:108DB0008DF80F3000F0D8FC02230DF10F01009365
:108DC0000122A123284600F0D3FC4FF400430822DF
:108DD000009306F16801A1230446284600F0F2FC46
:108DE0000440E4B2284600F0C1FC204604B070BD47
:108DF00030B58BB0044608F09FF90146574802F0A1
:108E00005FFA574802F05CFA204600F08BFB04F151
:108E1000580500F0BDFA00F069FA5248524902F0D4
:108E20004FFA284600F09AFC38B9504802F048FA48
:108E300040F233114E48FAF761FE06F009FF204672
:108E4000FFF7B0FF20B94FF49C714948FAF756FE7E
:108E500094F86F3094F86920049394F86E3094F885
:108E60006810039394F86D304248029394F86C3084
:108E7000019394F86B30009394F86A3002F020FA72
:108E8000284600F035FA284600F094FA04F144052B
:108E900084F8700004F1740000F012FC00212846F0
:108EA00000F0B2FB012000F0BBFD0021284600F0DD
:108EB000C1FB012000F0D2FD2046FFF7DBFE00F0F1
:108EC000C5FA2D4802F0FCF94FF4FA700EF04CF997
:108ED000054600283AD1294802F0F2F9284802F064
:108EE000EFF9284802F0ECF9274802F0E9F92748A1
:108EF00002F0E6F9264802F0E3F9264802F0E0F92C
:108F0000254802F0DDF9254802F0DAF9244A25491E
:108F1000254802F0D5F92549254802F0D1F9254820
:108F200002F0CEF904F12101234802F0C9F907A8A3
:108F300007F07CFB07A802F019F901461F4802F070
:108F4000BFF9104802F0BCF90BB030BD1C4802F06C
:108F5000B7F928460EF010F9C0E700BF85BE01083A
:108F60009BBE0108B2BE0108A0860100CDBE01086B
:108F700045BE0108E3BE010818BF01084BBF010848
:108F800061AC010889BF0108BABF0108C9BF010867
:108F9000EBBF01080EC0010832C0010862AC010835
:108FA00036AA010811AA010855C0010865C00108C8
:108FB0006CC0010877C0010897C00108A2C0010871
:108FC0007FBF01082DE9FF4100F15805284600F058
:108FD000CBFB04240226284F013C14F0FF0433D0BD
:108FE000A123012239460096284600F0C1FB4FF428
:108FF0000043804600930422A12302A9284600F0E2
:10900000E1FBB8F1000F01D10028E5D09DF8083050
:10901000442B20D19DF809306E2B1CD10DF10A0094
:1090200002F079FA0223013084B221460DF10900E1
:109030008DF8083002F090FA002303220093A02359
:1090400002A9284600F094FB284600F08FFB20463A
:1090500004B0BDE8F0814FF488430024ADF8083037
:109060006E2300210DF10B008DF80A3002F074FA26
:109070000094A0230522E3E780BD010838B50C4623
:109080001131054603F082FA214651F8683F28461F
:109090002B604B686B6038BD024B186803685B68D7
:1090A000184700BF0C480020024B186803689B68F3
:1090B000184700BF0C4800200023F0B51370144679
:1090C000022205460C4E85B030688DF80F100368FB
:1090D0000092DF6801222B460DF10F01B84748B11D
:1090E0004FF4004230682146036800921E69012255
:1090F0002B46B04705B0F0BD0C48002030B585B018
:109100008DF80D200022074B8DF80C101C6803A968
:1091100023680092DD68022203462046A84705B076
:1091200030BD00BF0C48002037B54FF40045064B5A
:109130001C68236800951D6913460A4601462046AF
:10914000A84703B030BD00BF0848002037B5002550
:10915000054B1C6823680095DD6813460A460146E6
:109160002046A84703B030BD0848002037B5022587
:10917000054B1C6823680095DD6813460A460146C6
:109180002046A84703B030BD08480020024B1868AD
:1091900003681B68184700BF08480020024B186886
:1091A00003685B68184700BF08480020024B186836
:1091B00003689B68184700BF084800204FF47A7383
:1091C0005843B0FBF3F0F8F7C1BE10B50446FFF703
:1091D0004FFC2146BDE81040FFF7F4BE10B5424CED
:1091E0000BF07EFA20460222002106F06DFF0122DC
:1091F0002046114606F068FF20460122022106F0B3
:1092000063FF20460222032106F05EFF2046002273
:10921000042106F059FF20460222082106F054FFDF
:1092200020460122092106F04FFF204601220A2193
:1092300006F04AFF204602220B2106F045FF06F009
:10924000F9FC002320461A460C2106F0FFFE2046BA
:1092500000220C2106F0C8FF2046002204F580649D
:109260000F2106F031FF20460122002106F02CFFDD
:1092700020460022022106F027FF2046002203217B
:1092800006F022FF20460222062106F01DFF20469E
:109290000022082106F018FF20460022092106F0CE
:1092A00013FF204601220C2106F00EFF2046022269
:1092B0000D2106F009FF204602220E2106F004FFD0
:1092C000204602220F2106F0FFFE002304F58064F1
:1092D00020461A460D2106F0B9FE2046BDE8104092
:1092E00000220D2106F080BF0000024007F006BA00
:1092F0001C4B00B51A6889B0D2075FBF1A4A1060CC
:1093000001221A60194B0493194B0593194B0393CF
:10931000194B0293194B0793194B069308AB13E9AA
:1093200003008DE8030002AB0FCB0BF063FD90B19F
:10933000144801F0C5FF00221348114606F0C4FE90
:109340000F2302220021104806F05EFD09B05DF8EF
:1093500004EB0BF0E9BC69210C4809B05DF804EBA3
:10936000FAF7CCBB044800200C4800209990000874
:10937000A9900008B9900008FD900008C1B200084B
:10938000BD910008DEC1010800000240EFC10108E4
:10939000002307B5ADF8043001238DF8063001989D
:1093A0000BF0FAF806F046FC03B05DF804EB0BF0A6
:1093B00045B90000194B10B51A688CB0D2075FBFD1
:1093C000174A106001221A60164B0793164B05933B
:1093D000164B0693164B0893164B0993164B0A939C
:1093E000164B0B930CAB13E907008DE8070005AB98
:1093F0000FCB0BF01FFA044601220F21104806F094
:1094000063FE3CB10F4801F05BFF0BF0F1F9204621
:109410000CB010BD0C4801F053FFF8E700480020E5
:1094200008480020299100084D9100086D9100081E
:109430008D9100089D910008AD910008C1B200080F
:109440000000024060C1010893C101082DE9F04706
:109450009EB002F003FDDFF8C890284C284E294F3B
:1094600016AD50B9CDE91944CDE91776CDF858902D
:10947000009495E80F0002F0F7FC234B4FF0000A30
:109480001793224B4FF001081693214B09A918930B
:10949000204B28461993204BCDE91C76CDE91A3490
:1094A0000423CDE9093A8DF8298009F095FB09F0EC
:1094B00087FB0EF0C9FC514610220CA80DF0A8FE47
:1094C000164BCDE91044159303238DF836800B938A
:1094D00002AC0BAD0FCDCDE91376CDF848900FC49B
:1094E0002B68236014AB93E803008DE8030010ABF6
:1094F0000FCB03F075F81EB0BDE8F087C1B20008CD
:10950000CDB30008F9B30008C1450108894401083A
:10951000994301083143010845430108CB910008F4
:10952000E90601082DE9F047044606F099FA1E49BC
:1095300005460DF051F90DF015FB01461B4801F0F1
:10954000BFFE4FF0804128460DF0E4FA48B30025F5
:10955000DFF86090DFF85080154E06F081FA49463A
:1095600007460DF0EBFAA8B9414638460DF034F93C
:109570000DF0F8FA0146304601F0A2FE236885F0AE
:1095800001052046DB68294698474FF47A7006F0BB
:1095900079FBE2E723682046BDE8F047DB6800215D
:1095A0001847BDE8F08700BF00007A44B1C1010848
:1095B000C3C101080000204008B50D49012006F094
:1095C000F5FE0C490B2006F0F1FE0B490A2006F0CF
:1095D000EDFE0A49042006F0E9FE0949072006F0DD
:1095E000E5FEBDE808400749052006F0DFBE00BFE4
:1095F000053F010815420108A14001082D4301085B
:109600008142010809430108002310B50C461A469F
:109610000D21074806F01AFD14B1012C00D010BD31
:109620002246BDE810400D21014806F0DDBD00BF17
:1096300000080240002310B50C461A460C210748CA
:1096400006F004FD14B1012C00D010BD2246BDE887
:1096500010400C21014806F0C7BD00BF00000240C9
:109660000BF022BA084611461A460BF0ABBA084670
:1096700011461A460BF038BA084611461A460BF046
:1096800065BA00000C2110B1024806F0A1BD0148E6
:1096900006F0A4BD0004024010B561B1FFF7E8F97F
:1096A00004460BF0DFF901462046FFF7ADFABDE8AE
:1096B00010400BF0D3BABDE810400BF0BDBA00006B
:1096C00070B588B0FFF7D4F91D490546FFF79CFA3D
:1096D0000C2106461B4806F07BFD00230C211A4690
:1096E000184806F0B3FC0021012007F043F91022CE
:1096F00000210DEB02000DF08BFD134B02AC029329
:10970000124B0693124B039308AB13E903008DE849
:10971000030094E80F000BF0B9FA60B10BF0C4F944
:1097200001460C4801F0CCFD3146284608B0BDE8A2
:109730007040FFF7C3B9084801F0C2FDF4E700BF6D
:1097400000004040000402408596000885FC0008A7
:109750002D0A010840C2010856C20108014806F05E
:10976000AFBD00BFA086010006F07ABD06F094BD33
:109770002DE9F041069F1E4607F00303032B8046A8
:109780000C46154603D12F210D48FAF7B7F92046AC
:10979000BC07324629460AD506F0CCFD10B101209F
:1097A000BDE8F0810123002088F80430F8E7FB07CA
:1097B00002D506F0CDFDF1E706F0AEFDEEE700BF05
:1097C00084C201082DE9F041069C0D46E107804660
:1097D00016461F4603D54C210D48FAF78FF9A2070C
:1097E00003D54F210A48FAF789F923043A4631464E
:1097F00028460AD506F0BAFD10B10120BDE8F08177
:109800000123002088F80430F8E706F077FDF3E73D
:1098100084C2010808B50321034806F0EEFC0030BD
:1098200018BF012008BD00BF000402400A460248DC
:10983000032106F0D9BC00BF0004024008B581B185
:10984000012303211A460A4806F000FC03210848B8
:1098500006F0BEFCBDE8084003220548114606F0AC
:10986000D5BB0122BDE808400321014806F02CBC0D
:109870000004024006F038BF084611461A469DF81B
:10988000003006F0D1BF06F07DBF06F095BF084658
:1098900006F00EBEDFB50023CDE90133ADF80C3084
:1098A00001238DF807308DF808306FF01D038DF817
:1098B00009300723044601A88DF80A3001F03DFC69
:1098C000236806461B6820460F469847864277EB7A
:1098D0000103B4BF0120002004B0D0BD7047704721
:1098E0007FB500F10806054630460C4601F0AEFE95
:1098F00060BB334801F0E4FCA27C617C314801F09C
:10990000DFFC637C3BB16868002103681B689847F3
:10991000022000F085F8A37C3BB168680021036851
:109920005B689847022000F099F861684E2918D0CA
:109930004F2916D0452914D015212348FAF7DEF80F
:109940001621224B224A20480DF00CFB64213046A0
:1099500001F068FE0028CFD142211B48FAF7CEF86B
:10996000CAE7A368073B022B15D81A4AD25CE36802
:109970000A2B18D009DC052B16D033211248FAF730
:10998000BDF8124B144A3421DDE70F2B0CD0142BF9
:10999000F3D1022308E023210B48FAF7AFF80B4B71
:1099A0000E4A2421CFE70123A07C0290607C019025
:1099B000207C0090206807F03FFA04B070BD00BF23
:1099C00017C3010870C3010830C30108AFA801081C
:1099D000B4C3010814C30108E4C3010818C4010892
:1099E00010B5044607F0FAF904F10800BDE810408C
:1099F00001F02FBE084607F0EFBA07F015BA084687
:109A000007F01ABB10B50446044BC0E90031012130
:109A1000083001F029FE204610BD00BF98C30108A0
:109A2000042817D8DFE800F00309100E1200002305
:109A300003211A46084806F009BB00220321064804
:109A400006F042BB0222F9E70122F7E703210248B0
:109A500006F060BB704700BF00000240042817D822
:109A6000DFE800F00309100E1200002302211A465D
:109A7000084806F0EBBA00220221064806F024BB93
:109A80000222F9E70122F7E70221024806F042BB71
:109A9000704700BF00000240406803681B68184719
:109AA000406803685B681847406803689B6818470C
:109AB00040680368DB681847406803681B691847FB
:109AC00070470000436910B504469BB983698BB9A0
:109AD0008168094801F0F4FBA168084801F0F0FB37
:109AE00041F28830F8F732FABDE8104031210448DD
:109AF000FAF704B810BD00BFFBC4010819C501087E
:109B000030C50108C0E903120346002210B5074C16
:109B1000C0E905224460064C8460064C0460064C93
:109B2000C0E90741586280F8282010BD69C50108C6
:109B30006FC501087CC501089CC50108436970B563
:109B400005460C4633B3012913D002291CD0002945
:109B50004CD10A46184601210BF010FE2246022184
:109B600068690BF00BFEE868BDE870400368DB68CD
:109B700018470A4618460BF001FE22466869022182
:109B8000BDE870400BF0FABD0E21BDE870401846EC
:109B90000BF056BD806948B301290CD0022914D0BE
:109BA00021BB0A4601210BF0DAFE22460221A869F8
:109BB0000BF0D5FED7E70A460BF0D1FE2246022174
:109BC000A869BDE870400BF0CABE1A4601210BF02F
:109BD000C6FE01222146A8690BF0C1FE0122042124
:109BE000A8690BF0BCFE01220821E9E770BD80687E
:109BF000FFF7A4BF38B504460C2000F075FC0546FD
:109C000021690BF0F9FC656128460BF0A5FD38B31E
:109C100042F26252A168144801F052FB002384F81A
:109C200028300C2000F060FC054621690BF0B8FDDF
:109C3000A56128460BF0FCFDA0B14FF41552A168B8
:109C4000094801F03DFBF021A0690BF07EFE0123E5
:109C500084F828302046BDE838400221FFF76EBF67
:109C60006061DEE7A061F5E750C401080221FFF75B
:109C700065BF034640690A4610B104210BF07EBD62
:109C8000986910B104210BF06ABE70470000000013
:109C90002DE9F04790F8284006460F46002C3CD0AE
:109CA000FEF7E6FE0546002F51D0FFF75DF80F24C2
:109CB00040F64759DFF8B08048450EDC0146404683
:109CC00001F0FEFA2B684FF47A711B692846984719
:109CD0002846FFF749F8013CEED1B168204801F071
:109CE000EFFA00213046FFF7C4FF1E24DFF87CA006
:109CF000DFF87C802846FEF773FF81460CF0FCF805
:109D000015A3D3E900230CF0DFFB48B12B6840F228
:109D1000DC511B69284698473C462046BDE8F08741
:109D2000514648460CF058FD0CF01CFFB168024645
:109D3000404601F0C5FA2B6864211B692846984704
:109D4000013CD7D101213046FFF793FFE5E7B16829
:109D5000044801F0B5FAF5E7666666666666064091
:109D6000A9C40108E5C4010871C4010800007A44CF
:109D7000BEC4010870B508B9002070BD0023466854
:109D80004D1CB5421360F7D803685C185B5C03F0A8
:109D90001F03A3F1180103290DD81449194411F820
:109DA000180C0544AE42E7D3042819D8DFE800F0C8
:109DB00003070B181200002013600130DDE7637801
:109DC00001201360F9E7B4F8013002205BBA9BB2BE
:109DD0001360F2E7D4F8013004201BBA1360ECE7FB
:109DE000D4F801301BBA1360E7E700BFBCC5010817
:109DF000F7B51F46436816464A1C9A4205460C466C
:109E000017D803685B5C03F0C003402B11D196B1F7
:109E100001AAFFF7AFFF50B1019A04446B68A11883
:109E2000994206D8296810440C4434603A6003B063
:109E3000F0BD0020FBE73046F9E72DE9F7439946EE
:109E4000436817464A1C9A4280460D4624D8036848
:109E50005B5C03F0C003402B1ED1FFB101AAFFF7EA
:109E600089FF0446A0B1019E09F10109B14513D350
:109E70000544D8F8043072199A420DD8D8F8001069
:109E80003246294438460DF09BF900233444BB5533
:109E9000204603B0BDE8F0830024F9E73C46F7E72D
:109EA000F0B581B3172A1CD8D3B2A3F11804032C40
:109EB0008CBF0024154C8D689CBFE41814F8184C16
:109EC0006F1C4E6804EB070CB4451CD20E68184397
:109ED0008F60E3007055083B13F1080F0BD1601C35
:109EE000F0BDFF2A05D9B2F5803F34BF19231A23EC
:109EF000DBE71823D9E788680D68461C8E6022FAD4
:109F000003F62E54E7E70020EAE700BFBCC50108CE
:109F1000172BF8B50D4616461C4612D8DBB2A3F136
:109F20001802032A8FBF0022144A9B1813F8182C1A
:109F3000AB680132234413446A6893420BD3002078
:109F4000F8BDFF2B05D9B3F5803F34BF19231A2381
:109F5000E5E71823E3E722462946FFF7A1FF074676
:109F60000028ECD02868AB68314618440DF028F979
:109F7000AA68E0192244AA60E2E700BFBCC5010854
:109F800018B10023C0E9001283607047436873B5BD
:109F900014464A1C9A4206460D4602D9002002B0D9
:109FA00070BD03685B5C13F0C00FF7D1002CF5D0D7
:109FB00001AAFFF7DFFE0028F0D03268019B525D56
:109FC00012F0E00F18BFDB432360E8E70A1EABBFC7
:109FD000014601460020D243B8BF2020FFF760BFF2
:109FE00003685B5C03F0E001E02907D132B1A3F123
:109FF000F5014B424B411370012070470020704720
:10A00000836810B544685A1CA24208D2002914BFC4
:10A01000F524F424016882600120CC5410BD002096
:10A02000FCE7F0B446684F1CB74208D805686C5C82
:10A0300004F0E004402C02D1F0BCFFF7D9BE0020B0
:10A04000F0BC704713460A4601464020FFF760BF48
:10A05000F0B446684F1CB74208D805686C5C04F041
:10A06000E004602C02D1F0BCFFF7E7BE0020F0BC9A
:10A070007047F0B446684F1CB74208D805686C5C5E
:10A0800004F0E004602C02D1F0BCFFF7B1BE002068
:10A09000F0BC704770B5054608460C460DF0A2FFAF
:10A0A000224603462946BDE870406020FFF730BFD6
:10A0B000836841685A1C8A423FBF8260BF220168A0
:10A0C000012034BFCA54002070470368585CA0F1D7
:10A0D000BF0358425841704713B5036814465B5C90
:10A0E00003F0E003A02B07D142B101AAFFF742FE23
:10A0F000019B236002B010BD0020FBE71046F9E78A
:10A10000836841685A1C8A423FBF8260FF2201680F
:10A11000012034BFCA540020704730B18068013834
:10A1200088428CBF0020012070470120704708B58D
:10A130000246FFF7F2FF30B91268505CA0F1FF034E
:10A140005842584108BD0120FCE743688B4207D9BB
:10A1500003685B5C13F0C00F0CBF01200020704748
:10A160000020704743688B4208D90368585C00F0B0
:10A17000E000A0F14003584258417047002070476A
:10A1800043688B4208D90368585C00F0E000A0F1F6
:10A1900060035842584170470020704743688B4223
:10A1A00008D90368585C00F0E000A0F1A003584211
:10A1B000584170470020704710B50446FFF7EEFF86
:10A1C00050B163688B4208D92368585C00F01F00C7
:10A1D000A0F11F035842584110BD0020FCE743681E
:10A1E0008B4208D90368585C0C30C0B201288CBF80
:10A1F000002001207047002070470023C0E9013390
:10A2000003690160C360704703468068F0B51D684C
:10A21000013090FBF5F405FB14005C68A04224D0EB
:10A2200000269642304601D11046F0BD8F5DD3E93D
:10A2300002452F559C681D68671C97FBF5F405FBCC
:10A2400014745F689C60BC4204F1010402BF94FB7B
:10A25000F5F705FB17475F6094FBF5F705FB17441F
:10A260005D68AC42E1D00136DBE70020DDE70000AD
:10A27000F8B503680446002B0D46164603DC3E2164
:10A280002948F9F73BFC3246002128460CF0C0FF74
:10A29000D4E90170B8420CD00021236801EB070C0F
:10A2A0009CFBF3F203FB12C2904205D100208842CE
:10A2B00004D14FF0FF3031E00131EFE7C21992FBDA
:10A2C000F3FE03FB1E2ED4F80CC01CF80EE0BEF10A
:10A2D0000A0F26D128B3013A92FBF3F103FB1122B6
:10A2E000002106F1FF3E71450ED2E7686368FB5C12
:10A2F0006B5467682668013797FBF6F306FB137704
:10A30000013188426760EEDA1CF802300D2B4FF005
:10A31000000304D1054405F8013C0138F8BD2B5475
:10A32000FCE70130C3E700BFC0C501084B1C017347
:10A3300043738B1C03318373C17370472DE9F04164
:10A34000074688461E4615461AB952211548F9F7A0
:10A35000D5FBD7E90143A34221D2E41ADEB1A3B968
:10A36000A5420ED33B7B3370BB6839682246194443
:10A3700040460CF025FFBB682344BB602046BDE887
:10A38000F0817B7B33702C46EEE7A54201D3FB7B4B
:10A39000E9E7BB7BF6E7AC4228BF2C46E4E70024A4
:10A3A000ECE700BF08C601080023C0E90012836083
:10A3B000704710B504460846C4E900120021A160A8
:10A3C00021730CF025FF204610BD000038B515465E
:10A3D000D0E9012304465819904202D9257B55B192
:10A3E000D51A20682A4618440CF0EAFEA3681D44DA
:10A3F000A560012503E01B210248F9F77FFB2846F1
:10A4000038BD00BF44C6010807B501228DF807100A
:10A410000DF10701FFF7DAFF03B05DF804FB0068F8
:10A42000704780687047002383607047D0E901203F
:10A43000101A7047026880681044704738B5D0E938
:10A4400001230D4659189142044602D9017B21B1DE
:10A45000D51AA1682944A16038BD49210148F9F7FE
:10A460004DFBF6E744C6010813B5044601A801F008
:10A4700073F8022201A92046FFF7A8FF02B010BD21
:10A4800013B50446684601F05DF80522694620468A
:10A49000FFF79CFF02B010BD13B5044601A801F000
:10A4A0005BF8022201A92046FFF790FF02B010BD21
:10A4B000014608B5034800F003FF0C210248F9F7F4
:10A4C0001DFB00BF7CC601089AC6010808B50448F8
:10A4D00000F0F6FEBDE808401E210248F9F70EBB69
:10A4E000FDC601082AC7010810B500F085FF044623
:10A4F00030B9044800F0E4FE27210348F9F7FEFADA
:10A50000204610BDEBC601082AC7010800F074BF41
:10A5100010B9024800F0D4BE00F058BFD6C60108FA
:10A52000FFF7E2BF00F068BFFFF7F2BFFFF7F0BF31
:10A5300010B5074C0A44914200D110BD11F8013BFF
:10A540004340DBB234F8133083EA1020F3E700BF56
:10A5500066C70108F8B50E46054680B14F1C38465F
:10A5600000F04AFF044640B13A4600210CF050FE8C
:10A570003246294620460CF023FE2046F8BD04460C
:10A58000FBE738B50D46044628B10DF02BFD2346F8
:10A590002044834201D1002038BD13F8012BAA4288
:10A5A000F7D10120F8E773B505460E4600240CF0FC
:10A5B00005FD2246046001A928460DF025FE05464A
:10A5C0000CF0FCFC0368222B0BD0019B1B7843B9D9
:10A5D000A542ADBF2846204601232346336002B082
:10A5E00070BD01232046F9E72DE9F04F05464FF0F5
:10A5F000010B002687B0CDE9031206F10903122BE7
:10A600008CBF0320022000F0F7FE0090E8B1324634
:10A6100036490DF0B5FC039B53F82690EDB90024A4
:10A62000009800F0D3FEBBF1000F02D1284600F0E5
:10A63000CDFE84B1049B0136B34225464FF0000B9A
:10A64000DBD1204607B0BDE8F08FBBF1000F02D18F
:10A65000284600F0BBFE0024F3E7254B4FF000082E
:10A66000B9F1000F08BF994648460DF0BBFC0190B8
:10A6700000980DF0B7FC0290284649460DF0DFFC2B
:10A68000B8B928460DF0AEFCDDE9012301309B1A74
:10A6900008FB030000F0B0FE04460028BFD00346CC
:10A6A0002F4618F1FF3809D2394618460DF092FCB2
:10A6B000B6E7019B08F101081844DEE74946384631
:10A6C00005930DF0BCFC059BA0EB070A52463946EA
:10A6D00018460DF0A1FC009950440DF07BFC019A46
:10A6E000029B9244C3185744DBE700BF41AA01080C
:10A6F00063AC010830B580B10346021F00F11804B5
:10A7000052F8045F8D4208D0A242F9D11C301A469B
:10A7100014680433013401D1116030BD8342F6D195
:10A72000FBE7000068B10849431E13F8010F00B9A8
:10A7300070470A5C02F00302022A08BF2038187032
:10A74000F3E70120704700BF64EB010870B50446D1
:10A7500080B1064600EB8105AE4204D12046BDE83B
:10A76000704000F033BE56F8040B0028F4D000F01F
:10A770002DFEF1E770BD00002DE9F74F8B460092EA
:10A78000002839D00027C35D93BB1D46064600EB69
:10A79000070A02463848524538D103B10135002D29
:10A7A00063D00137384600F027FE804600285AD093
:10A7B0003A4600210CF02CFDA80000F01DFE0446D6
:10A7C000002854D04FF000090021B2452CD131B1FE
:10A7D0004046FFF7BFFE002849D044F82900404614
:10A7E00000F0F4FD009B1D60204603B0BDE8F08F33
:10A7F0000137B7F5807FC6D10024254620460024C6
:10A800002946FFF7A3FF009B1C60EDE712F8011B30
:10A81000594504D1002BBED001350023BBE7095CAC
:10A82000090758BF0133B6E716F8013B5B4512D163
:10A830000029CAD04046FFF78DFEC0B109F10103DF
:10A8400044F829003A460021404601930CF0E0FC10
:10A85000019B9946B8E7084A985C02075CBF08F874
:10A8600001300131B1E70446C8E72C46BCE7404659
:10A8700000F0ACFDC2E700BF64EB01082DE9F7432F
:10A88000002506460820884691461F46009500F0A0
:10A89000B3FD0446002865D0C0E9005530460DF0F0
:10A8A000A1FB01280FD133782A2B0CD109F1FF33FA
:10A8B000C4F80080636022684A4502D263684B4551
:10A8C00040D3294B0DE02D213046FFF75AFE0546B7
:10A8D000B8B9019001A93046FFF765FE019B63B14D
:10A8E000224B3B6000992846FFF730FF002C35D003
:10A8F000204600F06BFD002430E0C4E900001D4656
:10A90000D9E76A462D213046FFF736FF009B054602
:10A91000013B012B01D9164BE3E7002301A9006895
:10A920000193FFF740FE2060019B0BB1114BD8E76C
:10A9300001A96868FFF737FE6060019B002BBAD061
:10A940000D4BCEE7424501D3434501D20B4BC8E73F
:10A9500000992846FFF7FAFE00233B60204603B02B
:10A96000BDE8F0830546BDE742CA0108BCC901083D
:10A97000DBC9010804CA010823CA010862CA010828
:10A9800008B520B34A1C22D0062920D8DFE801F000
:10A99000040D101316191C00002303600CF01AFD9F
:10A9A0000840431C5842584108BD00234360F5E766
:10A9B00000238360F2E700238361EFE70123C36094
:10A9C000ECE700230361E9E700234361E6E70120A8
:10A9D000EAE770B506460D1F01F1180455F8041F8B
:10A9E0004B1C03D1A542F9D1002070BD3046FFF7C2
:10A9F000C7FF0028F6D0F8E700290B46B8BFCB1DEB
:10AA00004A4202F0070201F0070158BF51420122F9
:10AA1000C3F3C703C9B202FA01F1C25C1143C154C6
:10AA2000704700290B46B8BFCB1D4A4202F007020F
:10AA300001F0070158BF51420122C3F3C703C9B255
:10AA40008A40C15C21EA0201C15470470B460029CB
:10AA5000B8BFCB1DC3F3C703C05C4B4203F0070371
:10AA600001F0070158BF5942C9B2084100F0010086
:10AA700070472DE9F047089E8A4690461D46DDF84E
:10AA80002890074610B11446A24507D875B901228F
:10AA900000240B9B1A602046BDE8F087214638460B
:10AAA000FFF7D4FF00285ED10134EDE7099B023B9C
:10AAB000042B04D8DFE803F0282C2C3034006B681A
:10AAC00001336B6028460CF085FC013108BFB0F102
:10AAD000FF3FDCD031462846FFF752FF0028D6D191
:10AAE00017B3044621463846FFF7B0FF00283FD190
:10AAF0000134A245F6D10446013E042E16D8DFE803
:10AB000006F0282A2C2E3000AB680133AB60D9E761
:10AB1000EB680133EB60D5E72B6901332B61D1E79B
:10AB20006B6901336B61CDE73C46E5E72C60284655
:10AB30000CF050FC013108BFB0F1FF3FA7D0B9F1D4
:10AB4000000FA4D049462846FFF743FF0028A2D0B3
:10AB50009DE76C60EBE7AC60E9E7AC61E7E7EC60D0
:10AB6000E5E72C61E3E7A04595D0002DC4D18EE741
:10AB7000A045C1D18FE72DE9F04F4FF000098BB010
:10AB800006461C200C469046CDF8249000F034FC7C
:10AB90000546002800F0E0801C2000F02DFC074650
:10ABA000002800F0D9804B464FF0FF3245F82320B3
:10ABB00047F823200133072BF8D100230121D4F8D3
:10ABC00000A00DF12409CDE90031CDE902793C2145
:10ABD000234652463046FFF74CFF0999002940F0C2
:10ABE0008E80824502D12846FFF784FD02234FF074
:10ABF000010AD4F804B0CDE900A3CDE902592346F7
:10AC00005A463C2106F10800FFF733FF099B002B51
:10AC100075D183456BD151462846FFF76BFD032361
:10AC20004FF0020AD4F808B0CDE900A3CDE90259EB
:10AC300023465A46182106F11000FFF71AFF099B18
:10AC4000002B5CD1834565D151462846FFF752FD64
:10AC500040F26F1BA3690593E368049306F11403A4
:10AC60000693DDF810A006F11303079351460698EA
:10AC7000FFF7ECFE20B105990798FFF7E7FE88B9CA
:10AC8000BBF1010B0ED0E36820460133E3600CF00A
:10AC9000A1FB013108BFB0F1FF3F44D101234FF0C8
:10ACA000000A0993099B53BB049B534544D10421DB
:10ACB0002846FFF71FFD05230622D4F810A0CDE992
:10ACC0000032CDE90259234652460C2106F1180004
:10ACD000FFF7CFFE099B93B9824510D06369A3EBC0
:10ACE0000803042B31D94FF0FF33099307E04246A4
:10ACF00021463046FFF73FFF099000288FD02846B5
:10AD000000F064FB17B1384600F060FB09980BB007
:10AD1000BDE8F08F424621463046FFF72CFF0990F0
:10AD2000002895D0EBE7A36929462046D4F80CA06B
:10AD30000593FFF74EFE99E7424621463046FFF75E
:10AD40001AFF09900028B6D0D9E74246214630467E
:10AD5000FFF711FF0990D2E74FF0FF330993002D61
:10AD6000D4D00027CBE700002DE9F04F002487B0B6
:10AD7000894692462C2103AA9846109D0394FFF71A
:10AD8000FBFC074688B93E4B2B6003993846FFF71A
:10AD9000DDFC07B0BDE8F08FD0F800B072685A450E
:10ADA0001CD2304600F012FB0134039BA342ECD9C5
:10ADB00057F824602F213046FFF7E3FBA8B92B4654
:10ADC000304642465146FFF759FD2B680646002B98
:10ADD000E2D00028D9D000F0F9FAD6E75946484623
:10ADE000FFF70AFE0BF1010BD8E700232F213046B5
:10ADF00004AA0493FFF7C0FC049906464B1E012BDE
:10AE000004D9204B2B60FFF7A1FCBEE742462B463E
:10AE100051460068FFF732FD2A6883462AB108B11F
:10AE200000F0D4FA04993046EDE72D213068FFF7A1
:10AE3000A8FB18B908F1FF32CBF80420002305A9BC
:10AE400070680593FFF7AFFB059A00901AB10E4AA0
:10AE500058462A60E4E7DBF80020DBF80410914252
:10AE600005D230460499FFF771FC58469AE711461F
:10AE700048460192FFF7C0FDDDE900321A44ECE7D5
:10AE800087CA010899CA0108BECA01082DE9FF4115
:10AE900000230E460393144602B902AC236048B95E
:10AEA0000546564B236003992846FFF74FFC04B034
:10AEB000BDE8F08103AA2021FFF75EFC039B054655
:10AEC000062B02D04E4B2360EDE71A2200213046BC
:10AED0000CF09EF9009400223C2331462868FFF7CD
:10AEE00043FF2268002ADED100943C2306F10801CA
:10AEF0006868FFF739FF2268002AD4D1009418232C
:10AF000006F11001A868FFF72FFF2368002BCAD1B4
:10AF10006869FFF707FC07223A496869FFF764FB95
:10AF200080460DF05FF8012806F1130706D198F866
:10AF300000303F2B04BF2A2388F80030002208236A
:10AF4000394640460094FFF70FFF404600F03EFAB6
:10AF50002268002AA7D107213846FFF777FD30B1D4
:10AF600011463846FFF748FD0721FFF75AFDEF6805
:10AF700006F1140838460DF035F8012804D13B7865
:10AF80003F2B04BF2A233B70202300224146384632
:10AF90000094FFF7E9FE00214046FFF742FD2368D9
:10AFA000002B80D12F693846FFF7BCFB00287FF4C7
:10AFB0007AAF38460D221449FFF716FB07460028E2
:10AFC0003FF471AF183600940D2301223146FFF78C
:10AFD000CBFE384600F0FAF9012421463046FFF74F
:10AFE00035FD30B1611E3046FFF706FD2146FFF703
:10AFF00018FD01340D2CF0D155E700BF66C90108DA
:10B000007EC90108700000208C000020F0B58DB0D2
:10B01000CDE90023054628B94FF0FF304FF0FF314E
:10B020000DB0F0BD2422002103A80CF0F1F803A913
:10B0300068460BF0EDFF04460028EDD00CF0CAF98D
:10B040004A1C08BFB0F1FF3F06460F46E4D06269D4
:10B0500021462846FFF78FFD0028DDD120460CF061
:10B06000B9F94B1C08BFB0F1FF3FD5D08F4208BFE4
:10B07000864203D020460CF0ADF9D1E72368204684
:10B08000013323600CF0A6F9013108BFB0F1FF3F96
:10B09000C2D0626921462846FFF76DFD0028E9D03D
:10B0A000BAE770B53C258AB0DDE90E64019496FBE1
:10B0B000F5F405FB14640294182493FBF4F505FBE6
:10B0C0001433CDE903300C20013991FBF0F300FB80
:10B0D000131305930023CDE907339DF84030A2F206
:10B0E0006C7201A8069209930CF074F90AB070BD55
:10B0F000F7B504466846CDE900230BF077FF0269F7
:10B10000037A551C426990F804C0077B02F26C7107
:10B11000067EC2690068A3700033207018BF012347
:10B120002046013284F801C0E7702571A4F80510AB
:10B13000E6712272637203B0F0BD1FB5437A0293C9
:10B1400003780193437800938378B0F80520017960
:10B15000C078FFF7A6FF05B05DF804FB904271EBE5
:10B160000303B4BF0120002070470000032210B584
:10B17000104986B00B780133B3FBF2F202EB4202C6
:10B180009B1A0D4A0B7052F8234003780B4A049324
:10B1900043781A21039383780293C3780193037948
:10B1A0000093B0F8053020460CF0B6FE204606B0FD
:10B1B00010BD00BF5E48002068CB01082DCB010800
:10B1C000B1F1004F08BF00281FB502460B4608D05A
:10B1D00001A8FFF78DFF01A8FFF7C8FF05B05DF8D4
:10B1E00004FB0148FAE700BF5FCB01082DE9FF47E8
:10B1F00003220D462B4900280B78044603F1010376
:10B20000B3FBF2F202EB4202A3EB0203264A0B70FD
:10B2100052F8236075F100033EDA4FF0010A444210
:10B2200065EB4505214A0023204629460BF0E0FC4A
:10B230001E4A07460023204629460BF0D9FC10463B
:10B2400019464FF4616200230BF0D2FC4FF46162A7
:10B2500080460023204629460BF0CAFC10461946BA
:10B260003C2200230BF0C4FC3C22814600232046F4
:10B2700029460BF0BDFCCDF80080CDE901923B469C
:10B28000BAF1000F0BD00A4A1A2130460CF044FEE6
:10B29000304604B0BDE8F0874FF0000AC2E7054A27
:10B2A000F2E700BF5E48002068CB01088051010032
:10B2B0004BCB01084CCB01080FB404B07047000021
:10B2C0000FB437B51B4C256855B903222946012018
:10B2D000F7F7B6FF2B462A4629462060F7F7D4FF3A
:10B2E000154D2A68013A03321ED864212068F8F708
:10B2F000B7F98022002111480BF08AFF07AB069AAC
:10B3000080210E4801930DF0EDF97F2803DD0C49F3
:10B310000C480CF05FFE2B68084898470023206813
:10B320001A461946F7F7B0FF03B0BDE8304004B045
:10B33000704700BFE84800206048002068480020AF
:10B34000E6C60108E34800200FB410B50D4CA2B0CA
:10B350002268013A033210D825AB249A802102A832
:10B3600001930DF0BFF97F2804DD07490DF183003B
:10B370000CF030FE236802A8984722B0BDE81040C8
:10B3800004B0704764480020E6C6010870B5044662
:10B39000054E4518AC4200D170BD14F8011B304673
:10B3A000FFF78EFFF6E700BFD3A8010838B50C46BB
:10B3B0001546FFF785FF20462946FFF7E7FFBDE862
:10B3C00038400148FFF77CBF62AC010810B5044665
:10B3D00070B1F7F795FD2046F7F730FEF7F76AFCF6
:10B3E000BDE81040034A938801339380F7F782BC8D
:10B3F00010BD00BF3C4F002070B5214C8AB02268C0
:10B4000006460132632A22601E4D0BDDF6F790FFDF
:10B410000523002201A9F6F73DFFF6F745FC0023BE
:10B4200028602360F6F740FC2B6803F57A73984296
:10B4300004D9F6F739FC002328602360124A134C24
:10B4400013781BB92360636001231370F7F758FD6D
:10B450003046F7F767FD054668B1324600210BF02C
:10B46000D7FEF7F727FC238801332380F7F742FC48
:10B4700028460AB070BD638801336380F8E700BFD7
:10B48000F0480020F4480020EC4800203C4F002009
:10B49000A0F14103052B02D83738C0B27047A0F1A4
:10B4A0006103052B01D85738F7E73038C0B20A28B6
:10B4B00028BFFF207047002210B5441E21B114F8A8
:10B4C000010F08B1002A01DA104610BDFFF7E0FFB6
:10B4D00001390F28C9B202D840EA0212EEE74FF054
:10B4E000FF32F1E700687047D0F8010000BAC117D9
:10B4F000704700687047006800BA704783784278E8
:10B500001B04007843EA022318437047427800780E
:10B5100040EA022070470278407840EA02207047F3
:10B520000B12017043700B1409168370C170042054
:10B5300070470B1603700B1443700B128370C170AD
:10B54000042070470370130E4370130C8370130AAA
:10B55000C3700271052070470B1203704170022006
:10B56000704738B505460C460CF092FC611B013162
:10B5700090FBF1F303FB1100284438BD0649013864
:10B5800010F8013F03B97047CA5C02F00302012AB8
:10B5900008BF20330370F3E764EB0108F8B50446F5
:10B5A0000CF020FDE8B10F4A00271646204410F8A1
:10B5B000011C2346895C451E09070AD4C21A194694
:10B5C00013F8015B4DB92046BDE8F84001320BF09D
:10B5D00005BE00F8017C2846E9E7755D2D07EDD42E
:10B5E000F1E7F8BD64EB010808B50CF0E9FCB0FA2E
:10B5F00080F0400908BD000010B50446034B03600D
:10B600004068F8F70BFA204610BD00BFBCCB01081C
:10B6100010B50446FFF7F0FF20460821FEF786FF2D
:10B62000204610BD38B5436804460D461BB90E21AF
:10B630000548F8F763FA29466068F8F711F8431EE1
:10B640005842584138BD00BF74CB01084068F8F734
:10B6500095B908B5002340681A461946F7F714FE55
:10B66000431E5842584108BD38B50D4600210B4BCA
:10B6700004464160036003220120F7F7E1FD6060AA
:10B6800018B957210648F8F739FA2DB10023606838
:10B690001A461946F7F7F8FD204638BD78BD01086F
:10B6A00074CB0108014BDB68184700BFF848002045
:10B6B0000120704701B1096818B1806A431A5842E5
:10B6C0005841704710B5044618B9D2210748F8F719
:10B6D00015FA074B5B689847D4E90623904271EB53
:10B6E0000304B4BF101A002010BD00BFFDCF010835
:10B6F000F84800202DE9F0418846044610B103695E
:10B70000012B03D1E7211648F8F7F8F9D4E906230D
:10B7100052EA030122D0D4E90867901B63EB0701CA
:10B720000BF01CF80546206901380AF0FDFF0146C0
:10B7300028460BF005F9054640460AF0F5FF294674
:10B740000BF04AF829460AF03DFF0BF031FA3218A7
:10B7500047F1000310461946C4E90601BDE8F0812F
:10B76000FDCF010838B50C4B0546186800F0E5FB25
:10B7700010B90023184638BD4FF47A7403686C433F
:10B780001A68A242F6D000F0CFFB0028F1D003687F
:10B790001A689442F6E700BFF848002041F6583294
:10B7A000A0F55223A3F61833934224D8A0F55423CE
:10B7B000A3F1F902622A1ED96FF454729A18C62AAC
:10B7C00019D9A3F21353302B15D9104B984214D921
:10B7D00003F6B833984212D903F51673984210D97C
:10B7E00003F5167398420ED903F5E17398428CBFA6
:10B7F0000620052070470020704701207047022076
:10B800007047032070470420704700BFE8320D00E6
:10B81000F8B5054618B9F3212148F8F76FF9214F1B
:10B82000386800F08AFB002838D0002D36D0036835
:10B830001A79AA422ED11E7B00F076FB08BB6EB3AC
:10B84000062D03D940211648F8F758F9164B53F83E
:10B8500035400CBBFE211248F8F750F938687443A4
:10B8600000F06BFB0646C8B107683B79AB4204D1D8
:10B8700021463846FFF73EFF3C61304600F054FB5E
:10B88000F0E703681A79AA42D6D11B7B002BD3D0EC
:10B890000136D1E70026CFE7012CDFD1F8BD00BF8C
:10B8A000FDCF0108F8480020C4CB010800000000CB
:10B8B0002DE9F04F044687B058B3254B00681D6949
:10B8C0000AF032FF0AF018FB1FA3D3E900230AF0A5
:10B8D00095FC227B06460F462379D4F82890D4F8AD
:10B8E0001080D4F808A0BAB1062B98BF194A204698
:10B8F00094BF52F823B0DFF868B0FFF7E3FE32469A
:10B900003B46CDE90198CDE903A01348CDF800B03E
:10B91000A84707B0BDE8F08F062B98BF0D4A204618
:10B9200094BF52F823B0DFF838B0FFF7CBFECDE973
:10B930000189CDE903A0CDF800B032463B46074867
:10B94000E6E700BFAFF300800000000080842E41D6
:10B95000F8480020FCCB0108E4CE010839CF0108EB
:10B96000D6CE010810B5104C206820B923690F48C5
:10B97000BDE81040184700F0E9FA2369014660B1BC
:10B980000B489847206800F0D8FA044638B920469A
:10B9900000F0CAFA044610B910BD0648E8E720686E
:10B9A000FFF786FFF3E700BFF848002058CE0108F4
:10B9B00076CE0108B0CE0108F8B5134D06462B7EB1
:10B9C0000F4623B94FF4B1711048F8F797F82C6877
:10B9D00024B96B690E4898472046F8BD0D4B2046A8
:10B9E000002E08BF1E4600F0A8FA054608B900243C
:10B9F000F2E7046839462046B0470028ECD12846D3
:10BA000000F092FAF1E700BFF8480020FDCF0108EE
:10BA100019CE0108B1B600082DE9F04F3E4D91B0A6
:10BA20002B7E83468946924623B94FF4C9713B4821
:10BA3000F8F764F82C6834B96B69394898472046A0
:10BA400011B0BDE8F08F374B2046B9F1000F08BFA9
:10BA5000994600F072FA064620B96B693248984759
:10BA60003446ECE70468237BF3B94FF0FF3700243A
:10BA70004FF00008304600F057FA064608BBBAF10E
:10BA8000000F01D0CAF80070002FD8D1B8F1010F13
:10BA9000D5D908F1FF313846FFF763FD10AB03EB52
:10BAA000800050F8404CCAE7A3685B45DDDB00210D
:10BAB0002046C8470028D8D02046FFF703FE074697
:10BAC000D6E735682B7B002BD4D0AB685B45D1DB48
:10BAD00000212846C8470028CCD02846FFF7F2FDB1
:10BAE00048B9B8F10F0F9FBF10AB03EB880343F8C1
:10BAF000405C08F101086CB187420AD8BAD1D4E998
:10BB00000823D5E90801FFF729FB002818BF2C46B8
:10BB1000B0E707462C46ADE7F8480020FDCF010806
:10BB200019CE0108B1B600083DCE010800000000A2
:10BB30002DE9FF478946044620B940F2E111284823
:10BB4000F7F7DCFF236923B94FF4F1712448F7F7C5
:10BB5000D5FFDFF894A00027DAF804309847C4E94D
:10BB600008010546206988460AF0DEFD49460AF0CC
:10BB700033FE49460AF026FD0AF0BEF916A3D3E9C2
:10BB800000230AF03BFB09F003FF0AF0A7FC2D1885
:10BB900048EB0703C4E90653064620680AF0C4FDD3
:10BBA0000AF0AAF90CA3D3E900230AF027FB044604
:10BBB00048460D46CDE902670AF09EF92246CDE9D6
:10BBC00000012B46DAF810100648884704B0BDE89B
:10BBD000F047FFF7C7BE00BF0000000080842E4181
:10BBE000FDCF010818CC0108F848002008B5FFF780
:10BBF000D5FD003018BF012008BD000038B50D4D3F
:10BC000004462A7E22B94FF407710B48F7F776FFF6
:10BC100074B1237B63B1002320792373FFF7F8FD10
:10BC20002B69064898472046BDE83840FFF740BEDC
:10BC300038BD00BFF8480020FDCF0108E8CD01085D
:10BC400038B50D4D04462A7E22B94FF40A710B48CF
:10BC5000F7F754FF74B1237B63B901232079237371
:10BC6000FFF7D6FD2B69064898472046BDE83840C7
:10BC7000FFF71EBE38BD00BFF8480020FDCF010809
:10BC800001CE0108F8B5194D06462B7E23B94FF4B5
:10BC90000D711748F7F732FF2C6824B96B69154806
:10BCA0009847204601E00EB90020F8BD204600F07C
:10BCB00044F904460028F7D023689E420CD1377916
:10BCC0003046FFF7EFFC2146286800F04DF9384672
:10BCD000FFF79EFD0120E8E7204600F025F9044625
:10BCE0000028E9D16B690448DAE700BFF848002072
:10BCF000FDCF0108B5CF0108D7CF01082DE9F843E2
:10BD0000384D06462B7E8846914623B940F2F911FC
:10BD10003548F7F7F3FE3046FFF768FF044630B9C1
:10BD20006B693146314898472046BDE8F883304674
:10BD3000FFF718FD044630B12D482B69314698476E
:10BD40002046FFF79FFF2B7E1BB976212648F7F789
:10BD5000D5FEAB6830209847044640B96B6925484A
:10BD600098476B693146244898470024DCE7302225
:10BD700000210BF04DFA3046FFF710FD0746207109
:10BD800038B9EB68204698476B6931461B4898479D
:10BD9000E7E7062803D940211348F7F7AFFE184B11
:10BDA000214603EBC70253F83730526823614FF442
:10BDB0007A73A2605E4300220023C4E906230123B4
:10BDC00026602373C4E90A89286800F097F820796F
:10BDD000FFF71EFD2B690B4898472046FFF768FDCB
:10BDE000A2E700BFF8480020FDCF0108D0CC010831
:10BDF00007CD01083CCD0108ADCD01086ACD010891
:10BE0000C4CB010895CD010870B50F4C0546237EC3
:10BE100023B94FF41C710D48F7F770FE23685BB12E
:10BE20000B4E29463046FFF7C7FD50B92369294616
:10BE3000BDE870400748184763690748BDE870408F
:10BE40001847FFF72FFCECE7F8480020FDCF01086A
:10BE5000B5B600088FCF0108B5CF0108014B187E99
:10BE6000704700BFF848002084B070B504AC84E887
:10BE70000F00154B1A7E1C462AB1BDE870405B6965
:10BE8000124804B018471D1D04AE0FCE0FC533680D
:10BE90002B600BB90E4B636123690BB90C4B23610B
:10BEA000E3680BB1A36833B923690A4898470A4B82
:10BEB000E3600A4BA36000F013F8012320602376AF
:10BEC000BDE8704004B07047F84800205CCC010821
:10BED000B9B2000895CC01087971010869710108AF
:10BEE00010B50820FFF788FA0446F5F7D5FE0023C1
:10BEF000C4E90034F5F776FF204610BD70B505465D
:10BF00000C200E46FFF778FA044660B10660F5F79C
:10BF1000C3FE002363606B68A3601C6004346C6024
:10BF2000F5F760FF012070BD10B50446F5F7B4FECB
:10BF30006468F5F757FF204610BD10B50446F5F7C5
:10BF4000ABFE2468F5F74EFF204610BD10B5044641
:10BF5000F5F7A2FE236800241BB9F5F743FF20463E
:10BF600010BD01345B68F7E738B50C460546F5F7B8
:10BF700093FED4E901324BB19A60A2681360F5F7E1
:10BF800031FF2046BDE83840FFF720BA6A60F4E789
:10BF900070B50446044E451814F8011B3046FFF7EF
:10BFA0008FF9AC42F8D170BDD3A8010870B5154621
:10BFB0000022C0E901150270C0E90332C0E9052280
:10BFC000C0E907224262DDE90412044600F11C06C2
:10BFD000F8F7F0F938B929460748FFF771F92B212E
:10BFE0000648F7F78BFDDDE9042331462046F8F7D4
:10BFF000CEF9204670BD00BFD49D0108FF9D010809
:10C00000F0B50126044608270D468DB0694B6A4AF3
:10C010003146009602A8F4F703F902A92046F9F781
:10C02000C9FA02A8F4F79EF8644BCDE900571A4606
:10C0300004210DEB0700FFF7B9FF0DEB07012046C8
:10C04000F9F7B8FA0DEB0700F4F78CF8EB195C4A36
:10C050000197009304215B4B0DEB0700FFF7A6FF50
:10C060000DEB07012046F9F7A5FA0DEB07001027A5
:10C07000F4F778F8EB190093534B04211A46019713
:10C0800002A8FFF793FF02A92046F9F793FA20359B
:10C0900002A8F4F767F84D4B4D4A0095042101972B
:10C0A00002A8FFF783FF02A92046F9F783FA02A846
:10C0B000F4F758F80C23474A00930221464B02A894
:10C0C000F4F786F802A92046F9F774FA02A8F4F703
:10C0D00049F8424B424A3146009602A8F4F7A0F8CC
:10C0E00002A92046F9F766FA02A8F4F73BF8032202
:10C0F000002303923B4D3C4A3C4902A88DF808308E
:10C100000495CDE90523CDE90733CDE909330B9338
:10C11000F8F738F938B929463548FFF7D1F8202122
:10C120003448F7F7EBFC0025304A09A902A8F8F7D4
:10C13000F3F802A92046F9F73DFA02A8F4F712F83D
:10C140002D4B2E4A0095022102A8F4F741F802A9CE
:10C150002046F9F72FFA02A8F4F704F8284B294AE9
:10C160000095022102A8F4F733F802A92046F9F756
:10C1700021FA02A8F3F7F6FF0121234B234A00918D
:10C1800002A8F4F74DF802A92046F9F713FA02A81D
:10C19000F3F7E8FF1E4B1F4A0095022102A8F4F7AF
:10C1A00017F802A92046F9F705FA02A8F3F7DAFF13
:10C1B0000DB0F0BDD3D0010874B80108E6D0010875
:10C1C00057D401083ED40108F4D001085FD4010817
:10C1D00089D40108BBB70108FBD0010854D101087C
:10C1E000F7B70108D4B7010890D4010877B801085F
:10C1F000D49D0108FF9D0108A5D40108FBB70108E3
:10C20000E3D4010822B801081ED5010875AB010866
:10C210003AD501084AB8010830B504468DB0014648
:10C220007A4A6846F8F7A9FF794A214603A8F8F741
:10C23000A4FF784A214606A8F8F79FFF76492046D2
:10C24000F8F792FF05467548FFF73AF80123039A7D
:10C2500002F11001914205D011F8010D002818BF1C
:10C260000023F7E7002B53D06D48FFF729F85DB3A3
:10C270006C48FFF725F86C4A214609A8F8F77DFFBE
:10C280006A48FFF71DF808210098FFF781FE68480B
:10C29000FFF716F808210998FFF77AFE6548FFF7BF
:10C2A0000FF810210698FFF773FE6348FFF708F8B0
:10C2B0000998069A009900F055FE09A8F8F736FA91
:10C2C0005E48FEF7FDFF61E05D48FEF7F9FF5D485F
:10C2D000FEF7F6FF0699009800F0A2FD5A48FEF717
:10C2E000EFFF042100980844FFF752FE5748FEF77D
:10C2F000E7FF10215648FFF74BFE5648FEF7E0FFD8
:10C3000010215548FFF744FE4B48FEF7D9FFD7E709
:10C31000102206980AF046FF5049514B002818BFDA
:10C3200019465048FEF7CCFF002D3DD03D48FEF7A2
:10C33000C7FF3D4A214609A8F8F71FFF4A48FEF704
:10C34000BFFF08210098FFF723FE4848FEF7B8FF1B
:10C3500008210998FFF71CFE4548FEF7B1FF1021A0
:10C360000398FFF715FE4348FEF7AAFF1021069831
:10C37000FFF70EFE3048FEF7A3FF0998039B069ACD
:10C38000009900F003FE09A8F8F7D0F92A48FEF753
:10C3900097FF06A8F8F7CAF903A8F8F7C7F968469F
:10C3A000F8F7C4F90DB030BD2548FEF789FF3248D3
:10C3B000FEF786FF039A0699009800F075FD224863
:10C3C000FEF77EFF042100980844FFF7E1FD2B48AB
:10C3D000FEF776FF10211E48FFF7DAFD2848FEF72A
:10C3E0006FFF10212748FFF7D3FD2748FEF768FFAE
:10C3F00010212648FFF7CCFD2548FEF761FF1648BF
:10C400001021FFF7C5FD0C485BE700BFE6D001082F
:10C4100089D40108F4D0010874B8010886D1010854
:10C420009DD10108B8D1010857D40108BED1010837
:10C43000CFD10108E1D1010862AC010889D201081D
:10C4400001D2010806D2010838D201084AD20108F7
:10C450006801002076D20108980100206FD1010800
:10C4600063AC0108A8D20108C5D20108D7D20108DF
:10C47000EAD201080AD3010853D301088DD3010879
:10C48000F9D301087801002010D4010888010020A8
:10C4900027D4010810B5084CD4F82C211AB964210E
:10C4A0000648F7F72BFBD4F82C010023BDE8104019
:10C4B00003222021F6F794B8C000002066D60108B8
:10C4C000F0B51F461446C7B005460E46F1220021BE
:10C4D00009A80AF09DFE09AA1021384602F048F882
:10C4E00020460BF07FFD07461022002101A80AF02C
:10C4F0008FFE102F3A46214628BF102201A80AF0CD
:10C500005FFE09AA05A901A802F0ACF8324605A908
:10C5100028460AF055FE47B0F0BD000038B50C4C77
:10C520000C4D94F83230022B0ED1062394F8FF20E4
:10C53000D4F80011012001F0D1FF6B6B0020984767
:10C54000042384F8303038BDEB6A98470123F8E7BC
:10C55000C0000020A4E6010810B5044600F0E4FF86
:10C5600020B92046BDE8104000F0B6BF10BD000065
:10C57000054B93F8212022B993F8350080F0010093
:10C5800070470020704700BFC0000020F0B5702742
:10C590009DB006460D463A46002168460AF038FE30
:10C5A00008212B460DEB010004AC0B4AFFF788FF76
:10C5B0002B462046094A102108ADFFF781FF94E879
:10C5C0000F0085E80F003A46694630460AF0F8FD4C
:10C5D00030461DB0F0BD00BF57D601085FD6010838
:10C5E00084B070B58AB00EAC84E80F00754C4FF47F
:10C5F0009C722546002120460EAE0AF009FE0FCEA1
:10C600000FC596E8030014AE85E803000FCE04F1D1
:10C6100018050FC533682B600E9B0BB96A4B23605E
:10C620000F9B0BB9684B2360109B23B94FF4A97182
:10C630006648F7F763FA129B23B94FF4AB7163486E
:10C64000F7F75CFA119B23B94FF4AD715F48F7F728
:10C6500055FA139B23B94FF4AF715C48F7F74EFAC4
:10C66000A3690BB90323A361E3690BB90A23E3614F
:10C6700094F8233013B9012384F8233001F0D0FC5F
:10C6800094F8243013B9012384F8243001F0C0FC5D
:10C69000A36A0BB94E4BA36201F0AEFC05F0EEFFAE
:10C6A000C4F828010138033004D963684948984721
:10C6B00000207EE0032200210120F6F7C1FDC4F82E
:10C6C000300120B940F287114048F7F717FA0022ED
:10C6D0000421E069F6F7B4FD606420B940F28B11E3
:10C6E0003A48F7F70BFA00220421E069F6F7A8FDB3
:10C6F000A06420B94FF4C7713448F7F7FFF900225E
:10C7000004210120F6F79CFDE06420B940F291116C
:10C710002E48F7F7F3F9082384F80931042384F845
:10C720000A31002384F83630012384F80D31FFF7F5
:10C7300095FB05AD68B9A368226905932368079244
:10C740000893E26863680692009395E80F00FFF78C
:10C750008BFB01F08BFC23681F4E079363680496E4
:10C76000089323690693E368059306F1A0030393F6
:10C7700003AB93E803008DE80300DC3695E80F0077
:10C7800002F0FCF80196A3694FF4CD7200931349AF
:10C7900001231348F5F766F8012805460ED100235A
:10C7A00003220421D4F82C01F5F71AFF284684F857
:10C7B00034500AB0BDE8704004B07047636809485F
:10C7C00075E700BFC0000020B9B2000866D60108B6
:10C7D00008E6D33389D5010810010020BCD5010833
:10C7E0004DC90008C4D5010810B5124CD4F82C313D
:10C7F00023B94FF4DF711048F7F780F904210023C3
:10C800000322D4F82C01F5F7EBFE42F21071D4F8B4
:10C810003001F6F725FF20B940F2C7110648F7F7B7
:10C820006DF90023D4F830011A46BDE810401946CE
:10C83000F6F72ABDC000002066D6010838B50E4DB7
:10C84000D5F8303123B940F2CF110C48F7F756F93B
:10C850000021D5F83001F6F703FF0128044608D17E
:10C860000023D5F830011A461946F6F70DFD20468B
:10C8700038BD0020FCE700BFC000002066D60108DC
:10C8800010B5FFF7DBFF68B1074C0023D4F82C018B
:10C8900003220821F5F7A4FED4F82C01BDE81040CE
:10C8A000F5F778B910BD00BFC0000020014BD86378
:10C8B000704700BFC0000020002307B50193054B5F
:10C8C000024601A9D86CF6F739FE019803B05DF86D
:10C8D00004FB00BFC000002038B5FFF7AFFF184DC4
:10C8E000044620B16B6817489847002038BD686C33
:10C8F000F7F744F8EB698342F7D32146204602F06C
:10C900006DF805460028F0D0047000F0D3FD044611
:10C9100018B9284602F09AF8E7E70B4A1368013382
:10C9200013605BB9136801331360636040F2031353
:10C9300020462380FFF710FE6068D7E71368F4E70E
:10C94000C0000020F4D501081449002001232DE97E
:10C95000F0415F4CDFF880815E4E84F830300A236E
:10C960005D4A4FF0FF310020F5F7F6FD012867D151
:10C97000D8F8000043071AD5337833B105F0CCFD61
:10C98000002005F01DFE00233370F6F793F9F6F74B
:10C99000B1F9022384F830300023D4F830011A466C
:10C9A0001946F6F771FC0020F5F748FBD7E710F0C1
:10C9B000080521D033787BB941F2883005F0D8FDE5
:10C9C00018B9A0214548F7F799F8454805F0F8FD52
:10C9D00001233370FFF7A2FD0020F5F7EFFE4FF4BF
:10C9E000FA61D4F83001F6F73BFE0028B7D1A72151
:10C9F0003A48F7F783F8B2E710F020003FD03378D9
:10CA0000DBB194F83030042B17D1364F2A46394623
:10CA1000D4F82801F6F7D4FE01280ED13B78072B75
:10CA200021D1284600F046FD38B140F20512C0E998
:10CA3000015505610280FFF78FFD0020F5F7BEFE6E
:10CA40003378002B8BD000F087FD0546002886D078
:10CA5000032384F830300378052B35D8DFE803F062
:10CA60001219192A2A312A463946D4F82801F6F72C
:10CA700065FD0128E1D1384605F0A8FDDDE7F5F7B1
:10CA80009DFE6CE7D6211548F7F738F8FFF746FD0D
:10CA900065E7FFF76DFD38B9284600F097FA60B1F9
:10CAA000284600F019FDF1E72846FFF755FDFFF78E
:10CAB00013FFEBE701F0E2F8F1E72846FFF74CFD42
:10CAC000E4E700F0C7FCEBE7636807489847E7E74F
:10CAD000C0000020184900202449002066D6010823
:10CAE00095C400081C49002069D50108024B93F841
:10CAF000FC0001F069BC00BFC0000020F0B585B0AB
:10CB000007460D461446ADF80430FFF797FE3D4E3C
:10CB100028B173683C489847002005B0F0BD706CA0
:10CB2000F6F72CFFF3698342F6D3FFF7DFFF854268
:10CB3000F2D8002C45D1002DEED12946384601F01F
:10CB40004DFF05460028E7D09DF80530002B14BFA7
:10CB50000423022303709DF8043033B10D23012216
:10CB600003A98DF80C3000F031FE96F8312096F8CC
:10CB70003230934203D196F83330934217D02023BA
:10CB8000022A18BF00228DF80C3095F8783003A9DE
:10CB90000BBF43F0040343F001038DF80D208DF823
:10CBA0000D20284685F87830022200F00FFE6C77C1
:10CBB000284600F07FFC044630B9284601F046FFC5
:10CBC000AAE7DF2CA8D8B8E70023104A83601368CF
:10CBD0000133136093B913680133136063600A9BD8
:10CBE0002046236140F20113238000F087FC38B90E
:10CBF000204600F071FC736805488CE71368EDE788
:10CC000060688AE7C0000020F4D5010814490020BC
:10CC10002FD60108082808BF0120034B83F8230002
:10CC200083F8FC00704700BFC0000020024B83F86F
:10CC3000240083F8FD007047C000002008B5FEF70F
:10CC40005AFC014B586508BDC0000020034630B5B2
:10CC5000054C00F11005224618685968083303C2D4
:10CC6000AB421446F7D130BD88010020034630B5F1
:10CC7000054C00F11005224618685968083303C2B4
:10CC8000AB421446F7D130BD78010020034630B5E1
:10CC9000054C00F11005224618685968083303C294
:10CCA000AB421446F7D130BD68010020034630B5D1
:10CCB000054C00F11005224618685968083303C274
:10CCC000AB421446F7D130BD9801002010B50446A0
:10CCD000FFF7BCFF2046FFF7C9FF2046BDE8104024
:10CCE000FFF7D4BF30B51025C3B0224CF12200218C
:10CCF00005A80AF08DFA2A46002101A80AF088FA50
:10CD000094F8673005AA8DF8053094F86630294606
:10CD10008DF8063094F8653004F178008DF807300E
:10CD200094F864308DF8083094F863308DF8093049
:10CD300094F862308DF80A3094F861308DF80B3039
:10CD400094F860308DF80C3001F012FC052305AA30
:10CD500004F1980101A88DF8043001F083FC06234A
:10CD600005AA04F1880101A88DF8043001F07AFCCD
:10CD700043B030BDC00000200246024B006851683D
:10CD800003C37047180100200246024B0068516837
:10CD900003C3704720010020034630B5054C00F165
:10CDA0001005224618685968083303C2AB4214467E
:10CDB000F7D130BD28010020034630B5054C00F105
:10CDC0001005224618685968083303C2AB4214465E
:10CDD000F7D130BD38010020014B83F822007047A5
:10CDE000C0000020014B83F831007047C0000020D4
:10CDF000014B1864704700BFC000002013B5002429
:10CE0000054B01AA054993F8FD000194FEF704FEC5
:10CE10002146019802B010BDC0000020BDCF00081F
:10CE200010B50430C6B00C46FFF708FF1C4B0DF1DF
:10CE3000050203F10C0153F8040B8B4242F8040B7A
:10CE4000F9D11B881021138000238DF813300223A1
:10CE500009AA20468DF8043001F08AFB09AA05A929
:10CE600001A801F0FFFB05A8FFF720FF012309AA95
:10CE7000102120468DF8043001F07AFB09AA05A99B
:10CE800001A801F0EFFB05A8FFF720FF4FF488721F
:10CE9000044B1A84102283F8502046B010BD00BF06
:10CEA00020D60108C000002030B50430C7B00C46C1
:10CEB0001546FFF7C3FE294B0DF1050203F10C01E6
:10CEC00053F8040B8B4242F8040BF9D11B8820461F
:10CED000138000238DF813300223012409AA1021A6
:10CEE0008DF8043001F044FB09AA05A901A801F05E
:10CEF000B9FB05A8FFF7DAFE09AA102128468DF82C
:10CF0000044001F035FB09AA05A901A801F0AAFB1C
:10CF100005A8FFF79BFE032309AA05A901A88DF820
:10CF2000043001F09FFB05A8FFF7A0FE042309AA27
:10CF30000DEB030005A98DF8043001F093FB05A863
:10CF4000FFF7A4FE40F21112054B1A84112283F858
:10CF5000074183F8502047B030BD00BF20D60108FC
:10CF6000C000002038B50D461446FFF705FF2846DF
:10CF7000FFF70AFF2046FFF70FFF2046FFF71CFFD1
:10CF80001022014B1A8438BDC000002070B50E4637
:10CF900015461C46FFF7F0FE3046FFF7F5FE284623
:10CFA000FFF7FAFE2046FFF707FF1122024B1A8413
:10CFB000BDE87040FFF796BEC000002028B1836A2C
:10CFC000012B01D1007B7047002070472DE9F0470D
:10CFD000044686B010B10378012B03D01C21794898
:10CFE000F6F78CFD63691BB91D217648F6F786FDBF
:10CFF00063691B78042B05D0022B03D01E217148D6
:10D00000F6F77CFD0026704D03AA704995F8FD00E7
:10D01000D5E93F9A0396FEF7FFFC074640B9204644
:10D0200000F0FCFA4FF00108404606B0BDE8F0877A
:10D03000039B93B1FEF796FC0399042905D920467A
:10D0400000F024FB4FF00008EEE74FF47A736048DD
:10D050004843B0FBF3F0F4F779FFA3680133012BE9
:10D06000A3600FD1D5F8F03060690133C5F8F03016
:10D0700095F80831013385F8083100F063FB6069E9
:10D0800000F0C4FB6B6D66697360D5F8F030738196
:10D0900095F80431002B63D0002385F80431337AEE
:10D0A00043F00403337295F8FC30384686F87C3040
:10D0B00001F01EF886F87D000121606900F058FB40
:10D0C00095F80D214FF47A7312F00F0208BF012278
:10D0D00000265A4305AB019304AB0093394602F591
:10D0E0007A736069049600F025F98046002896D08E
:10D0F000F4F7DAFDE060049860B1314600F038FBE7
:10D10000049B1B78052B04BF012385F80431002301
:10D1100085F80631049800F0F1FADDE9040100F029
:10D120005DFD049F77B13F7A17F0040703D04746AF
:10D1300095F80B31A36063691B78022B02D195F837
:10D140000B31A36000F01EFA0646F0B98A211D4893
:10D15000F6F7D4FC1F4B204A8B211A4809F002FF36
:10D16000A6F87A309FE73146606898476420F4F764
:10D17000EDFE304600F016FA95F80B31A2689A429F
:10D18000BFF452AF032333705CE78022616918302B
:10D190000AF016F80023049AC6F88030C6F89820E2
:10D1A00022787372337095F83530C6E9039A337577
:10D1B000236972703772002BD5D1304600F00CFA1B
:10D1C000DAE700BFB4D60108C0000020BDCF0008D8
:10D1D00040420F00F1D60108A6D60108F0B587B08D
:10D1E00007460C468DF80F202BB101220DF10F01DF
:10D1F000002005F08DFE0025194B9DF80F102046EC
:10D200009B6A984705AB009304AA2B4629469DF8D4
:10D210000F00CDE90455134E05F06EFA124B40F69F
:10D22000B8323146D3F82801F6F788F9B0B1F4F7EF
:10D230003BFD33780446012B30460BD105F0C6F98F
:10D24000049809F071FA01463846FEF771FC204651
:10D2500007B0F0BD05F0BAF92C46F8E70446F6E74A
:10D26000A4E6010828490020C00000202DE9F84F5D
:10D270002C4F1E467B6B0546894614464FF47A7840
:10D280009847BB46DFF8A8A0274F08FB05F202F538
:10D29000C332A032B2FBF8F22349DAF82801F6F7DC
:10D2A0004DF928B9DBF8303098474FF0FF3022E0D5
:10D2B0003B78072B07D105F0ADFD384605F086F920
:10D2C0004FF47A65E1E7032BDBF8305015D17F6826
:10D2D00038793968844228BF04464846224609F016
:10D2E0006FFF1EB1FB8833803B7AB3700E4805F0A8
:10D2F0006DF9A8472046BDE8F88F042B05D10A48F0
:10D3000005F064F9A8470020F5E7052B04D106488D
:10D3100005F05CF9A847C8E7C6210448F6F7EEFB1C
:10D32000F5E700BFA4E601083049002002D7010854
:10D33000C00000202DE9F04FC3B00F46DDE94C8559
:10D34000914602A9FF2282461E4601F099FB8346C0
:10D3500018B9002043B0BDE8F08F3D4C396894F80F
:10D36000FD3094F8FC20002001F0B8F800235A4664
:10D3700002A93846FFF732FF01900028E9D09AF859
:10D38000783013F0050F0AD013F0040F0CBF002300
:10D39000022394F832209A4218BF84F83230FF22D8
:10D3A000002102A809F034FF39684FF47A7794F825
:10D3B000FC2094F8FE30012093429ABFD21AD2B2D8
:10D3C0000022062301F08AF807FB09F1A1F5434189
:10D3D0005039B1FBF7F101A8A6EB0906F4F776FD89
:10D3E000FF222B4602A9A6F16400FFF73FFF421C73
:10D3F000AFD000280FDD0DB10123EB700023984260
:10D40000C8F8003005DDC1B202A801F097FEC8F8E7
:10D41000000001209EE77E43062394F8FF20D4F805
:10D420000011012001F05AF8B6FBF7F101A8F4F75A
:10D430004DFD2B46FF2202A940F6B830FFF716FF3C
:10D44000431C86D00028D9DD002DD7D00223D4E795
:10D45000C000002070B5C2B001ABFF2202A94FF49A
:10D460007A60FFF703FF061E1EDD114DF1B26A6DF3
:10D4700002A801F043FC0446B0B10378052B01D0AB
:10D48000032B0DD10021204600F072F9204600F058
:10D4900035F92046019900F0A1FB2B6C204613B909
:10D4A00001F0D4FA00E09847304642B070BD00BFAA
:10D4B000C000002038B5074B0546DB6818209847A8
:10D4C000044620B11422002109F0A2FE6561204625
:10D4D00038BD00BFC000002010B5044650B14069FF
:10D4E00001F0B4FA00236361034B2046BDE810400D
:10D4F0001B69184710BD00BFC0000020037807B5A6
:10D50000052B4FF00003019006481A4601A90CBFF5
:10D51000806C406CF5F7B8FE431E5842584103B08A
:10D520005DF804FBC000002007B5037801900948AE
:10D53000052B4FF000024FF0010301A90CBF806CD6
:10D54000406CF5F7A1FE431E5842584103B05DF808
:10D5500004FB00BFC0000020002213B5084C01A945
:10D56000A06C0192F5F7EAFF019B33B994F83620DD
:10D570001AB901A9606CF5F7E1FF019802B010BD7E
:10D58000C0000020064B10B5DB68A0209847044679
:10D5900018B1A022002109F03BFE204610BD00BFBB
:10D5A000C000002070B5044690B1D0F88000094D4D
:10D5B00008B12B699847D4F8980020B101F046FAD9
:10D5C0000023C4F898302B692046BDE87040184706
:10D5D00070BD00BFC00000201FB50E4C0190E06C74
:10D5E000F6F7DEF9024638B903A9E06CF5F7A6FFB5
:10D5F00010B10398FFF7D6FF002301A91A46E06C8B
:10D60000F5F742FE20B940F25B110348F6F776FACF
:10D6100004B010BDC000002002D70108F8B50423F3
:10D62000437003780546032B0ABF144B0469DC6B77
:10D63000FFF7A8FF0646B0B94FF4B5711048F6F7EA
:10D640005DFA104B104A40F26B110D4809F08AFC4C
:10D6500031466868A0473046FFF7A4FFFA20F4F788
:10D6600075FC3846F8BD01272B7807704370002CF5
:10D67000EED1FFF7B1FF2046F4E700BFC000002065
:10D6800002D70108FAD601083DD70108F8B503789A
:10D690000646032B08BF154B0F460CBFDC6B046915
:10D6A000FFF770FF0546B0B940F283111048F6F756
:10D6B00025FA104B104A4FF4C2710D4809F052FC84
:10D6C00029467068A0472846FFF76CFFFA20F4F758
:10D6D0003DFC0120F8BD022303703378476043709E
:10D6E000002CEDD1FFF778FF2046F3E7C0000020C3
:10D6F00002D70108FAD6010859D7010808B5104A1F
:10D7000010B1002382F8083192F82230BBB192F8B0
:10D71000083192F809118B4211D95B1A92F80A115B
:10D7200093FBF1F201FB12334BB900F081FC30B9ED
:10D7300000F08CFC18B9BDE8084000F097BC08BDAB
:10D74000C0000020094B93F822206AB1027A42F00F
:10D750000102027293F8082193F809319A4282BFBC
:10D76000037A43F002030372704700BFC000002039
:10D7700070470000064A1378FD2BDFBF007805498B
:10D78000C8540133DABF012013700020704700BF76
:10D79000394A00203A49002038B10078032803D0E4
:10D7A000431F58425841704701207047052307B571
:10D7B0000DF107008DF80730FFF7DCFF0248FFF797
:10D7C000D9FF03B05DF804FB38490020037A70B537
:10D7D0001B09D61804460F2E00F10C0015461844FC
:10D7E00009DC09F0EDFC0120237A05EB131565F344
:10D7F0000713237270BDC3F10F0209F0E1FC237A15
:10D80000002043F0F0032372F4E7000037B5114C19
:10D810000546227822B11049FFF7D8FF0023237074
:10D820000E4C94F806213AB10823012201A928469A
:10D830008DF80430FFF7CAFF94F8073143B140F286
:10D840000113022201A92846ADF80430FFF7BEFFFC
:10D8500003B030BD394A00203A490020C000002002
:10D860000122044B00F00F0083F80D0183F806211C
:10D87000704700BFC00000202DE9F04F814693465D
:10D880009A4600258BB09DF85080B44E02914545D4
:10D8900002D30BB0BDE8F08F1AF805300AEB05078C
:10D8A000013B1F2B00F29881DFE813F02000960166
:10D8B0002B003B01C600AE00FF0036013B011D01FD
:10D8C00096013D018B005501640196019601960178
:10D8D0009601960196019601960196019601960190
:10D8E000960196019601960196018301A8EB050326
:10D8F000DBB2012B4FF000041BD086F80741022455
:10D9000017E00024A8EB0503DBB201938DF81C405F
:10D91000019A231D934202DA3B5D032B0BD044B1E5
:10D92000032308A88DF82030FFF724FF07A8FFF78E
:10D9300021FF2C447AE039194B78A01C1A0938448D
:10D9400003F00F03059104920393FDF7DFFD0599A2
:10D95000049A09790534062AC1F3021CE4B201F0E5
:10D960000F01039B21D90F2A05D19DF81C2042F0FD
:10D9700002028DF81C205A1E042A19D90F2B05D13A
:10D980009DF81C3043F004038DF81C3009B186F873
:10D990000B11BCF1000F0ED100F034FC9DF81C30CF
:10D9A00043F001038DF81C30B2E786F8FC20DCE779
:10D9B00086F8FD30E4E7BCF1060FA9D14FF6FF7001
:10D9C000EAE7A8EB0503DBB2052B40F20381781CE4
:10D9D000FDF78FFD002197F90530002BACBF604BA0
:10D9E000604BC31841F10002002196F80D01C318E5
:10D9F00041EB0202BBF1020F02D1013342F10002FE
:10DA0000C9E91C32062494E7062307A88DF81C30C8
:10DA1000FFF7B0FE029B544803F01F038DF820303F
:10DA2000FFF7A8FE08A8FFF7A5FE6C1CE4B2A5420C
:10DA30003FF42FAF25462AE7A8EB0503DBB2042B02
:10DA400040F2C880D7F80120484C0892D2B2C2F305
:10DA5000021386F8FE302378C2F30302052A43F04E
:10DA6000040394BF43F002036FF341030DF121005F
:10DA700098BF86F8FF2023706427FDF73FFD4743DA
:10DA8000384605F0C9F960B12378C6F8007143F053
:10DA9000010301222370364B1A70FFF787FE05241D
:10DAA00047E7237860F30003F3E7A8EB0503DBB255
:10DAB000052B40F28F80642157F8010F3A79030A51
:10DAC00059430890C0B28DF8242000F033FB07239F
:10DAD0008DF8180007A88DF81C30FFF74BFE06A83C
:10DAE000FFF748FE8EE7A8EB0503DBB2042B71D9E4
:10DAF0006421D7F80100030A5943C0B200F04CFB7F
:10DB00000A238DF81C0008A88DF82030FFF732FE9C
:10DB100007A8FFF72FFEC2E7787800F00F00FFF7A5
:10DB20009FFEAC1C82E7A8EB0503DBB2012B51D0B2
:10DB300001237A7808A8110902F00F0203FA01F113
:10DB4000934086F80A310C2386F809118DF82030AD
:10DB5000FFF710FED3E6EC1C68E700BFC000002012
:10DB60006E3DD5126F3DD512CC0100203849002002
:10DB700039490020A8EB0503DBB2012B2AD0B3689A
:10DB80007C789847012223090A3302FA03F3C6F886
:10DB900018310F23C6E9440104F00F0408A8C6F8A1
:10DBA0001C418DF81C208DF82030FFF7E3FD07A8FD
:10DBB000CEE7A8EB0503DBB2012B0BD07B780BB1D2
:10DBC000022B07D196F833209A423FF498AE86F89C
:10DBD000333094E60024ACE62C4628E730B585B017
:10DBE00003910446174B30B91B7803B305B0BDE869
:10DBF0003040FFF7DBBD00259DF90E109DF80F208A
:10DC00001D70FFF7C9FD90B10F48237A90F822509C
:10DC10002DB113F0010518BF012580F805511B092E
:10DC200007D0009304F10C032046FFF725FE05B052
:10DC300030BD637F002BFAD1237F002BF7D00093F8
:10DC4000A36EF1E739490020C000002010B504465A
:10DC500078B1836A012B0CD1C36A1BB91021064825
:10DC6000F5F74CFFE36A587802288CBF00200120AA
:10DC700010BD0020FCE700BF81D701082DE9F04767
:10DC8000054686B018B10378033B012B03D9222146
:10DC9000BC48F5F733FF6B690BB11B781BB123212F
:10DCA000B848F5F72BFF4FF00009B74C94F8FD602A
:10DCB000D4E93F8700F0ACF900F0B2F9304603AA8E
:10DCC000B249CDF80C90FDF7A7FE064620B92846CC
:10DCD000FFF7A4FC01260AE0039BA3B1FDF742FE77
:10DCE0000399042907D92846FFF7D0FC4E46304651
:10DCF00006B0BDE8F0874FF47A73A5484843B0FBFF
:10DD0000F3F0F4F723F9AB6894F820200133102ADC
:10DD1000AB602FD1012B09D1D4F8F0300133C4F816
:10DD2000F0309C4B5B699847A4F8E800B4F8E83001
:10DD30000133A4F8E8304FF0000905AB019304ABC0
:10DD40000093314641F2707341F28832686994F869
:10DD5000FFA0CDF8109084F8FF90FFF7EBFA06468D
:10DD6000A8B92846FFF75AFC049800F06FFE84F823
:10DD7000FFA0AFE7112A05D1636987489847A4F847
:10DD8000E800D8E750217F48F5F7B8FED3E7049BB9
:10DD900084F8FFA013B11A78012A06D02846FFF7AD
:10DDA0003DFC049800F052FEA1E794F82020102AD0
:10DDB00040F09780102384F850300023049AD168F3
:10DDC00002F1530C616502F1630E002B00F09980A3
:10DDD000112384F850306346DFF8C0A1D14618689B
:10DDE00059680833A9E803007345CA46F6D1DFF83D
:10DDF000B09102F1230302F1330ACE461868596844
:10DE00000833AEE803005345F146F6D1DFF89491AC
:10DE100002F1430ACE46186859680833AEE8030099
:10DE20005345F146F6D1DFF88091CE46186859681F
:10DE30000833AEE803006345F146F6D19368A36367
:10DE4000137CC3F3030384F8FF30137CC3F3021382
:10DE500084F8FE30507CFFF703FD049894F83120DD
:10DE6000437C1230012B4FF0000398BF84F8063139
:10DE700012F0FD0F18BF84F83130C4E93D33C4F807
:10DE8000F030638600F0DEF9FDF76CFD012384F8C5
:10DE90003530FFF777FB802281466969183009F039
:10DEA0008FF90023049AC9F88030C9F8982094F8B3
:10DEB000352089F8093089F800302B7889F814204A
:10DEC00089F80130E36BC9E90387002B56D0494636
:10DED000686898476420F4F739F84846FFF762FB12
:10DEE00005E7112A07D193F82230002B3FF462AFE7
:10DEF00084F8502062E77D212248F5F7FFFD4B466C
:10DF00005CE7102384F850306346DFF89090CC46ED
:10DF1000186859680833ACE803007345E146F6D148
:10DF200002F1230C6346DFF878A002F1330ED146EC
:10DF3000DCF80000DCF804100CF1080CA9E8030080
:10DF4000F445CA46F3D19C46DFF858A0D146DCF828
:10DF50000000DCF804100CF1080CA9E80300F445FB
:10DF6000CA46F3D1DFF84090CC46186859680833A8
:10DF7000ACE803007345E146F6D15FE74846FFF79A
:10DF80002BFBB4E681D70108C00000204DDC00085F
:10DF900040420F00A4E6010818010020980100206B
:10DFA00088010020780100206801002043788278F1
:10DFB0001B02007843EA024303430A20B3FBF0F05C
:10DFC0007047000038B5044681B10D7884B1A36A6A
:10DFD000012B0DD1E36A1BB95D210648F5F78EFDD3
:10DFE000E36A5878431B5842584138BDFF25EDE796
:10DFF0000020FAE700D80108044B93F8252083F8A5
:10E00000FF209A6AC3F80021704700BFC0000020BB
:10E01000024B93F8242083F8FD207047C0000020B5
:10E02000024B93F8232083F8FC207047C0000020A7
:10E03000054B93F8242093F8FD1091423ABF01203C
:10E0400083F8FD2000207047C0000020064A92F8A7
:10E05000FC3092F8231099423DBF03F1FF330120B9
:10E0600082F8FC3000207047C000002010B5FFF798
:10E07000C3FF0120FDF7C8FE5023164C0121237079
:10E080000023224614486370FDF738FE18B9322188
:10E090001248F5F733FD50230121114A1148A370AE
:10E0A000E170FDF72BFE18B936210C48F5F726FD77
:10E0B0005023237102230C4A01210C486371FDF7A0
:10E0C0001DFE28B9BDE810403A210448F5F716BDF9
:10E0D00010BD00BF444F0020043F0D0000D80108D0
:10E0E000464F0020CC3F0D00484F002094400D00CB
:10E0F000836A10B5012B044608D1C36A1BB94B21B2
:10E100000348F5F7FBFCE36A587810BD0020FCE7F4
:10E1100000D8010807B58DF807000DF10701044884
:10E12000FDF74AFC08B1FDF7ADFD03B05DF804FB57
:10E13000C5DF00082DE9F0414FF47A769046B1FB37
:10E14000F6F6C8F30317052F044630468CBF0027A8
:10E1500001274FF00005FDF749FD18B10F2C8CBFCA
:10E160000020012067F3000560F3410505F003037B
:10E17000032B0CD12046FFF7CDFF064B012103EB0B
:10E180004402547003F814803046FDF7B7FD28466A
:10E19000BDE8F081444F00200F282DE9F0410546ED
:10E1A0000F461FD8164B03EB40035C78231A5C42E2
:10E1B0005C414FF47A78B7FBF8F0FDF717FD4FF0AC
:10E1C000000360F3000364F3410303F00303032B34
:10E1D000064609D04FF0000066F3000064F34100EA
:10E1E000BDE8F0810024E4E72846FFF793FF044AE6
:10E1F000012102EB450208FB07F0FDF77FFDE9E78F
:10E20000444F0020002337B504460D4D8DF80730EC
:10E210000DF107012846FDF7CFFB18B1E3070CD538
:10E22000FDF70EFD9DF8073064080133DBB20F2BBC
:10E230008DF80730ECD903B030BDFDF7DFFCF1E716
:10E24000C5DF000838B504460320FFF763FF04204C
:10E25000FFF760FF0520FFF75DFF0620FFF75AFF7D
:10E260000720FFF757FF2046FFF7A0FE0546FDF702
:10E27000BDFC48B15023294A012193710323063282
:10E2800053702846FDF73AFDE01CFFF78FFE054668
:10E29000FDF7ACFC48B15023204A0121137204233E
:10E2A000083253702846FDF729FDA01DFFF77EFEBA
:10E2B0000546FDF79BFC48B15023184A0121937293
:10E2C00005230A3253702846FDF718FD04F10900B2
:10E2D000FFF76CFE0546FDF789FC48B150230F4A55
:10E2E0000121137306230C3253702846FDF706FDF7
:10E2F00004F10C00FFF75AFE0446FDF777FC58B115
:10E300005023064A204693730723D3730121BDE8A7
:10E3100038400E32FDF7F2BC38BD00BF444F00203C
:10E320000738C0B205289ABF014B185C0820704717
:10E33000BCD7010806289ABF014B185C0020704723
:10E34000C2D70108052804D90628034818BF0020B1
:10E3500070470248704700BF90D0030048E80100B2
:10E36000052810B5044604D940F241110348F5F7D9
:10E37000C5FB034B13F9240010BD00BF00D80108F2
:10E38000CCD70108142808B506DD0E484FF4A37158
:10E39000F5F7B4FB062008BD06280ADD08280ADDCB
:10E3A0000A280ADD0C280ADD0E28CCBF0020012037
:10E3B000F1E70520EFE70420EDE70320EBE702207B
:10E3C000E9E700BF00D8010808B50F280DD8DFE83D
:10E3D00000F0181818081A1A1A0A0A0C0C0C0C0C5F
:10E3E0000C0A732008BD0020FCE74FF4BC710748FD
:10E3F000F5F784FB064B074A40F27911034808F011
:10E40000B1FD3320EEE7DE20ECE700BF00D80108C5
:10E41000AFA80108E4D701082DE9F0468DB0924677
:10E4200099462A4A149B074693420C4608D0284A2C
:10E43000934203D0A6212748F5F760FB002600E0B1
:10E440000126254DEB6A98472046EB689847012F37
:10E450004FF0000422D108230A22CDE90132AB6932
:10E4600031460B93CDE90877CDE90644CDE9044464
:10E47000039400943B464A4602200B9EB047214637
:10E48000FF2004F01DF9082004F010F93421392090
:10E490002B6C0B930DB0BDE8F04618474FF47A6330
:10E4A0000127CDE907430823CDE90173EB69CDE9E5
:10E4B00005440B93CDE9034722465146CDF8009021
:10E4C000334602200B9CA0473946D9E790D0030081
:10E4D00048E801003DD80108A4E601082DE9F34110
:10E4E0000446104615460E469846FFF72BFF074692
:10E4F0002846FFF71FFFC5B21DB9C9210948F5F726
:10E50000FDFA64B94046FFF72BFF024600972B4601
:10E5100031462046FFF780FF02B0BDE8F0810022BF
:10E52000F4E700BF3DD801080A6803685340036060
:10E530004A684368534043608A68836853408360F5
:10E54000CA68C3685340C36070470B6810B514684D
:10E550006340036054684B686340436094688B6811
:10E5600063408360CB68D2685340C36010BD000035
:10E57000A1F11003DBB2102B2DE9F0470C46154634
:10E5800008D84FF0010909FA03F303F0013323F02F
:10E5900080732BB90023FF2085F8F030BDE8F087A9
:10E5A0000A460146284608F00BFE04F11C0E4FEA0D
:10E5B0008E0E5FFA8EFE4FEA1E13013B85F8F03097
:10E5C00023462749B3FBF4F204FB1232E81812F099
:10E5D000FF0210F804AC10F803CC10F8027C10F81D
:10E5E000016C32D111F80C804FEAD91289EA08087F
:10E5F00011F807C08F5D11F80A604FEA420A5244D1
:10E60000C24602EBC20282EA49025FFA82F91A1B91
:10E61000D2B215F802802A448AEA080A05F803A053
:10E6200092F8018004338CEA080C80F801C092F85B
:10E6300002C0DBB287EA0C078770D2789E4586EA73
:10E640000206C670BED80020A8E7182CDFD9102A11
:10E6500001BF11F80AA011F80CC0CF5D8E5DD6E79E
:10E6600077DA01082DE9F04F92F8F03097B00D916C
:10E670000B92002B00F0628101460EA8FFF765FFA8
:10E680000127AF4CAF4DB04E0B9B03EB07130C9320
:10E690000B9B93F8F030BB4259D8A94B9DF838201A
:10E6A0009DF83D109A5C595C8DF838209DF83C200F
:10E6B0009A5C8DF83C209DF840209A5C8DF84020B3
:10E6C0009DF844209A5C8DF844209DF839208DF8FF
:10E6D00039109DF841109A5C595C8DF83D109DF8F9
:10E6E00045108DF84520595C9DF83A208DF8411071
:10E6F0009DF842109A5C595C8DF842208DF83A10D2
:10E700009DF846109DF83E20595C9A5C8DF83E10AD
:10E710009DF843108DF84620595C9DF847208DF8F0
:10E7200047109DF83F100D98595C8DF843109DF8E7
:10E730003B10595C9B5C8DF83F100C9A0EA98DF82C
:10E740003B30FFF702FF002017B0BDE8F08F0DF15E
:10E75000580C0EAB0FCB0CE90F009DF849309DF81B
:10E7600048E002939DF84A309DF84D9001939DF842
:10E770004B309DF84C1003939DF84E309DF8560099
:10E7800004939DF84F3005939DF8503006939DF803
:10E79000513007939DF8533008939DF854300993F6
:10E7A0009DF855300A939DF852809DF857C015F892
:10E7B0000E2016F809B014F808A014F80C3082EAFC
:10E7C0000B028AEA02025A408DF8382014F80E2013
:10E7D00015F809B053408BEA030316F808B015F892
:10E7E000088083EA0B038DF8393014F809305A4059
:10E7F00082EA080216F80C808AEA030A16F80E303C
:10E8000082EA08028DF83A2083EA0A0A079A15F884
:10E810000C3015F8018016F802E08AEA030A039B1F
:10E8200014F800C0E35C88EA0E028CEA02025A4047
:10E830008DF83C20625C8DF83BA083EA0208079BC0
:10E8400015F803E08EEA080316F800E083EA0E03E9
:10E850008DF83D30079BE35C285C5A408CEA030C42
:10E86000735C4240039883EA0C0C039B305CEB5CC6
:10E8700042408CEA030C8DF83E20019B069A0A98D0
:10E88000E15C305C059BAA5CE35C42404A405A4034
:10E890008DF84020069A0A98A25C285C53404340B9
:10E8A00001988DF83FC0305C43408DF841300A9BA1
:10E8B0000198E35C285C5A40424005985940305C1E
:10E8C000069B42408DF84220F35C059A4B40A95CC0
:10E8D00002984B408DF84330049B305CE15C089B10
:10E8E000E25C099BEB5C43404B4053408DF8443065
:10E8F000099B0298E35C285C5A4042400498305CD3
:10E9000042408DF84520029A0498A25C285C53404E
:10E91000434008984A40305C43408DF84630099B9C
:10E920000EA8F15C089B5140EB5C59408DF84710F4
:10E930000C99FFF7F9FD7B1CDFB2A5E6FF2003E78A
:10E9400077DA010877D8010877D90108006870479D
:10E9500082B0034668B16A465968006803C25A1E0D
:10E960000DF10701073311F8010902F8010F9A426E
:10E97000F9D102B070470FB404B0704730B585B01C
:10E980006D4685E80F00104C95E80F0084E80F00F5
:10E9900004F1100208A903C982E803000BB90B4B6C
:10E9A000E360A3680BB9094BA36063680BB12368EC
:10E9B00033B9A36806489847064B6360064B23604B
:10E9C0000123237605B030BD3C4A002077E90008DA
:10E9D000E5DB010879710108697101082DE9F04151
:10E9E000184D80462B7E0E461BB973211648F5F74D
:10E9F00085F8DE2E03D974211348F5F77FF82B68CC
:10EA000080209847044680B18022002108F000FC55
:10EA1000B8F1000F12D08EB12B68304698470746E8
:10EA200030B920466B6898473C462046BDE8F081E7
:10EA30003246414608F0C4FB2677A7660023637080
:10EA4000F3E700BF3C4A0020A0DB010870B50A4C88
:10EA50000546237E1BB98F210848F5F74FF855B1BD
:10EA6000A86E18B1636898470023AB6663682846B0
:10EA7000BDE87040184770BD3C4A0020A0DB01088B
:10EA80002DE9F0479A4B17461A7E92B006460D467E
:10EA900098461AB9A7219748F5F730F8032F01D8FF
:10EAA0000024D7E03278737843EA42132B7033782E
:10EAB000022B02D0042B40F08C800023042F8DF811
:10EAC0002630EDD073686B7073681B0AAB70F388E7
:10EAD000EB70F3792B717368CDF822309DF82630F6
:10EAE000002B40F0C080052FDAD00624327AC2F322
:10EAF000400302F001019B0143EAC11343EA1213F0
:10EB0000C2F3800243EA42136B7196F808904FEA11
:10EB10001919631C9F42C3DD7289DBB22A557289C1
:10EB20000234120AEA54D8F810301A8873899A42CB
:10EB300004D040F247116F48F4F7E0FFD8F81420F2
:10EB4000D8F8103011781B6810290A930DD9029358
:10EB50000DF1220301930123317A009358320023EF
:10EB6000090906F10C0000F0C7FCB9F1000F0BD049
:10EB700004EB090A574593DB28194A4606F10C01B4
:10EB800008F01EFB5FFA8AF4337F002B76D0BC427C
:10EB900086D2727F04F101095FFA89F92A55D8F803
:10EBA0001430002A68D158330693B36E06A9079330
:10EBB000337F05EB0900ADF8203000F095FB4844A9
:10EBC000C4B2A7425AD240F275114A48F4F796FFF0
:10EBD00066E7032B01D0052B01D101236EE7002B43
:10EBE0003CD1082F7FF65CAFD8F81440681C224651
:10EBF00052F8083FC5F8013053684360FFF7A8FE9C
:10EC0000102F7FF64DAF224652F8103F05F1090054
:10EC1000C5F8093053684360FFF79AFE122F7FF65C
:10EC20003FAFB4F8983006A96B74B4F8983005A8D3
:10EC30001B0AAB7413232834CDE90645ADF8203008
:10EC400000F01CFB162F7FF62BAF1724059BC5F891
:10EC500013307366204612B0BDE8F087D8F80C3048
:10EC6000254898471CE740F23D112248F4F746FF3B
:10EC70004FF0000905244CE7883395E7E31C9F42D9
:10EC80007FF70EAFD8F814301A78102A0DD17833E8
:10EC900006A905A8CDE90635ADF8204000F057FAE1
:10ECA000059B2B510434E4B2D4E7112A19D103F1A6
:10ECB000780268330B930DF122030F930A9B0BA983
:10ECC0001093B6F87A3005A8ADF84430B6F87C3029
:10ECD0000C92ADF846300D95ADF8384000F06FFA63
:10ECE000DEE74FF4CB710348F4F708FFB2E700BF4B
:10ECF0003C4A0020A0DB010877DB01082DE9F04F3A
:10ED00009C4DA3B02B7E06460F46904623B940F299
:10ED1000A3119948F4F7F2FE022F40F294802B6879
:10ED200080209847044630B9EB68944898472046BD
:10ED300023B0BDE8F08F8022002108F069FA337813
:10ED40005B0923703278072B02F00302627003D153
:10ED5000EB688B48984773E0B8F1000F04D0012BA3
:10ED600002D1AB688748F5E7032B25D0052B23D0CC
:10ED7000012B40F0DB81112F40F0F680002384F856
:10ED800021306B691FFA87F828330893731C0993A5
:10ED900008F1FF33ADF82830337808A90DF13500BC
:10EDA0008DF8343000F082FA00280DF1340900F3B8
:10EDB000FD80EB687448CDE7701CFFF7C7FD014686
:10EDC0006060B8F1000F05D04045EB6835D1414691
:10EDD0006E4898470023052F6377A7F1040807D9E9
:10EDE000737903F00F0308339845C4BFF35C63776E
:10EDF000F379B07994F81DE040EA032096F805C055
:10EE000069696081BEF1000F1FD101F158034FF015
:10EE10000109CDE908360B786268102BCDF82A205D
:10EE2000ADF828808DF82E902A6902D9BEF1000F26
:10EE30000ED193684FF000090BE0424654489847C2
:10EE40006B6820469847002471E701F18803DEE7EC
:10EE50005368227A4FEADC1E6EF300024FEA5C1E12
:10EE60006EF382024FEA1C1E6EF3C3026CF30712AC
:10EE700022721A0C9BB2834284BF013292B200EB21
:10EE8000024B06EB0800CDF830B0FFF75FFD6831AC
:10EE90006066089107A808A900F059F9079B626EFF
:10EEA000934204D0EE683B493B48B047C8E72B6922
:10EEB0000BF10102B9F1000F2DD05A6094F808A0AF
:10EEC00004F10C034FEA1A1A5246184606F10801DB
:10EED000059308F075F96A691378102B0CD90DF1B8
:10EEE0002A0301930023CDF808B0009358324B4613
:10EEF0005146059800F000FB237A1B0903F10C0230
:10EF000097422DD903F10D02974206D100232348E1
:10EF10002377EB680AE79A60D0E70933A8EB030090
:10EF2000617FC0B220776A6961B958321E44089285
:10EF30000996ADF828002B689847A06620B9EB68C1
:10EF4000174807E78832F1E708A900F0CDF9002853
:10EF50003FF7EDAEEB68134898476B68A06EF9E693
:10EF600000232377A366E2E6212F3FF408AFEB6886
:10EF70000D48EFE63C4A0020A0DB010812DC010846
:10EF80002ADC010858DC010802DE010877DC0108F0
:10EF9000A7DC010834A20108E2DC010827DD010832
:10EFA0005BDD01088DDD0108B3DD01089DF83F3010
:10EFB000043F09EB0700DB09FFF7C8FC6E696066D8
:10EFC000A3B30DF1580A00213022504608F020F971
:10EFD000FF2332468DF8583052F8083F0DF15900A2
:10EFE000CDF8593053683836CDF85D30FFF7B0FCB6
:10EFF000B6F860303A468DF8613049461B0A0DF18B
:10F0000063008DF8623008F0DBF8CDE9086A08F19A
:10F01000070808A907A8ADF8288000F02FF9636E4B
:10F02000079A9A4208D0EB68424893E62836CDE921
:10F030000869A8F10408ECE79DF837609DF83630C0
:10F04000360446EA03269DF835300DF13B001E4399
:10F0500066609DF83A709DF839303F0447EA03270F
:10F060009DF838301F43A760FFF770FCE0609DF803
:10F070003F20237CD10961F3C713110961F3061303
:10F0800062F3030323749DF84030637494F82130D5
:10F0900003B3BDF8413063829DF84330BDF844208E
:10F0A00023759DF84630A4F81520E375BDF8473068
:10F0B00023839DF84930A376BDF84A30A4F81B306D
:10F0C0009DF84C306377BDF84D30E3839DF84F30A9
:10F0D00084F820306D6994F9102005F1280C002A7D
:10F0E000B5F8981004F1230004F15303CDF858C08B
:10F0F00016AA12DA05F11807ADF868100092083563
:10F1000004F1430204F13301CDE91776199500F0BB
:10F1100083F9012384F8223009E6ADF8641019461A
:10F12000CDE9176700F03AF90023F3E7EB680248EE
:10F1300010E600BF25DE01085ADE01080022FFF7B5
:10F14000DDBD0B0C0180090E8370C170704770B576
:10F150001025CEB00C462A4606460021684608F027
:10F1600057F849238DF80030A37BD4F80A100DF12D
:10F1700006008DF80530FFF7E4FF21690DF10A0064
:10F18000FFF7DFFF238908A88DF80F3000F0F8F9AA
:10F19000216808A800F004FA2A46694608A800F089
:10F1A00005FA2289616808A800F000FA08A90DEBA9
:10F1B000050000F062FA049B33604EB070BD492335
:10F1C00070B500250C460646CEB08DF800300B8B8E
:10F1D000CDE901558DF801301B0A8DF802308B7E88
:10F1E00003958DF80330CB7E0DF106008DF80430C9
:10F1F0000B691968FFF7A5FF61690DF10A00FFF7B8
:10F20000A0FFA38908A88DF80F308DF80E5000F0EC
:10F21000B7F9216808A800F0C3F9694608A81022C8
:10F2200000F0C4F9A289A16808A800F0BFF908A9F4
:10F2300004A800F022FABDF8103008A833808DF839
:10F240000150ADF802508DF8045000F099F9616852
:10F2500008A800F0A5F9694608A8102200F0A6F950
:10F26000A289A16808A800F0A1F908A904A800F0E3
:10F2700004FABDF8103073804EB070BD30B50C4646
:10F28000CBB0054604A800F07BF9216804A800F083
:10F2900087F92289616804A800F088F904A9684602
:10F2A00000F0EBF9009B2B604BB030BD70B50C89C2
:10F2B000BEB006460D46A4B114F00F0411D101AA48
:10F2C00010212868FFF754F92889A04201DC3EB0DC
:10F2D00070BD68683119204401AAFFF7C3F91034E2
:10F2E000F2E74FF0FF30F2E72DE9F0430F89C7B0A6
:10F2F00081460D46002F4ED0012410224FEA1718E8
:10F30000002117F00F0701A818BF08F1010807F046
:10F310007FFFAB7BD5F80A100DF10A008DF809309C
:10F320008DF80440FFF70DFF29690DF10E00FFF77E
:10F3300008FF6E68013E444503DD288947B0BDE8FB
:10F34000F08309AA102128688DF81340FFF710F9FF
:10F3500009AA05A901A8FFF785F9444510DB002F8C
:10F3600014BF3B46102330464A464B440DF1140C63
:10F37000934207D80134A4B209F110091036DAE734
:10F380001023F0E710F801EF1CF8011B81EA0E01D1
:10F3900002F8011BECE74FF0FF30CFE770B5C2B0C9
:10F3A000144606460D46F122002105A807F030FF5D
:10F3B0000023CDE90333636810218DF805301A0A64
:10F3C0001B0C8DF8073023898DF80620ADF8083026
:10F3D000638905AA8DF80A30A38920688DF80B305F
:10F3E0001B0A8DF80C3001238DF80430FFF7C0F8AC
:10F3F00005AA314601A8FFF735F9022305AA102115
:10F4000020688DF80430FFF7B3F805AA294601A853
:10F41000FFF728F942B070BD2DE9F0431025C3B0C5
:10F420004A9C80460F4616460021F12205A89946BF
:10F4300007F0EEFE2A46002101A807F0E9FEA268C7
:10F4400029468DF80520130AEA408DF80720E26866
:10F450008DF80630D37920688DF8083093798DF8CF
:10F46000093053798DF80A3013798DF80B30D37841
:10F470008DF80C3093788DF80D3053788DF80E3070
:10F48000137805AA8DF80F30238AADF810300123C8
:10F490008DF80430FFF76CF805AA414601A8FFF784
:10F4A000E1F8022305AA294660688DF80430FFF7C9
:10F4B0005FF805AA494601A8FFF7D4F8032305AA77
:10F4C000294620688DF80430FFF752F805AA39461E
:10F4D00001A8FFF7C7F8042305AA294620688DF87C
:10F4E0000430FFF745F805AA314601A8FFF7BAF83E
:10F4F00043B0BDE8F0830000F0B50F29C7B0044663
:10F500000D4616461F4604D94FF4A1711B48F4F767
:10F51000F5FA0123002F019318BF02238DF808305C
:10F520009DF830310DF10A0083F001038DF80930A8
:10F530004D9B1968FFF705FE4E990DF10E00FFF780
:10F5400000FE4FF4807309AA1021304605AEADF8D5
:10F550001230FFF70DF809AA314601A8FFF782F82B
:10F560000023601EDAB2954201D847B0F0BD10F812
:10F57000012FF15C01334A400270F3E794DE010889
:10F5800010B5102204460021F13007F041FE0021A1
:10F590002046C4F81411F022BDE8104007F038BE30
:10F5A0000B46024610211846FEF7E2BF2DE9FF4741
:10F5B0000446D0F814018846154604F2011910B328
:10F5C000C0F1100797423E4628BF164648443246CF
:10F5D00007F0F6FDD4F8143133440F2BC4F814317E
:10F5E0001CD9AF421AD204F1F10319461A78187CDB
:10F5F000424003F8012B4B45F8D122460846FFF75D
:10F6000031F8B044AD1B0DF1100A102D09D82A466F
:10F610004146484607F0D4FDC4F8145104B0BDE893
:10F62000F08704F1F1031E4608F1FF311A7811F852
:10F63000010F424003F8012B4B45F7D16A46334690
:10F6400017469446186859680833ACE803004B45E0
:10F650006246F6D1224639463846FFF703F833466C
:10F660003A4603CA524518605960174603F1080329
:10F67000F6D108F11008103DC7E7F0B50C4689B087
:10F68000102200210546684607F0C2FD2246694661
:10F690006846FEF7E7FF9DF900306A46002B4FF001
:10F6A00000013EDA537810780131DB0943EA400368
:10F6B0000F2902F8013BF5D19DF80F305B0083F074
:10F6C00087038DF80F30D4F81431102B37D16946E9
:10F6D00004F2011304F211101A7811F8016B724050
:10F6E00003F8012B9842F7D104F1F102134604F21A
:10F6F00001171178107C414002F8011B9742F8D1A4
:10F7000004AA9446164618685968083303C6BB42D3
:10F710003246F7D1224629466046FEF7A3FF09B0DC
:10F72000F0BD537810780131DB0943EA40030F291B
:10F7300002F8013BF5D19DF80F305B00C1E79DF960
:10F7400000206946002A4FF0000028DA4A780E7837
:10F750000130D20942EA46020F2801F8012BF5D107
:10F760009DF80F20520082F0870280218DF80F2033
:10F77000E21882F80111002104F2011201330F2B6B
:10F780001BD9C4F814316B4604F21110117813F828
:10F79000016B714002F8011B9042F7D1A4E74A784F
:10F7A0000E780130D20942EA46020F2801F8012BF7
:10F7B000F5D19DF80F205200D7E7D154DEE70000C5
:10F7C000002103E00A4B5B584350043109480A4BBF
:10F7D00042189A42F6D3094A02E0002342F8043B59
:10F7E000074B9A42F9D300F00DF8F1F78BFC704704
:10F7F00028EE010800000020180300201803002054
:10F80000F84F0020314B82B01A6842F480721A60BF
:10F8100099682F4A0A409A601A6822F0885222F0AA
:10F8200001121A601A6822F480221A609A6822F47F
:10F830007D029A600022DA6001921B6813F4007363
:10F8400018BF01230193019B012B37D14FF4805145
:10F85000204B1A68A3F5806322F00102C3F800244C
:10F86000D3F8002422F00202C3F80024D3F80024C5
:10F8700022F00402C3F800245A6A42F080525A620D
:10F88000154A11605168C906FCD49A689A609A6852
:10F890009A609A689A605A6822F460425A605A687C
:10F8A00042F440425A609A6822F003029A609A68D1
:10F8B0009A60064A936813F00C0FFBD14FF0006278
:10F8C000064B9A60064ADA6002B070470038024080
:10F8D0000CC0FF88003C02400070004000ED00E0DA
:10F8E0000003FA0570B5064688B02D4801F086FC85
:10F8F0002C4B1A680092009A91073AD501214FF4D7
:10F90000007001F0D5FE012001F0C6FC264A5368C4
:10F9100043F400335360A2F5374253681B07FCD50C
:10F920000024012502A801F0A3FC02A91C480694AA
:10F930008DF81C50ADF80C4001F074FC2A460623EB
:10F940003146174801F0B4FC2946154801F09BFCEC
:10F950000221134801F03EFD114801F02DFD134D29
:10F9600001940F4C0221204601F02EFD58B108B041
:10F9700070BD1A6842F001021A60009A9207BDD465
:10F980001A680092F9E7019B01330193019BB3F5DB
:10F99000805FE7DB38212846F4F7B0F8E2E700BFE4
:10F9A000002401400038024000270140DFDE01084A
:10F9B00008B5002001F070FC0021074801F063FC4D
:10F9C00000214FF4007001F073FE044A136823F025
:10F9D0000103136008BD00BF00240140003802404D
:10F9E00013B5072301220146114801F061FC0221F1
:10F9F0000F4801F0EFFC0E4801F0DEFC00230D4C37
:10FA0000019302210A4801F0DFFC28B1084802B046
:10FA1000BDE8104001F0D5BC019B01330193019B6F
:10FA2000B3F5805FEDDB4C212046F4F767F8E8E79B
:10FA300000240140DFDE010870B506460825FFF707
:10FA400051FF00243046FFF7CBFF013D0444F9D1BC
:10FA5000FFF7AEFFC4F3CF0070BD00000000000050
:10FA600008B51120FFF7E8FF06F05EFE01460848E2
:10FA700006F066FF06F040FA03A3D3E9002306F080
:10FA800093FA06F04BFD08BD2FDD24068195F33F68
:10FA900000F07F450F4A536A43F0805353620E4B88
:10FAA0001A465968C906FCD41B68022823F4C053BF
:10FAB00006D143F4C05313605368DB06FCD470478F
:10FAC000012802D143F48053F5E70028F3D143F431
:10FAD0000063F0E7003802400070004010B50C4BA6
:10FAE0005A68D206FCD41C6814F4C05F0BD114F41D
:10FAF00080500AD114F4006404D106482A21F3F797
:10FB0000FDFF204610BD0220FCE70120FAE700BF00
:10FB10000070004025DF010838B50546012001F0DE
:10FB200069FC022D01BF144A136843F001031360FE
:10FB3000124B1A6842F480721A601A689205FCD55A
:10FB40005A6822F4604242F440425A6000229A60AD
:10FB50000A4B9C6814F00C04FBD14FF480721A60BD
:10FB6000074B084A28461A60FFF794FF2046BDE875
:10FB7000384001F033BC00BF003C02400038024076
:10FB8000F8010020D0FE3F000C4B5A6B900513D4B7
:10FB90005A6A42F080525A62094A116841F48071EF
:10FBA0001160596B41F480715963596B8905FCD51B
:10FBB000136823F480731360704700BF003802405D
:10FBC00000700040054B5A6B910706D45A6B42F007
:10FBD00001025A635A6B9207FCD570470038024005
:10FBE000094B5A6A42F020025A629A6942F0200296
:10FBF0009A619A6922F020029A610022A3F50933E2
:10FC00001A801A855A627047003802401521002276
:10FC100002384143064B1A85D962012199825A6202
:10FC20001A8219801A8AD207FCD500221A807047DE
:10FC300000140040002349F6FE7282B00193019B3C
:10FC4000934201DD02B07047019B01330193F6E757
:10FC5000002340F6FE7282B00193019B934201DDC6
:10FC600002B07047019B01330193F6E7002382B095
:10FC70000193019BB3F5CC7F01DD02B07047019B7E
:10FC80000133F5E7D0B1012801D1FFF7EFBF0C4BED
:10FC900000211A684FF47A73B2FBF3F2094B013A70
:10FCA00092B21A8501220138D8629A825962198269
:10FCB0001A801A8AD207FCD500221A80704700BF2A
:10FCC000F80100200014004000F1774303F57803A9
:10FCD000B3F5804F2DE9F04106460C4617462DD26C
:10FCE00002F1F73303F608030344B3F5804F25D23E
:10FCF000FFF7F4FE804610B10020FFF7CBFE01F0C5
:10FD000091FB01252744361BA7420AD101F09AFB3B
:10FD1000B8F1000F02D04046FFF7BCFE2846BDE810
:10FD2000F08141F6027001F095FB301914F8011BC7
:10FD300001F0ECFB042818BF0025E5E70025EDE7FE
:10FD400010B50C4600F1774101F57801B1F5804F0F
:10FD50000DD202F1F73303F608030344B3F5804FE5
:10FD600005D20146204607F02BFA012010BD0020E5
:10FD7000FCE7000008B5114B984215D003F58063ED
:10FD8000984213D003F58063984211D003F5806345
:10FD900098420FD003F5006398420DD0084B094AF2
:10FDA0001421094807F0DEF8002008BD0120FCE717
:10FDB0000220FAE70320F8E70520F6E700000240FA
:10FDC000B4DF01086EDF0108CDDF01080F2808B598
:10FDD00005D9094B094A3B21094807F0C3F801231B
:10FDE00003FA00F0C043074A5168014051601368AC
:10FDF0001840106008BD00BF16E0010878DF010858
:10FE0000CDDF0108000401400F292DE9F84F82469B
:10FE10000D4693461F4605D95A4B5B4A54215B4811
:10FE200007F0A0F84FF0010909FA05F900F0B8F859
:10FE30006FEA0903564E032D7268564C02EA03021C
:10FE40007260326803EA0203534A3360136A43F074
:10FE5000010313622ED80F22A3684FEA850802FA25
:10FE600008F223EA0203A3605046FFF783FFA3686A
:10FE700000FA08F01843A0601BF0020F18BFB36827
:10FE8000464A1CBF43EA0903B3601BF0040F1EBFC0
:10FE9000F36843EA0903F360336843EA0903336014
:10FEA0003B01DBB2002D45D182F8063340231360BD
:10FEB000BDE8F88F072D13D80F22A5F10408E368D9
:10FEC0004FEA880802FA08F223EA0203E360504688
:10FED000FFF750FFE36800FA08F01843E060CBE753
:10FEE0000B2D13D80F22A5F1080823694FEA8808C3
:10FEF00002FA08F223EA020323615046FFF73AFFB1
:10FF0000236900FA08F018432061B5E70F22A5F134
:10FF10000C0863694FEA880802FA08F223EA020330
:10FF200063615046FFF726FF636900FA08F0184343
:10FF30006061A1E7012D03D182F807338023B6E782
:10FF4000022D04D182F808334FF48073AFE7032DFC
:10FF500004D182F809334FF40073A8E7042D04D1CB
:10FF600082F80A334FF48063A1E7092D04D882F8A0
:10FF700017334FF400039AE782F828334FF4807365
:10FF8000536095E722E0010893DF0108CDDF010807
:10FF900000040140000001400038024000E100E0A0
:10FFA000144B984205D1144AD36943F00103D3613D
:10FFB0007047124B984204D10F4AD36943F00203B1
:10FFC000F5E70F4B984204D10B4AD36943F0040381
:10FFD000EDE70C4B984204D1074AD36943F008037C
:10FFE000E5E7094B9842E3D1034AD36943F0200384
:10FFF000DDE700BF0000024000380240000402407C
:020000040801F1
:1000000000080240000C0240001402400323490093
:1000100010B584688B4024EA030484600124022A1A
:1000200004FA01F407D0032A0DD0012A07D183680E
:100030002343836003E083688A401A4382608368B5
:100040001C43846010BD82681343F2E70F29F8B5A2
:1000500004460F4615461E4603D940211948F3F7BA
:100060004DFD2046FFF79CFF03237A009340DB43BE
:100070002168194021600121D4F800C001FA02F082
:100080004CEA000CB940C4F800C009B266B1A688B9
:10009000314389B2A180E168012D03EA0103E360E5
:1000A00006D0022D08D0F8BDA68826EA0101F1E7A6
:1000B000E3680343E360F6E7E36805FA02F21A43F4
:1000C000E260F0E772E001080F2970B505460C46C2
:1000D000164603D960210E48F3F710FD2846FFF7B6
:1000E0005FFF032361008B40DB43EA68012E02EAD5
:1000F0000302EA6005D0022E03D02A6813402B6069
:1001000070BDEA6806FA01F11143E960F5E700BF46
:1001100072E001080F2910B505D9074B074A76216F
:10012000074806F01FFFFFF73BFF4B000321026863
:1001300099401143016010BD16E001082EE001084E
:1001400072E001080F2938B50446154605D97C210F
:100150001B4B1C4A1C4806F005FF0F2A03D91B4BFA
:10016000184A7D21F6E7FFF71BFF07294FF00F0321
:1001700018D8006A8A00934020EA03032362236AA6
:1001800005FA02F21A4322620322236849008A40D8
:1001900023EA020323600223226803FA01F11143D8
:1001A000216038BDA1F10802406A9200934020EA24
:1001B00003036362636A95401D436562E4E700BF21
:1001C00016E0010841E0010872E001085FE0010863
:1001D000012303FA01F189B201837047012303FA75
:1001E00001F189B241837047012303FA01F189B219
:1001F0000AB10183704741837047008A084100F0CB
:10020000010070470F2938B505460C4603D9A921CE
:100210000548F3F773FC28686400E04000F0030031
:10022000431E5842584138BD72E00108808A084197
:10023000C04300F00100704710B5074C236853B964
:100240000120F3F7C5F8206028B9BDE81040362139
:100250000248F3F753BC10BD584A0020B9E001082A
:1002600010B50B4C22681AB93C210A48F3F746FC3A
:10027000206842F21071F3F7F3F901280CBF012452
:10028000002403D040210348F3F738FC204610BD7A
:10029000584A0020B9E0010810B5074C22681AB985
:1002A0004D210648F3F72AFC002320681A46BDE8D2
:1002B00010401946F2F7E8BF584A0020B9E001089B
:1002C00010B50446FFF7B8FFFFF7CAFF214610221A
:1002D000034801F0A7FE0446FFF7DEFF204610BDED
:1002E0000054004010B5FFF7A7FFFFF7B9FF01F07A
:1002F00051FE0446FFF7D0FF204610BD08B5134657
:100300000A460146034801F0BDFA003018BF01203B
:1003100008BD00BF0054004008B513460A46014618
:10032000034801F0B5FB003018BF012008BD00BF35
:100330000054004008B513460A460146034801F040
:100340003BFC003018BF012008BD00BF0054004036
:1003500008B513460A460146034801F0BFFC0030C9
:1003600018BF012008BD00BF0054004008B5134667
:100370000A460146034801F00BFD003018BF01207A
:1003800008BD00BF005400400123064A8340516964
:10039000194205D05361044B53F8203003B118477C
:1003A000704700BF000401405C4A00200F2838B5A8
:1003B00004460D4603D926210348F3F79FFB034B60
:1003C00043F8245038BD00BFFFE001085C4A00201C
:1003D0000020FFF7D9BF0120FFF7D6BF0220FFF7AB
:1003E000D3BF0320FFF7D0BF0420FFF7CDBF08B570
:1003F0000920FFF7C9FF0820FFF7C6FF0720FFF716
:10040000C3FF0620FFF7C0FFBDE808400520FFF747
:10041000BBBF08B50F20FFF7B7FF0E20FFF7B4FFF3
:100420000D20FFF7B1FF0C20FFF7AEFF0B20FFF709
:10043000ABFFBDE808400A20FFF7A6BFFEE7FEE7D6
:10044000FEE7FEE7FEE7FEE7FEE7FEE7FEE7FEE784
:10045000FEE7FEE7FEE7FEE7FEE7FEE7FEE7FEE774
:10046000FEE7FEE7FEE7FEE7FEE7FEE7FEE7FEE764
:10047000FEE7FEE7FEE7FEE7FEE7FEE7FEE7FEE754
:10048000FEE7FEE7FEE7FEE7FEE7FEE70A23B0FB36
:10049000F3F203FB120040EA0210C0B27047000002
:1004A000CA22024B5A6253225A6270470028004007
:1004B000014B1860704700BF9C4A00204FF4003287
:1004C0000F4B10B50F4C5A61E368DB0503D43021A4
:1004D0000D48F3F713FBFFF7E3FF4FF40072A36837
:1004E00023F48853A360094BC3F88420FF2363627D
:1004F000074B1B6813B1BDE81040184710BD00BF83
:10050000000401400028004045E1010800E100E04E
:100510009C4A00202DE9FF479A46364B80461B78BF
:1005200091469DF830709DF834602BB9324B334AB8
:100530008C21334806F016FD431E1E2B58D80C297B
:1005400056D8A2F5FA63632B52D8BAF1170F4FD8D9
:100550003B2F4DD83B2E4BD802F13000C0B2FFF7F5
:1005600095FF05460846FFF791FF000240EA054562
:100570004046FFF78BFF05435046FFF787FF0446D1
:100580003846FFF783FF000240EA04443046FFF795
:100590007DFF20431B4CFFF783FFE36845F40055C4
:1005A00043F08003E360E3685B06FCD56560206090
:1005B000E36823F08003E360124BDA689206FCD50F
:1005C000FF2201A85A628DF807808DF80810ADF857
:1005D00009908DF806A08DF805708DF80460FAF783
:1005E000ACFD094BC3E90001012004B0BDE8F08770
:1005F0000020FAE7A04A0020BEE101089DE10108C1
:1006000045E1010800280040A84A002007B503780A
:100610000193437800938378B0F805200179C0787E
:10062000FFF778FF03B05DF804FB000038B52B4BF3
:1006300004461B781BB9E4212948F3F75FFA294ADD
:10064000D36823F02003D360D3689B06FCD51368DE
:100650005268C2F30741080900EB800001F00F0166
:1006600001EB4001C9B201F5FA61A4F80510C2F32B
:100670000721C1F300108500284401F00F0101EBB0
:100680004001D2B22171C2F3011101EB810102F0EC
:100690000F0202EB4102E270C3F30742C2F3011101
:1006A00001EB810102F00F0202EB4102A270C3F3E1
:1006B0000722C2F3021101EB810102F00F0202EBEB
:1006C0004102DBB26270C3F3021202EB820203F05A
:1006D0000F0303EB4203237038BD00BFA04A002084
:1006E00045E10108002800401FB501A8FFF79EFF63
:1006F00001A8FAF722FD05B05DF804FB08B5FFF785
:1007000043FA1B4A136843F480731360FFF7C8FE73
:10071000184A536B23F4403343F482035363164B5C
:10072000DA6842F08002DA60DA685106FCD5FF220E
:100730001A611A6942F4FE021A619A6822F04002B4
:100740009A609A6822F44C529A60DA6822F0800229
:10075000DA60094BDA689206FCD5FF225A62012260
:10076000064B1A70FFF7C0FF054BC3E9000108BD37
:10077000007000400038024000280040A04A0020DD
:10078000A84A002008B5094B1B7823B940F21F1175
:100790000748F3F7B3F9FFF783FE064B9A6822F494
:1007A00080729A60FF225A6208BD00BFA04A0020F2
:1007B00045E101080028004008B5144B1B7833B907
:1007C000134B144A40F22711134806F0CBFBFFF7F6
:1007D00067FE124BDA6822F48072DA60104A916880
:1007E00041F400319160116841F400311160F02151
:1007F0000C4A82F829134FF4007151609A6842F450
:1008000088529A60FF225A6208BD00BFA04A0020A9
:10081000BEE10108A9E1010845E101080028004006
:100820000004014000E100E0F8B51E46194B1746F0
:100830001B7833B9184B194A4FF4A371184806F0C6
:1008400091FB184CFFF72CFEA56825F48075A56078
:10085000E56825F48075E560FFF718FE0546084653
:10086000FFF714FE000440EA05613846FFF70EFE6C
:1008700005463046FFF70AFE084340EA0520E368D4
:10088000DB07FCD5FF23E0616362BDE8F840FFF7BA
:1008900093BF00BFA04A0020BEE101088BE1010820
:1008A00045E101080028004038B50D460446F2F73E
:1008B00001FA194A136823F001031360F2F71AFAD8
:1008C00025B1164A536843F00603536072B6BFF36E
:1008D0004F8FBFF36F8F124A0120136823F0030379
:1008E00043F4007343F00103136000F08FFD0D4BE0
:1008F0001A6942F004021A6130BF1A69022022F01C
:1009000004021A61FFF708F9034A136843F0010370
:10091000136004B162B638BD10E000E0002004E0CE
:100920000070004000ED00E062B6704700220E4B00
:1009300010B51A700D4A0E4C1388204623F0400360
:100940001B041B0C13800D210222FFF7BDFB204668
:1009500002220E21FFF7B8FB2046BDE8104002221C
:100960000F21FFF7B1BB00BFB04A002000380040A4
:100970000004024038B50546284A2948536A0C4607
:1009800043F4804353620D210522FFF7DBFB052270
:100990000E212348FFF7D6FB05220F212048FFF741
:1009A000D1FBC5B101220D211D48FFF72FFB01220C
:1009B0000E211B48FFF72AFB01220F211848FFF7E1
:1009C00025FB012C1BD144F451740122154B1C80D2
:1009D000154B1A7038BD2A460D211148FFF716FB3A
:1009E0002A460E210E48FFF711FB2A460F210C481C
:1009F000FFF70CFB012C09D144F45974E5E7022CF4
:100A0000E1D0032C0CBF03240024DCE7022CF3D03C
:100A1000032C14BF00240324EEE700BF003802407B
:100A20000004024000380040B04A0020064B074A4C
:100A3000988111781A461889C00701D40029FAD183
:100A40009089C0B2704700BF00380040B04A002013
:100A5000294A38B5136A054643F4805313620522C8
:100A600026480C461146FFF76DFB05220621234858
:100A7000FFF768FB052207212048FFF763FBC5B19C
:100A8000022205211D48FFF7C1FA022206211B4858
:100A9000FFF7BCFA022207211848FFF7B7FA012C2A
:100AA0001BD144F451740122154B1C80154B1A7054
:100AB00038BD2A4605211148FFF7A8FA2A46062123
:100AC0000E48FFF7A3FA2A4607210C48FFF79EFAC3
:100AD000012C09D144F45974E5E7022CE1D0032C30
:100AE0000CBF03240024DCE7022CF3D0032C14BF3A
:100AF00000240324EEE700BF00380240000002405B
:100B000000300140B14A002000220E4B10B51A708F
:100B10000D4A0E4C1388204623F040031B041B0C87
:100B2000138005210222FFF7CFFA20460222062178
:100B3000FFF7CAFA2046BDE8104002220721FFF75E
:100B4000C3BA00BFB14A002000300140000002409B
:100B5000064B074A988111781A461889C00701D4B4
:100B60000029FAD19089C0B2704700BF003001401F
:100B7000B14A0020054AD36823F4E0631B041B0C30
:100B800043F0BF6343F40033D360704700ED00E0EF
:100B900020220021114B10B5C3F88420104B114CBA
:100BA0001A6A204642F480421A625A6942F480422C
:100BB0005A615A6922F480425A610B4A91811A6A39
:100BC000092122F480421A620222FFF77DFA2046B0
:100BD000BDE8104002220A21FFF776BA00E100E0EA
:100BE00000380240000002400038014008B5064BC2
:100BF0000246186000B1012240F22551034800F07E
:100C0000FCFD012008BD00BFB44A002000380140AF
:100C100010B50B4C40F22551204600F00CFE48B1B7
:100C2000204600F0E6FD074B1B683BB1BDE81040D5
:100C3000C0B21847A388044ADBB2137010BD00BFCE
:100C400000380140B44A0020644F002010B504462B
:100C50008021084800F0E9FD0028F9D02146054828
:100C600000F0C3FD034C4021204600F0DEFD0028CB
:100C7000F9D010BD0038014010B5441E14F8010F22
:100C800000B910BDFFF7E2FFF8E7000008B5024821
:100C900000F0AFFDC0B208BD003801402DE9F041C1
:100CA0000F4601214FF4C066804688B008461446BE
:100CB0001D4600F0EFFC01214FF4804000F0F8FCED
:100CC0003B4B02A93B48CDE9026300F045FC0722FB
:100CD0000921384800F082FC07220A21354800F03B
:100CE0007DFC452FCDF810803AD14FF48063ADF8EC
:100CF0001830072C40D10023ADF81430052D4CD10D
:100D00004FF48053ADF816300023ADF81C300C239F
:100D100004A92948ADF81A3000F00CFD274B1A68D9
:100D200002B1012240F22551234800F066FD012165
:100D3000214800F04FFDFFF7A9FF25238DF804306F
:100D40009DF838308DF805304FF48073ADF80630DB
:100D5000FFF710FF01A800F035FA08B0BDE8F081F8
:100D60004F2F02D1ADF81860C3E70023072CADF870
:100D700018300DD1592107E0082C02D14FF48053CF
:100D8000BAE7092CBAD154210D48F2F7B7FEB5E7FE
:100D9000082CB0D0092CB1D1F0E70F2D02D14FF4BF
:100DA0004053AFE7022D0CBF4FF400530023A9E7D7
:100DB000020200010000024000380140B44A002055
:100DC000C7E101080E2307B5082200934E21012335
:100DD000FFF764FF03B05DF804FB00004022002130
:100DE0000D4B0E48C3F884200D4B5A6A42F4003272
:100DF0005A629A6942F400329A619A6922F4003286
:100E00009A61084A91815A6A032122F400325A6297
:100E10000222FFF759B900BF00E100E000000240E4
:100E2000003802400044004008B5024800F0E1FCF0
:100E3000C0B208BD004400402DE9F0471F462623FC
:100E400088B08DF8043000239DF840808946144610
:100E5000ADF8063082469DF844509DF848608DF804
:100E60000580FFF787FE01A800F0ACF901210846D4
:100E700000F010FC01214FF4003000F027FC65B1B8
:100E80000821504B5048CDE9021302A900F064FB41
:100E9000072203214C4800F0A1FB66B10422494B14
:100EA00002A94948CDE9022300F056FB072202219E
:100EB000454800F093FBB9F1450FCDF810A041D1A2
:100EC0004FF48063072CADF8183049D10023ADF8FA
:100ED0001430052F55D14FF480530024ADF816304F
:100EE000ADF81C40002E57D1ADF81A6075B1BDF8B1
:100EF0001A3043F00403ADF81A30344B1A6802B1CB
:100F0000012240F22551324800F077FC04A9304814
:100F100000F010FC01212E4800F05CFC0DB1FFF741
:100F200083FF26238DF804304FF480738DF80580FD
:100F3000ADF80630FFF71EFE01A800F043F908B037
:100F4000BDE8F087B9F14F0F02D14FF4C063B9E7A4
:100F50000023072CADF818300ED14FF4827107E052
:100F6000082C02D14FF48053B1E7092CB1D1FF21F5
:100F70001848F2F7C3FDACE7082CA7D0092CA8D17C
:100F8000F0E70F2F02D14FF44053A6E7022F0CBF1A
:100F90004FF400530023A0E70823224640F22771B4
:100FA0000B48ADF81A3000F028FC40F226610848E2
:100FB00000F060FC224640F22661054800F01DFC6E
:100FC00094E700BF0203000100000240B84A00207D
:100FD00000440040C7E10108F8B505460024134E5F
:100FE000134F8021134800F020FC68B129461148B6
:100FF00000F0FBFB00240F4D0C4E0D4F4021284606
:1010000000F013FC48B1F8BD0134B442E9D94FF403
:10101000A4713846F2F772FDE3E70134B442EDD92A
:1010200040F251113846F2F769FDE7E7FFFF0F0084
:10103000C7E101080044004008B5064B02461860AD
:1010400000B1012240F22551034800F0D6FB0120F7
:1010500008BD00BFB84A00200044004070B5134CE2
:1010600040F22551204600F0E6FBC0B1104B1D6850
:1010700025B1204600F0BDFBC0B2A84740F2266172
:101080000A4800F0D8FB78B140F22661074800F02A
:10109000F1FB084B1B683BB1BDE870401847A388C3
:1010A000054ADBB21370E9E770BD00BF00440040A1
:1010B000B84A0020BC4A0020644F0020BFF34F8F85
:1010C0000449054BCA6802F4E0621343CB60BFF3E6
:1010D0004F8FFEE700ED00E00400FA0510B5441E56
:1010E000E3B2052B03D90E211148F2F707FDFEF7F5
:1010F00069FD45F255520F4B1A60DA68D207FCD4ED
:10110000052C06D8DFE804F0030A0C0E10120122A9
:101110005A604CF6CC42074B1A6010BD0222F7E72A
:101120000322F5E70422F3E70522F1E70622EFE7C1
:1011300098E201080030004010B5194C23683BB913
:101140005F2000F0DFFA28B1164B236000F0EAFAC6
:10115000206810BD5E2000F0D5FA08B1124BF4E70C
:101160005D2000F0CFFA08B1104BEEE75C2000F0F4
:10117000C9FA08B10E4BE8E75B2000F0C3FA08B1EA
:101180000C4BE2E75A2000F0BDFA08B10A4BDCE74D
:10119000592000F0B7FA08B1084BD6E7084BD4E75E
:1011A000C04A00200EE201081EE2010834E20108F4
:1011B0004FE201085EE201086DE2010886E20108E3
:1011C00090E2010830B5012403780A4D03F01F02B4
:1011D0009440C278590952B1074A2B44D2684278E8
:1011E0001201D2B283F8002345F8214030BD2031EE
:1011F000FAE700BF00E100E000ED00E008B5084BB1
:1012000098420BD101214FF4007000F06DFABDE857
:10121000084000214FF4007000F066BA08BD00BF1E
:101220000024014043680A7923F0407323F480735B
:1012300043EA02230A6810B513434360D1E903234C
:1012400013438A6884681343084A224013434A7947
:1012500043EA420383600A7D036B013A23F0F8738B
:10126000D2B243EA0253036310BD00BFFDF7FFC0D3
:1012700000234FF04072036083808360C0E9032342
:10128000012303757047836819B143F0010383603C
:10129000704723F00103FAE7044B5A6818B142F48F
:1012A00000025A60704722F40002FAE7002701406A
:1012B0001D2970B51BD90725A1F11E06C46D06EBCB
:1012C0004606B54024EA050403FA06F62643C66539
:1012D000062A38D81F24013A036C02EB820294409C
:1012E00023EA040301FA02F21A43026470BD1329CF
:1012F0000DD90726A1F11405C46805EB4505AE40DC
:1013000024EA060403FA05F52543C560E0E7092948
:101310000DD90726A1F10A04056904EB4404A6408F
:1013200025EA060503FA04F42C430461D0E70726F6
:10133000446901EB4105AE4024EA060403FA05F6D0
:1013400026434661C4E70C2A0CD81F24073AC36B16
:1013500002EB8202944023EA040301FA02F21A43E8
:10136000C263C3E7122A0CD81F240D3A836B02EB29
:101370008202944023EA040301FA02F21A438263D0
:10138000B4E7182A0CD81F24133A436B02EB8202ED
:10139000944023EA040301FA02F21A434263A5E7E8
:1013A0001F24193A036B02EB8202944023EA0403E0
:1013B00091401943016399E7836843F08043836058
:1013C0007047806D80B270470368194214BF0120D6
:1013D00000207047C943016070470000044B1A6841
:1013E00018B142F002021A60704722F00202FAE7D6
:1013F000003C0240044B1A6818B142F004021A6023
:10140000704722F00402FAE7003C0240044B1A68DD
:1014100018B142F008021A60704722F00802FAE799
:10142000003C0240044B5A68D20741BF034ADA60CD
:10143000034ADA60704700BF003C0240EFCDAB8941
:1014400005040302024A536843F0010353607047E6
:10145000003C0240014B9861704700BF003C0240D5
:10146000084B9A69D10709D49A69D20508D49B69B7
:1014700013F4F05F14BF032004207047012070476D
:1014800002207047003C0240042313B504468DF847
:101490000730FFF7E5FF8DF807009DF80730012BB7
:1014A0000AD11CB905238DF8073007E0FFF7D8FFF4
:1014B000013C8DF80700F0E7002CF3D09DF8070001
:1014C00002B010BD10B504464FF40040FFF7DCFF3A
:1014D000042804BF0023236010BD000038B5044673
:1014E0004FF400400D46FFF7CFFF04280BD1064A0A
:1014F0004FF40040536823F4807353602560BDE8C7
:101500003840FFF7C1BF38BD003C024038B5044643
:101510004FF400400D46FFF7B7FF04281BD135B14B
:1015200025704FF40040BDE83840FFF7ADBFFF2302
:1015300024F0030504F003042968E40003FA04F42A
:1015400021EA04042846FFF7BDFF21462846BDE8EE
:101550003840FFF7C3BF38BD2DE9F0430022012713
:1015600003250E6807FA02F333EA060431D14FEA85
:10157000420C05FA0CF4E44391F804E0D0F8009032
:101580000EFA0CF804EA09090EF1FF3E48EA0908D0
:10159000BEF1010FC0F8008011D8D0F808E004EACD
:1015A0000E0E4C7904FA0CF444EA0E04846084882C
:1015B00024EA03048B7993409BB223438380C3685E
:1015C00005FA0CF423EA0404CB7903FA0CF3234361
:1015D000C3600132102AC5D1BDE8F08310B50F24D5
:1015E00001F00703C90800EB8100016A9B009C40E1
:1015F00021EA04010162016A9A400A43026210BDB5
:10160000204B10B59A6802F00C020C2A30D8DFE8A3
:1016100002F02F2F2F2F072F2F2F072F2F2F2000D4
:10162000194B184A036093681849C3F30313CC5C41
:101630000368E34043609468C4F302240C5D23FA1A
:1016400004F484609268C2F3C2228A5CD340C3600F
:1016500010BD99680E4CC1F383419A68615C9B6828
:10166000094BC2F381524B430132B3FBF2F3D8E78B
:101670004FF400425B68C3F34233013302FA03F3D1
:10168000CFE700BF003802400024F400FC01002036
:101690000C020020054B19B1D9690143D96170478B
:1016A000DA6922EA0002DA61704700BF00380240BE
:1016B000054B19B1196A0143196270471A6A22EA87
:1016C00000021A62704700BF00380240054B19B192
:1016D000596A0143596270475A6A22EA00025A6203
:1016E000704700BF00380240054B19B159690143EA
:1016F000596170475A6922EA00025A61704700BF77
:10170000003802404309012B054B00F01F000CBFBD
:101710001B685B6B23FA00F000F00100704700BF0C
:1017200000380240024A536B43F0807353637047A2
:101730000038024030B50D460446028AEB8892B26A
:1017400022F440521A43898902828389288923F42A
:10175000B052AB8822F00C020343688985B0034382
:101760001343A381A38A68469BB223F440730B43BF
:10177000A382FFF745FFDDE90213154A944208BF33
:1017800019461923A2894B43296810044CBF49000C
:101790008900B3FBF1F16425B1FBF5F3A2891801CF
:1017A000120405FB13130BD5DA003232B2FBF5F24B
:1017B00002F0070242EA00039BB2238105B030BD6C
:1017C0001B013233B3FBF5F303F00F030343F3E7DD
:1017D00000380140838919B143F400538381704775
:1017E00023F400531B041B0CF8E7C1F308018180AC
:1017F00070478088C0F30800704701F01F0310B5E0
:10180000C1F342140121012C01FA03F105D10C307E
:1018100003683AB11943016010BD022C0CBF1030AF
:101820001430F5E723EA0101F5E70388194214BFF4
:101830000120002070470123C1F3421210B5012A94
:1018400001F01F0403FA04F30DD1828913400288CA
:1018500092B26BB10123090A03FA01F10A4214BFE3
:101860001846002010BD022A0CBF028A828AEDE7CA
:101870001846F7E70123090A8B40DB439BB203803C
:10188000704700002DE9F3411F46002304460E4631
:10189000019315461AB9012002B0BDE8F08140F667
:1018A000FF7301934FF40031204600F014FD00282F
:1018B00052D10121204600F0DEFC4FF2FF7120469C
:1018C00000F0F2FC0121204600F0BFFC40F6FF735F
:1018D000DFF8B88101934146204600F0F1FC002872
:1018E00041D039460122204600F0D0FC40F6FF737B
:1018F000614F01933946204600F0EDFC002838D0B6
:10190000012D42D10021204600F0B5FCF1F7D2F9BB
:1019100029462046238B00F0A3FCF1F7EBF940F6B3
:10192000FF73564D01932946204600F0D4FC30B396
:10193000204600F0B6FC307040F6FF73504D019326
:101940002946204600F0C7FC0028A4D0019B5A1E5F
:101950000192002BF4D104E0019B5A1E0192002B4E
:10196000A0D1002098E7019B5A1E0192002BB2D112
:10197000F7E7019B5A1E0192002BBBD1F1E7019BB7
:101980005A1E0192002BCED1EBE7022D25D1F1F7A3
:1019900091F94FF40061204600F086FC00212046BA
:1019A00000F069FC238BF1F7A5F940F6FF73354D84
:1019B00001932946204600F08EFC40B101212046CB
:1019C00000F04EFC238A3370238A7370B4E7019BC6
:1019D0005A1E0192002BECD1C3E740F6FF77033D7E
:1019E000238BDFF8A0803544AE4201972CD1254EE1
:1019F0003146204600F06FFC90B30021204600F0F5
:101A00003AFCF1F757F9204600F04BFC0121287011
:101A1000204600F025FCF1F76DF9204600F041FC6E
:101A200040F6FF73184E687001933146204600F06F
:101A300047FCD8B1204600F034FCA8707CE7019B3D
:101A40005A1E0192002B8CD04146204600F043FCE8
:101A50000028F4D0204600F024FC06F8010BC3E770
:101A6000019B5A1E0192002BC2D17AE7019B5A1E9C
:101A70000192002BD9D174E7020000104000001041
:101A800010000010040000104000030001000300DB
:101A90002DE9F3411D46002304460E4601931746E7
:101AA0001AB9012002B0BDE8F08140F6FF7301933E
:101AB0004FF40031204600F00EFC002847D10121F0
:101AC000204600F0C2FB40F6FF73DFF8E880019388
:101AD0004146204600F0F4FB00283FD02946002272
:101AE000204600F0D3FB40F6FF732E4D01932946AC
:101AF000204600F0E5FB002836D03546204615F894
:101B0000011B3E4400F0CBFB40F6FF77DFF89880E6
:101B1000B542019733D1244D2946204600F0DBFB26
:101B2000002838D02046012100F09AFB40F6FF73D0
:101B30001E4D1F4C01932946204600F0CCFB002887
:101B4000AFD0019B5A1E0192002BF4D104E0019BFF
:101B50005A1E0192002BABD10020A3E7019B5A1E15
:101B60000192002BB4D1F7E7019B5A1E0192002B82
:101B7000BDD1F1E7019B5A1E0192002BECD04146EA
:101B8000204600F0A8FB0028F4D015F8011B2046E1
:101B900000F085FBBCE7019B5A1E0192002BBBD1D4
:101BA000DAE700BF820007000400001010000010F8
:101BB00000540040010003002DE9F3411D460023BD
:101BC00004460E46019317461AB9012002B0BDE83B
:101BD000F08140F6FF7301934FF40031204600F08E
:101BE0007AFB002838D10121204600F02EFB40F678
:101BF000FF73DFF8E48001934146204600F060FB6C
